:020000040000fa
:08000000c07d040001000000b6
:020000040000fa
:100200001206040000000000400604000000000088
:100210006fe62100807f22000001880000000000be
:10022000050007000c000700be37020000000000b8
:100230000040da000000fe004440a900c0072a0088
:100240000000e0000300320010002000a001880040
:100250004440a80000000600406f2d00010020006f
:100260001600370062004000e080480091018800dd
:100270009001ba0062004000e080480091018800cf
:100280009002ba0062004000e08048000002eb00eb
:100290006028e10005003a008301e900070033000f
:1002a000038009000059eb00040037006128e100d9
:1002b000010032000082eb00050007009101880078
:1002c0001001ba000200e000e6ff3a00000005005d
:1002d000910188008002780062004000e0804800c0
:1002e0003559ba008301e900080032002559ba00e7
:1002f0008301e900050032000400e000f4ff320051
:1003000015d9ba008301e900f1ff3a0000000600a8
:100310001004b100070035009001b1000400340062
:100320007000b100030035009001b10001003c00f5
:100330001000050000000500ea874700889fbe0006
:100340008a9fbe008c9fbe008e1f780080067800ba
:10035000010678008204780000047800010037006c
:100360000804e8001800fb00880207000000e00015
:10037000fbff3a0098407800d0c2b30080cf500015
:100380000400320000c0e900d0ef9f0080cf500091
:1003900002003a00d1ef9f000804e8000900e000e5
:1003a00046003500e18f5400440032004002200036
:1003b000808f540041003c000900e0000d00340033
:1003c000f08f54001a003a0000c3b300984f100099
:1003d00017003a009840900080c7b30080cf5000cb
:1003e0001200320080c5b30080cf500010003a00e8
:1003f0000e00370000c3b300984f10000200320017
:10040000a90020000a0037009840900080c7b30080
:1004100080cf5000040032008900200080c5b30066
:1004200080cf500002003a00090120000884e80053
:10043000d8b79f0000c3b300984f100002003a00e5
:10044000d84f1000feff32006055b8000807780052
:100450000e003700fab79f008bbf9f00e05f2100be
:1004600000425200c4ef9f006149b9000a00be007b
:10047000001407004fea97000401fb00cf91de0053
:1004800000054100818549000804e8001800fb00d0
:10049000400107008000780009017800e05f21003a
:1004a00028020700000278000000e000e9ff3a009f
:1004b0005fb09700880f500005003a000c00e00084
:1004c000010032000d0e78006000b80027003700f0
:1004d0008e00540030622100694078000000fb006b
:1004e00000805000170033004240a9000f003c007c
:1004f0004fe997000200fb00cf80de0000005500ae
:1005000081805d00800f5500818f5d0007003900fc
:100510006149b900281007007fb197008fb9970093
:10052000820f5000838f5800060032002002200006
:1005300020bf88000085eb008085eb00b3c2b300cc
:10054000d3ef9f00d0c2b3005fea9700804f520004
:1005500002003a0060051500e0851d000c00e00077
:1005600001003200080e78000a00be004f07780034
:100570004f06be004f05be004f04be00af00b100e5
:1005800000000600f8874700889fbe008a9fbe00d3
:100590008c9fbe008e1f7800c0b79f0001047800ba
:1005a0000206be000005780078805700ff010700b2
:1005b000680760000030a100e10f500043003a00de
:1005c000cfb0970024002000c3fd2f008f81410091
:1005d000080178000a00780076020700800578009c
:1005e0000000e00007003a006000b8006011b800a9
:1005f000d0b79f00e1b79f00f2b79f0083bf9f0075
:100600002d0037006400b800c2fd2f000f0141002b
:10061000000041001000be00e20e0700d0b79f00ae
:10062000e1b79f00f2b79f0083bf9f000b05e90071
:100630004240a900200034006450b800c2fd2f00e1
:100640000f014100000041001000be00e00f50000b
:10065000e08f5800150032000a8455006844b80045
:10066000e274210002044400ce0e07000002be0026
:100670000203be003800be002801be000f100700b4
:100680000002be000203be005fb09700efb097000b
:100690007fb197008fb99700450f0700d0b79f0033
:1006a000e1b79f00f2b79f0083bf9f000a05e900f2
:1006b0004240a900e0ff3c006fa89700ffa8970008
:1006c0000c0240008d82480045003700e20f5000c8
:1006d00049003a00cfb0970000027800c3fd2f0018
:1006e0008f814100080178000a0078001703070095
:1006f000800578000000e00007003a006000b800c4
:100700006011b800d0b79f00e1b79f00f2b79f001b
:1007100083bf9f002d0037006400b800c2fd2f008a
:100720000f014100000041001000be009d0e0700b7
:10073000d0b79f00e1b79f00f2b79f0083bf9f0033
:100740000b05e9004240a900200034006450b800c5
:10075000c2fd2f000f014100000041001000be004b
:10076000e00f5000e08f5800150032000a84550059
:100770006844b800e275210002044400890e0700b5
:100780000002be000203be003800be002801be0009
:10079000ca0f07000002be000203be005fb0970050
:1007a000efb097007fb197008fb99700000f070057
:1007b000d0b79f00e1b79f00f2b79f0083bf9f00b3
:1007c0000a05e9004240a900e0ff3c006fa997003c
:1007d000ffa9970076805700d40307000c02be00e3
:1007e0005fb09700efb097007fb197008fb9970087
:1007f0005e04070013003700e30f500004003a00c6
:100800006000b8000200200003ff27000600370048
:10081000e40f500009003a00f0ff2f00f1ff2f0015
:10082000f2ff2f00f3ff2700d0b79f00e1b79f0032
:10083000f2b79f0083bf9f00060037006000b8003a
:100840006011b800d0b79f00e1b79f00f2b79f00da
:1008500083bf9f005fb09700efb097007fb1970014
:100860008fb997000e00e0000100320003f0a200f3
:100870004f0778004f06be004f05be004f04be0074
:100880008f01b10000000600800178000200e00046
:10089000070032001104e00005003200b159780071
:1008a0000201e900020032001104e000fbff3a00ff
:1008b0000200e000030032008059eb000201e90071
:1008c000fdff3a00000006001004e0000a003200bc
:1008d000010178001104e000050032009041780029
:1008e00092cf5100050032005204e000fbff3a00b5
:1008f0005004e000f6ff3a000000eb0000000600a4
:10090000800178000200e000030032008159780085
:100910000201e900fdff3a000000060080007800b7
:100920001004e000020032005104e000feff3a0033
:1009300000805000000006000400fa00889fbe00fe
:100940008a9fbe008c9fbe0080bf9f0091bf9f000a
:100950000206be00cd1207000001be000004be006a
:100960000c00be00c31207000fb997009fb9970093
:1009700000055100818559000800be000a01be0033
:100980004f06be004f05be004f04be000080fa00b7
:1009900000000600800078001104b100030035005b
:1009a0009101b10001003c000050a00000000600d1
:1009b00080027800800178001004e0000b00320013
:1009c0000101780012427800058051000404e00023
:1009d00007003200934f1200020032000201e800cb
:1009e000f8ff37005304e000f5ff3a00058051009e
:1009f00000000600800178001004e0000a003200c8
:100a0000010178001104e000050032001042780076
:100a1000924f5200040032005204e000fbff3a0003
:100a20005004e000f6ff3a0003005000000006000a
:100a3000800178000200e00003003200b159780024
:100a40000201e900fdff3a00000006000001780005
:100a5000314978003204e000fdff3a000000060052
:100a6000800078001106b100030035009101b1004b
:100a700001003c000050a100000006000200fa0046
:100a8000889fbe008a9fbe008c1f780000057800fa
:100a900081047800020678000100e00001003a00bd
:100aa000ec8457000a047800010037000804e800cd
:100ab0001800fb00b50007000000e000fbff3a0053
:100ac00098407800d0c2b30080cf500003003200bd
:100ad000bbc2b3008bcf500002003a0081457800c2
:100ae0000804e8000c0178000800be0012fe0700b0
:100af0000001be00990f540001003a008a0c7800f2
:100b0000990f550003003a00e00f5100e08f5900a3
:100b10000e003a00b0c2b30080cf550003003a0087
:100b2000e00f5100e08f590008003500d0c2b3003b
:100b300080cf55000f003a0000002000010028007f
:100b4000800f5100818f59000a00360020022000da
:100b500020bf880002002000030028006b404000f6
:100b600080cf550008003200f2ff2f00f3ff27006e
:100b700005003700d0c2b30080cf550002003a0014
:100b800060011100e08119000200be004f067800ec
:100b90004f05be004f04be000080fa0000000600b2
:100ba000800278000200e0000e00320095417800db
:100bb0001142780084cf5100030032000080eb0026
:100bc00009003900100005000000eb000304e000fc
:100bd000050032008502e8008100e8000201e9001a
:100be000f2ff3a000000eb00000006000003b10035
:100bf000030035009000b10001003c00100005002a
:100c00000000050090cf1000050032001004e00045
:100c100001003a0000000500d0cf1000fbff3a00b1
:100c200000000600881f78000204780080ff07009b
:100c3000080040004f047800000006000000fa00a1
:100c4000881f7800000478003fb99700ea815700b8
:100c50008000780020612000f30307008000780006
:100c60000000e000020035000040eb0000f47800d6
:100c7000010078004f0478000080fa0000000600b0
:100c8000889fbe0000047800820478001001900064
:100c9000890f5100010031008204780018007800ab
:100ca0000901780062ff0700188c440018009000ca
:100cb0000900500010049800080078004f04be009e
:100cc000000006000400fa000100e00004003a0001
:100cd0000f80e900e0bf9f000008eb000300370031
:100ce000e0bf9f008100e900f1bf9f00e480570052
:100cf00000642000cc030700efb897008048eb00a9
:100d00000080fa00000006000200e0000b00320044
:100d10001042780091417800834f52000300320066
:100d20000080eb0006003900100005000000e8001c
:100d30008100e8000201e900f5ff3a000000eb0045
:100d4000000006000200e0000500320090cf100015
:100d5000040032000000e8000201e900fbff3a0055
:100d60000000eb000000060001017800000278009e
:100d7000110009000200d8000002fd000491b90032
:100d8000820250000400be00000006006900e1007d
:100d9000040035006d00e100030034000002b100e2
:100da000010032000000050010000500889fbe0011
:100db0008a9fbe008c1f78000006780081057800ad
:100dc000100478000005eb00010037000804e8007b
:100dd0001800fb00edff07000000e000fbff3a00f9
:100de00098407800d0c2b30080cf500002003a0093
:100df0008a00200003003700b0c2b30080cf50004b
:100e000001003a000804e80098407800e2c6b30008
:100e100082cf500003003200e3c4b30083cf500000
:100e20001f003a00d840780010c6b30080cf5000b1
:100e30000300320010c4b30080cf50002a003a00f3
:100e4000d840780082cf500003003200e0c4b300e5
:100e500080cf500024003a000804e800880478009d
:100e60004a00200080c2b300984f100007003a00eb
:100e70005900fb00210407000000e000fcff3a00dd
:100e8000f0c5b300994f1000f9ff320090c2b300d3
:100e9000994f10003c003a000904e8003a0037007e
:100ea00090c6b30080cf50000300320090c4b3005e
:100eb00080cf500038003a0058407800824f5000f0
:100ec00002003200834f500007003a00d8407800fb
:100ed00060c6b30080cf50000600320060c4b3008b
:100ee00080cf5000030032001c0478000005eb00a6
:100ef000250037003a00b300d840780093c6b3000d
:100f000083cf50000300320090c4b30080cf500064
:100f10001d003a008800e80011417800e0c6b300e7
:100f2000804f510003003200e0c4b300804f5100f5
:100f300015003a0051417800834f51000300320000
:100f400090c4b300804f51000f003a005141780027
:100f500040c7b300804f51000300320040c5b300ca
:100f6000804f510008003a005141780090c7b3000b
:100f7000804f51000300320090c5b300804f5100f4
:100f800001003a000104e8000b00e0000300320019
:100f9000880d7800010037000a00a000080e7800d4
:100fa0000a0078004f0678004f05be004f04be00cf
:100fb00000000600e6874700889fbe008a9fbe00ab
:100fc0008c9fbe008e1f7800f0b79f00010578004f
:100fd00082bf9f0003067800830478006920b9006f
:100fe000000478008006eb0000c3b3009a4f1000a5
:100ff00003003a001d002000da4f1000fdff320010
:101000008005eb00000eeb003c167800280037004e
:10101000888f550016003d00920020001100090045
:101020008205d800010078000000e00003003a00cb
:10103000e4844400800ceb00b91478001900be0071
:10104000a2002000030020000a1107001a417800c6
:101050000201fb00cf91de000000410081804900c9
:101060000003b1000180b100808cbe000d0037008c
:1010700010002000010020001c0e40005c9648007b
:10108000888f550008003a0040c3b3009a4f100003
:10109000050034001200200003002000990c4100dc
:1010a000d99449008b05e8000a05e8001d002000de
:1010b0001a00fb00cdfe07000000e000d4ff3a005c
:1010c0008b0f540001003d0088057800e0c2b3009a
:1010d0009a4f100001003a000a05e8000b00e000fa
:1010e00029003a0000c3b3009a4f100026003a00ce
:1010f0000081eb008081eb001c0e41005c964900f2
:101100001d002000da4f1000f9ff32001e003700ea
:10111000888f55001a003d00920020001100090040
:101120008205d800010078000000e00003003a00ca
:10113000e4844400800ceb00b91478001900be0070
:10114000a200200003002000ca1007001a41780006
:101150000201fb00cf91de000000410081804900c8
:101160000003b1000180b100808cbe008b05e80057
:101170000080eb008080eb001c0e40005c96480075
:101180000a05e8001d0020001a00fb0097fe07007a
:101190000000e000deff3a0092002000110009008c
:1011a0008205d800010478000800e0001000320039
:1011b000690414001902be00e00f5200e08f5a00cb
:1011c000070032006440b80022772100020040008e
:1011d0001001be000400be00a6100700808cbe00f7
:1011e000888545006140b9001c1e10001c9618003f
:1011f000e88f5500100034001900be00e00f5000c9
:10120000e08f58000c003a00e9855500900020005e
:10121000010020001c0e40005c964800e48454004d
:10122000e88f5500040034001900be00e00f5000a4
:10123000e08f5800f4ff32000d00e0003100320072
:101240009a40780050c6b30080cf500003003200af
:1012500050c4b30080cf50002a003a00da40780032
:10126000b0c2b30080cf50000400320000477800c5
:1012700000c0e80080cf500002003a00014778002b
:101280000a05e8006044b8008006eb001200370051
:10129000f00f2e00515f2000800f5400818f5c0002
:1012a0000b003c00a2002000030020000800be004c
:1012b000701007001a4178000201fb00cf91de0098
:1012c00000044100818449000803b1000980b10095
:1012d0000a05e8001d0020001a00fb0043fe07007d
:1012e0000000e000eaff3a00d0c2b300804f570090
:1012f00002003a0060041400e0841c001c0e44004c
:101300005c964c008fb897000100e00006003200a8
:10131000ffb097000d00e000010032008a00780065
:101320000fb9970001097800920020001100090010
:101330008205d8004f0778004f06be004f05be005b
:101340004f04be006f00b10000000600e6874700b2
:10135000889fbe008a9fbe008c9fbe008e1f7800b3
:10136000f0b79f000105780082bf9f0083057800d9
:10137000030478006720b900800478008006eb0041
:1013800000c3b3009a4f100003003a001d00200074
:10139000da4f1000fdff32000006eb00800deb007d
:1013a000bb1578002e003700890f560019003d004c
:1013b00072002000811f7800110009000206d80089
:1013c00001007800cf0078000000e00003003a0040
:1013d00064044400000ceb00381478001801be00cf
:1013e0004418dd00cc11de00830170004411dd00e3
:1013f000a06d210000805000116f210060c07800b6
:101400000000fb00cf80de00001c41000194490079
:101410001000370012002000030020009b0d410047
:10142000db954900890f56000b003a00a06d2100a2
:1014300000805000116f210060c07800e74f50001d
:10144000050034001000200001002000180c4000ae
:10145000589448000c06e8000a05e8001d0020002a
:101460009a00fb0062012000a06d210035fe0700fc
:10147000800078000000e000cbff3a008c8f540021
:1014800001003d0009067800e0c2b3009a4f100049
:1014900001003a000a05e8000c00e0002c003a00c8
:1014a00000c3b3009a4f100029003a000081eb00fe
:1014b0008081eb009b0d4100db9549001d00200061
:1014c000da4f1000f9ff320021003700890f560073
:1014d0001d003d0072002000811f780011000900ee
:1014e0000206d80001007800cf0078000000e0007c
:1014f00003003a0064044400000ceb003814780048
:101500001801be004418dd00cc11de00830170001c
:101510004411dd00a06d210000805000116f2100fa
:1015200060c078000000fb00cf80de00001c41009e
:10153000019449000c06e8000081eb008081eb007b
:101540009b0d4100db9549000a05e8001d002000c5
:101550009a00fb0062012000a06d2100f9fd070048
:10156000800078000000e000d8ff3a007200200000
:10157000110009000206d800010078000000e00018
:101580000d003200670010006402b9001801be00af
:101590000402e90003003300020141008381490095
:1015a000fbff3700028cbe0000064600cf80de0045
:1015b0009b1d10009b951800e60f5600100034008c
:1015c0001800be00e00f5000e08f58000c003a00f9
:1015d0006706560070002000010020009b0d4000af
:1015e000db95480064045400e60f56000400340004
:1015f0001800be00e00f5000e08f5800f4ff3200ea
:101600001b00be004209dd00ce00de00810071003b
:101610004200dd00808dbe000d00e0003100320090
:101620009a40780000c7b30080cf5000030032001a
:1016300000c5b30080cf50002a003a00da4078009d
:10164000b0c2b30080cf50000400320000477800e1
:1016500000c0e80080cf500002003a000147780047
:101660000a05e8006044b8008006eb00120037006d
:10167000f00f2e00515f2000800f5400818f5c001e
:101680000b003c00a2002000030020000800be0068
:10169000780f07001a4178000201fb00cf91de00ad
:1016a00000044100818449000803b1000980b100b1
:1016b0000a05e8001d0020001a00fb004bfd070092
:1016c0000000e000eaff3a00d0c2b300804f5700ac
:1016d00002003a0060041400e0841c009b0d4400ea
:1016e000db954c008fb997000300e0000600320044
:1016f000ffb097000d00e000010032008a00780082
:101700000fb897000108780072002000110009004e
:101710000206d8004f0778004f06be004f05be00f6
:101720004f04be006f00b10000000600881f780063
:101730008a9fbe00000478000205be0030019000c0
:101740000200d000c500de00f07f2000808f500036
:101750000c003a006f00610008003a002800900079
:101760000000e00005003a00180090000000e000d2
:1017700002003a001800e0001c00320020002000a7
:101780005d0037000100e00006003a000800780024
:10179000e8010700800078000000eb000100e00095
:1017a00055003c006108b9000a0540008b854800df
:1017b000e07f2000800f5500e08f5d000d003400b9
:1017c000380090006022b8000600200007ff2f00bc
:1017d0000000e000030035006022b8000600200091
:1017e00007ff2700049cbe000694be0010002000e6
:1017f00041003700b8009000e00f5500e08f5d0019
:1018000005003400f000280000806000c450dd00b6
:101810000100700036003700000028008082600060
:101820006f8060000040a000300498006105550002
:10183000e0855d00c0fc2f00f1ff2f00800f5500f8
:10184000818f5d0006003d00350498000000eb002c
:101850002004980010049800000ceb0026003700cc
:101860000a027800f00f45000b003c0018009000c1
:10187000000c7800280090001004980038009000b8
:10188000200498000000eb00300498007002420031
:10189000f00f4200f5ff34000402ea0012003200ab
:1018a000180178000411de00f00112001800900009
:1018b0008300dd00010c71000400de0028019000af
:1018c0008310dd0001007000100498000411de0098
:1018d000380090008301dd000301710022049800ac
:1018e0000400de003004980038009000050070000d
:1018f000300498000080eb004f05be004f047800d4
:10190000000006000200fa00889fbe008a9fbe0009
:101910008c1f7800000678000404be000605be0097
:10192000800078006c805700d50107003c00be00a5
:101930002c01be000802be000a03be005f0b0700b8
:10194000009ebe000296be002fb99700cf91de0028
:101950000c00780075ff07004f0678004f05be00a9
:101960004f04be000080fa00000006001800fa00d4
:10197000889fbe008a1f780090b79f00a1b79f0084
:10198000b2b79f00c3b79f000404be00e00f52002f
:10199000e08f5a009c0032006022b8006033b8002b
:1019a000000b07000000e000970032006000b80064
:1019b0000200200003ff2300d0b79f00e1b79f0083
:1019c000f2b79f0083bf9f00e00f5400e08f5c00e0
:1019d00048003d0060041400e0841c000005eb009a
:1019e0001a0032000808a300100032006850b80046
:1019f00082642100020040003002be002003be00cd
:101a00005fb09700efb097007fb197008fb9970054
:101a10002a0b07000002be000203be00d4b79f00dd
:101a2000e5b79f00f6b79f0087bf9f008904d100ec
:101a30000884d3000a05e800e00f5400e08f5c0042
:101a400002003200e70f5500e6ff36005fb2970054
:101a5000efb297007fb397008fbb97006000b8008c
:101a60000200200003ff2300d10907000002be008e
:101a70000203be007e805700a2ff07000005780029
:101a80000000e00059003d00e00f5400e08f5c00d2
:101a900056003200836821003302be002303be00db
:101aa0006000b8000200200003ff2300c009070007
:101ab00090bf9f00a1bf9f00b2bf9f00c3bf9f0008
:101ac0001fba9700afba97003fbb9700cfbb9700f4
:101ad0007e8057008bff0700000578000000e000c3
:101ae00042003d0061045400e0845c00f4ff3a00d1
:101af0003e003700e00f5400e08f5c003b003400f4
:101b00000005eb000808a300100032006850b80080
:101b100082642100020040003002be002003be00ab
:101b20005fb09700efb097007fb197008fb9970033
:101b3000e20a07000002be000203be00d4b79f0005
:101b4000e5b79f00f6b79f0087bf9f008984d1004b
:101b50000884d3000a05e800e00f5400e08f5c0021
:101b600002003400e70f5500e6ff36005fb2970031
:101b7000efb297007fb397008fbb97007e8057002e
:101b800060ff0700000578000000e00017003d003e
:101b9000e00f5400e08f5c001400340081682100e5
:101ba0005101be004100be00d0b79f00e1b79f00c9
:101bb000f2b79f0083bf9f005fb29700efb297001c
:101bc0007fb397008fbb97007e8057004dff0700c3
:101bd000000578000000e00004003d0061045400ae
:101be000e0845c004240a900f3ff3c0000012000bb
:101bf0000a00e00003003200e10f550002003a0045
:101c0000800020004c0107001fb09700afb0970084
:101c10003fb19700cfb197004f0578004f04be0049
:101c20000080fa00000006006200fa00889fbe00f3
:101c30008a9fbe000004be00020578008300780081
:101c40006a80570047010700f88f9f0089979f001f
:101c50000000eb00909f9f001a80fb008005fb00b6
:101c60000000ea00cf04de000904780050022000e2
:101c7000808f550001003a000904e9000800e000e7
:101c80000c0034000f909700080178008a0078005b
:101c9000ff8997000300010080979f008080eb0080
:101ca0000000e000900032001f98970008004000fc
:101cb000909f9f000905450050022000808f55002d
:101cc000040032000b00e000e3ff3a009f98970009
:101cd000850037000000eb00f0979f00e0979f0021
:101ce000d0979f00c0979f00b0979f00a0979f003c
:101cf000b09f9f0009003700c07a2100008050008b
:101d00000000d000217b210001004000bf98970017
:101d100090807000b19f9f000a05e8009a00fb00c8
:101d2000c07a2100b7fb0700800078000000e000c7
:101d3000f1ff3a00a0c2b3009a4f10000e003a0023
:101d40003fb897000080e900b0bf9f001000780006
:101d5000a09f9f000000e00005003d000000ea0099
:101d6000a09f9f003f9897000020a000b09f9f0079
:101d70000a05e80011003700a19f9f000b00370003
:101d8000af989700f0ff2700808f500006003200c8
:101d90006a09b9001a00fb000200400001fd2f0093
:101da00001004000a09f9f000a05e8001a00fb0008
:101db0008efb07000000e000f1ff3a00e0c2b30034
:101dc0009a4f1000030032000080eb00809f9f00bc
:101dd0001c003700a0c2b300da4f100007003a0021
:101de0003fb897000080e900b0bf9f001000780066
:101df000809f9f000a05e800120037000000eb00fa
:101e0000809f9f000b0037008f989700f0ff2700fe
:101e1000808f5000060032006a09b9001a00fb00ea
:101e20000200400001fd2f0001004000809f9f0044
:101e30000a05e8001a00fb006cfb07000000e00048
:101e4000f1ff3a009a00fb00c0e521006dfb07009e
:101e50008040eb000000e00001003200ba40780052
:101e6000817f9f0080c6b30080cf500004003a00fd
:101e70009acf100002003a00664050000700370079
:101e80008f789700c0c6b30080cf500005003a009d
:101e90009acf100003003a0065404000807f9f0009
:101ea0000a05e800a0fb2f00008447003a01fb0070
:101eb00088017800ea80570060f92f000f00400089
:101ec000780107000000e00006003a008800780072
:101ed00060f92f000f004000a40007000000e000a0
:101ee0005dff3d008080eb00010078004f05be00e3
:101ef0004f04be000080fa00000006000003b1009d
:101f00000b0035009000b100080034008000b100e3
:101f1000070035009001b100040034007000b100ea
:101f2000030035009001b10001003c0010000500e5
:101f30000000050000027800300090000100280039
:101f400001036000150020006f006000300298005f
:101f500008003a00240090000000e00005003a006c
:101f6000140090000000e00002003a001400e000bd
:101f70003e003200340090000000e0000b003a0008
:101f80002400900030029800140090002002980075
:101f90001400780010029800000aeb00f082520052
:101fa000340090000000e000f5ff320034009000a3
:101fb000ef0f500014003e008001d000a4009000fc
:101fc0004f08de0080817100330298008100d0004c
:101fd000140190004f10de008080700021029800f4
:101fe0000201d000940078004f08de00000171006b
:101ff00012029800010ad0008502e900030078006f
:10200000ef8f5100ecff3600b4019000ff8f5100bc
:10201000130036001401d10014009000cf00dd0041
:10202000010a71000000d100a40090004f09dd00fa
:1020300002007000100298008100d1004f18dd00ee
:1020400080807000210298000300d10030029800c7
:102050008502e80080017800ff0f5000edff3e0090
:10206000340090006f00600030029800340090004f
:10207000060070003002980005007800000006009d
:10208000889fbe0080047800010478003100900031
:102090000000d0004501de00f07f2000800f5100dd
:1020a00010003a00800ceb00310090006f006000df
:1020b00008003a00210090000000e00005003a000e
:1020c000110090000000e00002003a001100e00062
:1020d0000200320020002000150037001000200010
:1020e000130037000200e00005003c00010078000a
:1020f00090ff0700000178000000e0000a003c00ab
:1021000038009000f10028000100600001fe23006b
:10211000010070003004980020c02f00800c4100a6
:102120000080eb0002003700800ceb000000eb00a9
:102130004f04be00000006008000780065006000cb
:10214000030032001002200020bf880000000600bb
:1021500078806000020032002002200020bf88004a
:102160000000060001087800000006000400fa00e4
:10217000889fbe008a9fbe008c1f780000047800f4
:102180000106780070089000f800900001005000ef
:10219000880890000100500098089000010050004d
:1021a000a808900001005000b808900001005000fd
:1021b000c8089000810550000002220090bf9f00d7
:1021c00000032300a0bf9f00081090000028a30078
:1021d00018003a000b00e000160034000b057800f0
:1021e0008a047800e20f5500010036002900200023
:1021f0000900e0000c00340058009000c801900075
:1022000009017800ee805700030001005004980097
:102210008080eb000000e0009c0032006808900025
:1022200009004000600c9800090555004240a900d3
:10223000ebff3c00780190000200e0000c0034004d
:1022400058009000c80190008c0078000300010045
:10225000500498008080eb000000e0008b0032000a
:1022600068089000f800900001004000600c9800a1
:10227000080890000000e000160034000005780017
:102280008a047800e20f5500010036002900200082
:102290000900e0000c00340058009000c8019000d4
:1022a00009017800ec8057000300010050049800f9
:1022b0008080eb000000e0007400320068089000ad
:1022c00009004000600c9800090555004240a90033
:1022d000ebff3c00180990000200e0000c00340005
:1022e000e800900058009000c80190000300010031
:1022f000500498008080eb000000e0006300320092
:10230000680890009808900001004000600c980058
:10231000280890000000e000160034000005780056
:102320008a047800e20f55000100360029002000e1
:102330000900e0000c00340058009000c801900033
:1023400009017800ec805700030001005004980058
:102350008080eb000000e0004c0032006808900034
:1023600009004000600c9800090555004240a90092
:10237000ebff3c00380990000200e0000e00340042
:10238000e8009000180890008080400058009000fd
:10239000c801900003000100500498008080eb0009
:1023a0000000e0003900320068089000b808900092
:1023b00001004000600c9800480890000000e00018
:1023c00016003400000578008a047800e20f5500fa
:1023d00001003600290020000900e0000c00340054
:1023e00058009000c801900009017800ec80570067
:1023f00003000100500498008080eb000000e00022
:10240000220032006808900009004000600c98002b
:10241000090555004240a900ebff3c000810900060
:102420000028a300180032000b00e0001600340062
:102430000b0578008a047800e20f55000100360091
:10244000290020000900e0000c0034005800900032
:10245000c801900009017800ee80570003000100d8
:10246000500498008080eb000000e000070032007c
:102470006808900009004000600c980009055500ac
:102480004240a900ebff3c008000eb000100780017
:102490004f0678004f05be004f04be000080fa00d2
:1024a00000000600889fbe008a1f780000047800a4
:1024b0000102780002457800830478000200fb00e6
:1024c000cf80de005002b1000180b1003205200053
:1024d000820f5000e08f58008c013e000060010028
:1024e00084013700890137008801370087013700f0
:1024f00086013700850137008401370083013700ea
:102500008201370081013700800137007f013700e9
:102510007e0137007d0137007c0137007b013700e9
:102520007a013700790137007801370077013700e9
:1025300076013700750137007401370073013700e9
:102540007201370071013700700137006f013700e9
:10255000ed0037006d0137006c0137006b0137006b
:10256000e9003700e8003700e7003700670137006f
:1025700066013700650137006401370063013700e9
:102580006201370061013700600137005f013700e9
:102590005e0137005d013700420137005b01370003
:1025a0005a013700590137005801370080003700c1
:1025b00056013700550137005401370053013700e9
:1025c0005201370051013700500137004f013700e9
:1025d000cd0037004d013700150037001c003700d3
:1025e000c9003700c8003700c7003700470137006f
:1025f0001700370045013700440137004301370019
:1026000042013700e3003700690037001601370048
:102610003e0137003d013700220137003b01370002
:102620006300370039013700380137006000370098
:102630006e01440012007800808141009480e9001e
:10264000010a78000009e800914978003801370054
:10265000a8609000c0c6b30080cf50000a003a00c6
:102660009400780064805000000a78001000be00da
:102670004f89de00cf91de000002be000203780029
:10268000820378001500370010c7b30080cf5000d8
:1026900002003a00140178000400370014017800a9
:1026a000a0c6b30080cf500005003a00680051007a
:1026b000000a78003002be002003be000700370089
:1026c0000280e900000a780010007800000278001b
:1026d000cfa2de000503780086037800049cbe00cc
:1026e0000694be00a860900080c6b30080cf500062
:1026f0000f00320020c6b30080cf500006003a0021
:10270000184078000000fb00cf80de000101780057
:10271000820178000a00370040c7b30080cf500024
:10272000030032006640400080cf500006003a00af
:1027300018007800cf80de00010178008201780067
:10274000009cbe000294be003800be002801be00fe
:10275000e00f5000e08f5800e00f5900e08f590063
:1027600004003d006e01440092007800d0c2b30026
:102770000c003700081090000018a300040032007d
:102780006e01440092007800b0c2b300050037002b
:102790000008a300570032006e0144009200780048
:1027a00000c2b30080f478000109e800510037004e
:1027b000a8609000c0c6b30080cf500006003a0069
:1027c0009400780064805000000a78001002be0077
:1027d0006033b8001500370010c7b30080cf500039
:1027e00002003a0014017800040037001401780058
:1027f000a0c6b30080cf500005003a006800510029
:10280000000a78003002be002003be000700370037
:102810000280e900000a78001000780000027800c9
:10282000050020000600200007002000049cbe00d8
:102830000694be00a860900080c6b30080cf500010
:102840000f00320020c6b30080cf500006003a00cf
:10285000184078000080fb000100200002002000ea
:10286000030020000a00370040c7b30080cf5000ab
:10287000030032006640400080cf500006003a005e
:102880001800780001002000020020000300200052
:10289000009cbe000294be00081090000038a30007
:1028a000140032003800be002801be00e00f5000c6
:1028b000e08f5800e00f5900e08f59000d00320002
:1028c00080c7b300804f55000300320080c5b300bd
:1028d000804f550007003a006e00440090007800d9
:1028e00002c3b30082f478008100e8008af4780023
:1028f0000108e8007800900000804400600498001f
:102900008a407800640037001401780068005100a4
:10291000000a78005001be004000be00009cbe00ce
:102920000294be00380090000000e00004003d006a
:102930006e01440092007800d0c2b3000c00370052
:10294000081090000018a300040032006e0144003b
:1029500092007800b0c2b300050037000008a30061
:10296000050032006e0144009200780000c2b300fe
:1029700080f478000109e8007800900000804400ad
:10298000600498008a407800080078001e01070063
:1029900067003700286090008000fb00c006200020
:1029a000808f5000230032000a003c006400500079
:1029b000808f50002600320004003c00660050006a
:1029c000808f50000b00320021003700a00620004d
:1029d0000500370040072000808f50001c003200a7
:1029e0001b003c0063005000808f50000700320045
:1029f000170037001480e900000a78001000780002
:102a0000485c900008487800490037001480e900cd
:102a1000000a78001002780068089000cf80de007d
:102a20000101780082017800009abe000292be0087
:102a30003f0037001480e900000a78001001780098
:102a400068089000cf80de000089be0038003700a3
:102a50001480e900000a780010007800680c9000eb
:102a600008087800320037001480e900000a780076
:102a700010007800cf80de0001017800820178002c
:102a8000009cbe000294be007800900000804400cc
:102a90006004980081c7b300080078002800070090
:102aa000230037001480e900000a78001000780045
:102ab00060049800580990000200e00002003d0008
:102ac00096f70700090037008000eb009df807002b
:102ad000800078000000e0000300320068009000f1
:102ae000008050000100370058089000100c98003a
:102af0000f0037006e0144009200780050c2b3000e
:102b000080f178000109e80009003700ee00440078
:102b100011007800808144000a4278008008e800b3
:102b20000a04e00001003a0054c2b300844978006e
:102b30000000eb004f0578004f04be0000000600c7
:102b40006f02b000889fbe008a9fbe008c9fbe00af
:102b50008e1f78008006780050742100b0b79f0067
:102b600080c5b30080cf50000200320042732100c4
:102b7000b2b79f0083002000c3b79f00f0c6b30028
:102b800080cf50000a0032006940400080cf5000e2
:102b900005003200a4002000c4b79f0080c5b30028
:102ba00080cf500002003a0000012000c0b79f0013
:102bb0008e0120003d04be002d05be0040c6b300be
:102bc00080cf5000030032006540400080cf5000ad
:102bd0000a003a00e00f5400e08f5c00e00f5d0057
:102be000e08f5d0005003d000800be000a01be0048
:102bf000350a07000205be000004be00e00f5400c5
:102c0000e08f5c00e00f5d00e08f5d0003003a00a4
:102c10005d0890000000e0000c0032007e01200002
:102c2000cfb0970001027800cfa2de000503780044
:102c3000860378000800be000a01be00b80a07003b
:102c40003fb2970064407800d0e79f004fb09700f4
:102c5000cf80de000101780082017800d0b79f00ac
:102c6000e1b79f00f2b79f0083bf9f000203be0041
:102c70000002be000800be000a01be00a10a070053
:102c8000809ebe008296be00e00f5000e08f58008c
:102c9000e00f5900e08f5900220034000e00e000e0
:102ca000200034003d00be002d01be005fb2970041
:102cb000efb297007fb397008fbb97009c0a070085
:102cc0000205be000004be000e07e900e1fc2f0073
:102cd0008f804000010647005fb29700efb2970077
:102ce0007fb397008fbb97000800be000a01be00ab
:102cf0002c0b07001d0010003fb19700624e7800ba
:102d0000889ebe008a96be00e00f5400e08f5c00f3
:102d1000e00f5d00e08f5d00020034000e00e00077
:102d2000e0ff3c00cfb19700e88f510010003a005f
:102d30000d1090000038a3000d003200f70f57006f
:102d400006003e00e4fc2f000e024200e4c07f00bb
:102d500000c3b30080cf5000050032000e07e90029
:102d600000c3b300e1fc2f008e80400080f07f00a4
:102d700078011700920e98006d009000e3fc2f0080
:102d80008f8141008e80410029f707001d0e9000c1
:102d90005d089000800f560006003d000c005000ba
:102da000800e98000d1090000040a1008016980041
:102db0000f0037000000e0000d003d000d109000f6
:102dc00074006000f00f500009003a007d08900088
:102dd000fd009000010050008d089000010050009f
:102de0000c0750004240a900010034008e0e9800ec
:102df0004f0778004f06be004f05be004f04be00cf
:102e00006f02b10000000600ef04b000889fbe0012
:102e10008a9fbe008c9fbe008e1f7800c0af9f00af
:102e2000a1df9f0060fa2f000f004000e0af9f007d
:102e3000cfaa97005503be004502be0084af9f0095
:102e400095af9f00a6af9f00b7af9f0010c6b3001d
:102e500080cf50001600320010c4b30080cf500065
:102e6000130032004fab9700560890000000e000be
:102e700003003d0060002000500b98000c0037005c
:102e80000000e0000a003a0070c6b300afdb970014
:102e900080cf53000300320070c4b30080cf5300d2
:102ea00003003a0010002000cfa89700d008980037
:102eb000cfa89700e2fc2f000280470070fc0700bb
:102ec00080017800e20f500014003a00cfa997006b
:102ed000e3009000300020009009980010c6b30075
:102ee0002fda9700804f52000a0032006440400001
:102ef000804f5200070032000040e800804f52002f
:102f000004003200a2e221000040e800804f52009d
:102f100017003a00e2e22100150037000000e0004f
:102f200018003400cfaa9700e50090003000200080
:102f3000900a980010c6b3002fdb9700804f530013
:102f40000a00320064404000804f53000700320006
:102f50000040e800804f53000400320022e32100cb
:102f60000040e800804f530001003a0062e3210076
:102f7000b258780002007800b05878009048780085
:102f8000f201370014c6b300afdb970084cf5300c3
:102f90000300320010c4b30080cf530010003a0089
:102fa0004fa89700ec0040001101780000c3b30067
:102fb000005978008208e80080c7b300afd89700b6
:102fc00084cf50000100320080c5b3000049780072
:102fd0004fa99700720090000080e80070019800ef
:102fe0000300e00003003a008006eb00fda79f000d
:102ff000d001370011c6b300afd9970081cf51007f
:103000000300320010c4b30080cf5100ad003a007d
:10301000aee321002fda9700814f52000100320009
:10302000bee42100cfaa9700550890008006e80072
:103030000000e00001003d001d0220000d06e80038
:103040004fab97003604be002605be006022b800d4
:103050006033b8000fa897009fa897002fa997008a
:10306000bfa997004f0507000000e00001003d00e8
:103070000bf0a20088af9f0099af9f00aaaf9f00fe
:10308000bbaf9f007fa0970064005000f0a79f0097
:10309000efab9700805beb00e7af9f003f0037008e
:1030a000c20120000300200001fd2f000180470025
:1030b0009ef907000faa97009faa97002fab9700d1
:1030c000bfab9700f4af9f0085b79f0096b79f00f6
:1030d000a7b79f000400be000601be004905070017
:1030e0000004be000005be00670656004240a9006d
:1030f0000c0034002b0407000002be000203be00d7
:103100007fa897008fb097001fb19700afb19700cd
:103110006805070080af9f0091af9f00a2af9f009e
:10312000b3af9f00efaa9700e7824200e5af9f0090
:1031300070002000e00f5400e08f5c000d003400b0
:10314000600020006fab97006f636500e6af9f00e3
:10315000cc5bdd004455de000a857300c4ddde0073
:10316000e00f5500e08f5d00020034000000e90030
:10317000f4ff3b000000e90005003300efa89700d2
:103180008060eb00e1af9f000000e900fbff3b0027
:103190006fa9970067014100e2af9f000c00e000bb
:1031a000090034006022b8006033b8000fa897000f
:1031b0009fa897002fa99700bfa997001e0a070094
:1031c0000000e000b6ff3c00efa9970064fa2f0072
:1031d0000f024200048051000006e90075fa2f003a
:1031e00085824700e5af9f008d0f560001003d002e
:1031f0008c0678000d00e0002b0035008c8f560007
:1032000005003d006fab970066c07e00f2c0b300c2
:10321000e74f500001003c000041eb008d00e90049
:10322000efab970067c07800824f500006003a006d
:103230008d06e9008100e900efa9970063c07800de
:10324000824f5000faff3200ef4f510004003a0065
:103250006faa970064c078000040e80000f2780090
:103260000100e00007003d00efaa97008502e90099
:10327000e5af9f008d06e8007fa097006400400046
:10328000f0a79f008d00e900070033006fab9700a7
:1032900066c078000000fb006e40780000f3780004
:1032a0008100e900f9ff3b00cfab97005708900081
:1032b0000000e0001f013d000d00e900d00b980068
:1032c0001c0137000fac97009fac97002fad970003
:1032d000bfad97006022b8006033b8000800be00a0
:1032e0000a01be00af0407000000e00005003d0039
:1032f0000bf0a20088af9f0099af9f00aaaf9f007c
:10330000bbaf9f007fa09700725927000280b900d1
:10331000026a2800130020005c080700e400500047
:10332000f1a79f001d003b0063801000c1ff2f002c
:10333000010460000800ea00f0a79f008004eb0091
:103340000800e000470034000808a3000e00320027
:103350006848b80022692100020040003002be0027
:103360002003be000fa897009fa897002fa99700e1
:10337000bfa99700d104070080af9f0091af9f00c5
:10338000a2af9f00b3af9f000884d1008904e8007a
:103390000800e000ecff3c00320037000100e000d4
:1033a000300034006022b8000600200007ff230030
:1033b000b4b79f00c5b79f00d6b79f00e7b79f007f
:1033c000c0ff2f0000806000f0a79f00000478007d
:1033d0008004eb00160034000808a300100032003f
:1033e0006848b80025692100050040003002be0091
:1033f0002003be003fb09700cfb097005fb19700a9
:10340000efb19700ad0407000002be000203be004a
:10341000b4b79f00c5b79f00d6b79f00e7b79f001e
:103420000884d1008904e8000800e000eaff3c00bd
:103430003fb29700cfb297005fb39700efb397000a
:103440000fa897009fa897002fa99700bfa99700e2
:103450005703070080af9f0091af9f00a2af9f006e
:10346000b3af9f004fab9700d608900060c6b30083
:10347000afdb970080cf5300040032006687400026
:1034800060c4b30080cf530003003a007fa09700d0
:10349000008040006a074000f30f5700010034002d
:1034a0003e01200000c3b300efa8970080587800c9
:1034b000e1af9f003a0037000800be000a01be00dd
:1034c000500407000006be00f0b79f0081bf9f00b8
:1034d000680757004240a9000e003400310307007e
:1034e0000002be000203be000800be000a01be00ca
:1034f000700407006022b80046782d007719240078
:103500006e04070080af9f0091af9f00a2af9f00a5
:10351000b3af9f00efa99700e8814100e3af9f00a0
:1035200088002000e00f5600e08f5e00110034009c
:1035300078002000a2002000030020007fb0970048
:103540008fb89700fcf407006faa970005c3b3007b
:1035500005624100e4af9f00f0b79f0081bf9f006c
:10356000e00f5000e08f5800020034000804e9002a
:10357000f0ff3b000804e9000600330000c3b3007d
:10358000efab970080637800e7af9f000804e90085
:10359000faff3b006fa8970068004000e0af9f0073
:1035a0000e00e0000b0034000fac97009fac9700ba
:1035b0002fad9700bfad97006022b8006033b80010
:1035c0000800be000a01be001b0907000000e00061
:1035d000b9ff3c00efa8970062fa2f000f014100ed
:1035e000028050000007e90073fa2f008381470032
:1035f000e3af9f007fa0970067004000f0a79f0007
:1036000001c3b30093cf10000a003a000e07e9008f
:103610007fa097000000e900f0a79f006faa970025
:103620000402e800e4af9f0014427800814f52008a
:10363000f6ff3200cfaa9700d508900060c6b3000d
:103640002fdb9700804f53000300320060c4b300ab
:10365000804f530004003a007fa097000080400094
:103660008006e8000a0037008001eb0050c6b30076
:10367000afdb970080cf53000300320050c4b3008b
:1036800080cf530001003a001300200083864000e1
:103690008d0f570001003d008e0678000d00e00000
:1036a000240035008e8f560006003d006fa897005d
:1036b000e0c07e0092c3b30040c3b30080cf50008f
:1036c00001003c0002c3b3008d00e900efa99700a0
:1036d00063c07800824f500006003a008d06e90072
:1036e0008100e9006faa970064c07800824f500003
:1036f000faff320090c3b300804f510004003a003b
:10370000efaa970065c078000040e80080f27800da
:103710000100e00007003d006fab97000603e900e1
:10372000e6af9f008d06e8007fa097000000e8004c
:10373000f0a79f007fa297008d0178006fa99700e6
:10374000afd897004fa89700060007004f077800f2
:103750004f06be004f05be004f04be00ef04b1008f
:10376000000006000a00fa00889fbe008a9fbe0083
:103770008c9fbe0000047800014578008205780027
:1037800083047800040678000300e00002003c0097
:10379000190020004be6210060c6b300804f5500a1
:1037a0000e00320060c4b300804f55000b003200a1
:1037b00070c6b300804f55000300320070c4b300e0
:1037c000804f550083003a00e40f46008100350029
:1037d00058089000800f56007e003d000c06e8005f
:1037e00060c6b300804f55001000320060c4b300c3
:1037f000804f55000d003200081090000038a300e3
:1038000004003a0058089000808f540001003d00e9
:10381000590c9800580890000c005000500c98006b
:1038200002003b000000eb00500c98000c00e00090
:1038300027003c00f201440013017800680090006a
:1038400001c3b300017079000201e8008209780029
:10385000580890000000e00003003c0008109000b1
:103860000038a30004003200e8009000e0c2b3007a
:10387000807079008209e8000c00ea00d808900006
:10388000808f500001003d000106ea000c00ea00b4
:10389000200c98000c804000500c9800890f5000bc
:1038a00001003d00800478006800900098089000b6
:1038b00001004000390c9800090178008b00780065
:1038c0005bf4070058089000090050001a00370008
:1038d000e8009000180890008c8f540018003d00fc
:1038e00000804000090178008b00780050f4070048
:1038f0001808900009014000120c980009005600b9
:10390000200c9800580890000000e00003003c00e4
:10391000081090000038a30006003200e800900074
:10392000e0c2b30080707900380890000000e80021
:10393000300c980058089000400c9800a300370005
:10394000008040000c0178008b00780038f40700fc
:10395000180890000c004000100c98008c84540053
:10396000580890000000e00003003c0008109000a0
:103970000038a30006003200f201440093007800f2
:1039800068019000e0c2b30000f178008109e8000e
:1039900058089000890f500001003d008004780015
:1039a0006800900098089000010040008c8045005d
:1039b000090178001ef40700180890000900400073
:1039c000100c98005808900009005000200c980036
:1039d0007e00370070c6b300804f550003003200f0
:1039e00070c4b300804f550014003a00580890008e
:1039f000808f540004003d00081090000038a300a0
:103a000001003a00590c9800580890000000e900a5
:103a1000500c980002003b000000eb00500c980096
:103a200051c6b30070c6b300804f5500010032008c
:103a300051c4b300014578000900370010c6b30037
:103a4000804f550002003a000ac7b3000400370057
:103a500010c4b300804f550001003a000ac5b300fe
:103a6000f201440013017800680090003b70790077
:103a70000201e80082097800580890000000e00088
:103a800003003c00081090000038a300040032003e
:103a9000e8009000e0c2b300807079008209e8007d
:103aa000580890000000e000100034008904e9008c
:103ab000890f500001003d008004780068009000ec
:103ac0009808900001004000090178008b00780000
:103ad000d7f307001808900009004000100c980068
:103ae0005808900009005000200c9800e800900051
:103af00018089000808540008a5d78008b06e800f9
:103b00000c00e00004003500b0c2b300804d780026
:103b10008d05780004003700d0c2b300804d7800d6
:103b20008d0578000c06ea008004eb000c00e00034
:103b300009003400a10020000c0078008af407007e
:103b40007681540001f17f00000678008904e800c6
:103b50000000e000f7ff3c00e18f540009003c004a
:103b600050c6b300804f55000300320050c4b3006c
:103b7000804f550003003a0000c3b300805e780018
:103b80008d0578000900e00002003a0000c3b30090
:103b9000805d78000900e000070034008904e90036
:103ba000f680540061c07f0002c3b300825d400014
:103bb0000900e000f9ff3c006800900098089000c0
:103bc0000100400000805500300c98000810900063
:103bd00074006000f00f50000e003a007800900072
:103be0009808900001004000a808900001004000e3
:103bf000b808900001004000c80890008100400013
:103c000078089000808f500002003d0001005000b5
:103c1000000c98004f06be004f05be004f04be00ca
:103c20000080fa0000000600f4ff2f009803370020
:103c30001400200096033700889fbe008a9fbe00b4
:103c40008c1f7800ad030700b403330003866c00bb
:103c50006450e100240032006420e10027003200bb
:103c60006150e100220032006120e10021003200b9
:103c70008b854200eb07b1000134b800003ab80070
:103c80000804420089844a00013ab8000030b800b4
:103c90008880400009014a00040033000000400011
:103ca00081804800020149008b05e900c909dd0057
:103cb000830170000100320013002000c814de00f0
:103cc0004814dd004709de001200b200c808de001b
:103cd00008847000a103070001f0a1000cf0a70008
:103ce00001f0a000960337006120e1009803320044
:103cf0000801be000200be00f7ff37006150e1007e
:103d0000fcff3a009203370003f0a200889fbe0038
:103d10008a9fbe008c1f7800780307007f03330062
:103d20006450e1004f0032006420e1005200320094
:103d300003826c0007003b000905d0000306d00099
:103d4000820f54000c065d000200390002003200b0
:103d500089017800030678008582550004003d0043
:103d60000003fd008103fd008502ea008b8542000f
:103d7000840f720002003b0060001000e080180019
:103d80006011b8000005eb007a28e1000a00390054
:103d900006007800c75ddd00f707b2008780750078
:103da0002d003700828171000a01780061056000f2
:103db0008180d1000080d3008502e900f9ff3b003b
:103dc000060440008784480002003b0060041400a1
:103dd000e0841c000988a300070032008a8171007a
:103de00082817100610164008904d1000884d300dc
:103df0008b05e800170037000978a30013003a008c
:103e00000b00e000130034008b05e90008044400b7
:103e100089844c000a4474000978a3000d003a001c
:103e20000b00e000070034008b05e90008044400a3
:103e300089844c0001003a000b0020000978a3009f
:103e4000f7ff32000001eb000200370082817100b1
:103e50000a017800410307000cf0a70001f0a00060
:103e6000370337006420e10002003a00838f6c00c2
:103e7000370333000801be000200be0030033700e4
:103e8000810378005b0307000001be006000b800fa
:103e90000478a30013003a006220e10015003e0000
:103ea0000d0039008301d1000281d3008180d3004d
:103eb0008301d1000281d3008180d3008301d1002e
:103ec0000281d3008180d3000538b000c42add0010
:103ed000f300b2008381720007f0a70003f0a00096
:103ee00000000600f3ff2700f2ff2f006110b90069
:103ef000fbff370003ff2700f7ff3700889fbe0056
:103f00008a9fbe00010578000100e0000400350032
:103f100008003c000000e0002000320005003700ef
:103f200060001000e080180002003b0001f02c004f
:103f30001a0037000004be006011b8006b092000b1
:103f40000982cf00020039000882cf000441b0008e
:103f5000694252000e00320008003b00828171006d
:103f6000610164008904d1000884d3008b05e80056
:103f70000442e800f9ff3a00050037000804440055
:103f800089844c008b05e9000442e900fbff3a00fc
:103f9000f20207000af0a70001f0a0004f05be00e2
:103fa0004f04be00000006001400fa00889fbe0007
:103fb0008a9fbe008c9fbe000005be000206be00a8
:103fc000680047000c90be000a90be001e03070068
:103fd0006400e1001a00320016003e006100e100ba
:103fe0001a0032006e049000fe0490000e0b900048
:103ff0009e0b90006011b8009e0590000b38b10038
:10400000d501200082817100610164008703d10025
:104010000683d3008984d3000884d3008502e90095
:10402000f8ff3a00cd0207000df0a70001f0a00054
:1040300040033700f1ff2700f0ff2f003d0337005a
:1040400001f8270000002000f7ff37006000b800eb
:10405000f5ff37000081eb003b033700889fbe006f
:104060008a9fbe008c1f78000004be00e10207009a
:104070000478a30026003a006120e1002500320008
:1040800009f8a30025003a006420e1002100320075
:10409000f507b1000508a30002003200000040004f
:1040a000818048006044b800031020000200200016
:1040b00000004000818048000805440089854c00cc
:1040c0000a0541008b8549000a0550008b85580080
:1040d000030033000a00be000204740083847400ed
:1040e0008301d1000281d300830f7100f0ff3a00f9
:1040f0008904d1000884d30060014900820178005e
:10410000c1adde00fb07b000940207008c0237004f
:104110000960a0000800be008902370012022000da
:1041200022bf8800f0ff2f00f1ff27008402370034
:10413000889fbe008a9fbe008c1f78006f02070018
:104140001002200002003b0020bf880073023700ed
:104150008a0062006408e10002003a0020bf880083
:104160007b0237006108e100fcff32000800be005e
:1041700003047800c601070001f0a1005b030700fb
:1041800008f0a600040037000001be0091042400de
:10419000b0fd2000dcfe070009f0a70001f0a2003e
:1041a000670237004f89de0082017800b4033700d0
:1041b0002800fa00889fbe008a9fbe008c9fbe0028
:1041c00003866b00c70207006400e1004400320070
:1041d0006408e1004a0032006100e100460032005c
:1041e0006108e10049003200ec0647006000b800b9
:1041f0003d02be003d03be00f48657006011b800ca
:104200003d04be003d05be007d0320000b003700cd
:104210000000a0008d06e9001300320004024200f5
:1042200085824a0006034b0087834b000000400054
:104230008180480002014900838149000802520040
:1042400089825a000a035b008b835b00f0ff3b000e
:104250000802420089824a000a034b008b834b000c
:104260008d06e900edff3a008482720086827200ba
:10427000f707b200878272000100320015002000ab
:104280001e0490003e0b900006035400e63fb00071
:104290000368a300070032000000a7000500a0008b
:1042a0008301d1000281d3008180d3000080d3003c
:1042b0000603e8008301d1000281d3008180d3008e
:1042c0000080d3000002eb000482d200a3030700a9
:1042d00003f0a1000cf0a70003f0a0009502370046
:1042e000640247006408e1008f0232003400be001f
:1042f0003401be00f6ff37006108e1008a02320097
:104300006011b8006000b800f1ff370003ff27001c
:1043100002002000fbff37001400fa00889fbe0057
:104320008a9fbe008c9fbe000004be000205be0036
:10433000680047000a90be000890be0042020700d5
:104340000070a7000bf0a1000bf8a30016003a00c4
:104350009e0290003043200080825200b0fe2f0069
:104360000028e1000d003c00b0fc2f000028e10017
:104370000d0034001e0990008e0890007e00900011
:104380000501b0000201d1008180d3000080d3007c
:104390008502e800fbff3a006602370001002800b2
:1043a00000002000630237006000b800610237009f
:1043b0002800fa00889fbe008a9fbe008c9fbe0026
:1043c00007067800878669000c003b00030478002c
:1043d0008704780008f0a10009f0a100840f5000c4
:1043e000858f5800860f5900890f5c000300330049
:1043f0000cf0a20001003a000cf0a1003902070005
:104400006400e1005f003200780147006408e100c9
:10441000610032006c014700748557003200be0015
:104420001201be003a04be001a05be001e03900031
:10443000be0a90008503530006003d000004fd0005
:104440008104fd000205fd008305fd008703ea00ed
:10445000050378000df8a300040032006004140086
:10446000e0841c0060051d00e0851d006022b8008e
:104470007d0320000d38e1008006eb000b003900c1
:104480004433dd00f300b2008301730039003700cc
:10449000848272000d027800e10664008b85d100f1
:1044a0000a85d3008984d3000884d3008703e900f8
:1044b000f7ff3b0008004000898048000a014900de
:1044c0008b81490004003b0060001000e080180070
:1044d00060011900e08119000358a30009003200af
:1044e0008d82720084827200610260008301d100bb
:1044f0000281d3008180d3000080d3000603e8004e
:104500001b0037000348a30017003a000600e00034
:10451000170034000603e9000d00a3000000480066
:104520008180480002014900838149000348a300bb
:104530000f003a000600e000090034000603e9001d
:104540000000400081804800020149008381490049
:1045500001003a000003eb000348a300f5ff32001e
:104560006022b80002003700848272006182660017
:10457000fa02070003f0a1000cf0a70003f0a0006e
:10458000ec013700640147006408e10002003a00d2
:104590000df8a300e4013a003200be001201be0093
:1045a000e40137008f1fd100180307008f87e9004f
:1045b0000000e000000006006022b80006022000b3
:1045c0000000d0008180d2000482d2008582d20017
:1045d0000000a0000202520083825a0003003b0048
:1045e0000202420083824a000000a1000603e900a3
:1045f000f3ff3a0000000600efff07000400be00d2
:10460000000006001400fa00889fbe008a9fbe00ca
:104610008c9fbe000004be000205be00680047007b
:104620000a90be000890be00870107000070a70036
:104630000bf0a100304320009e02900080825200c7
:10464000b0fe2f000028e10011003d00b0fc2f005b
:104650000028e100150034001e0990008e0890002b
:104660007e0090000501b0000201d1008180d300de
:104670000080d3008502e800fbff3a000b00e00059
:10468000ac013b0060001000e0801800a901370079
:10469000f0ff2f00f1ff27000b00e000a5013b0019
:1046a0000100280000002000a20137006000b800cf
:1046b000a001370007f0a2003dff37002800fa00f4
:1046c000889fbe008a9fbe008c9fbe0003866b0041
:1046d000840107000028a30064003a000128a30019
:1046e00067003a000008a30062003a000108a30036
:1046f00065003a001e009000be0890008106400050
:10470000ed3fb100f4805700ee019000111ab8009f
:104710008e099000311bb8009e099000311cb80032
:10472000511db800f485570046000700fe019000b7
:104730003a0007008b85e8003e0007008e099000d4
:1047400040000700ee019000340007008b85e80070
:10475000380007008e099000400007009e09900075
:104760001b18b800890440000a854800fe0190002b
:10477000340007008b85e80038000700ee01900048
:10478000300007008e0990001b18b8008904400013
:104790000a8548000a98a30008003a000402420073
:1047a00085824a0006034b0087834b0008044c00b7
:1047b00089844c000a054d008d06e9008482720050
:1047c000850273004c3add00850272000100320060
:1047d00015002000443ade001400b2004538de0027
:1047e000cb45dd000b007000c540de00cb4ddd0089
:1047f0008b8070004549de00cb55dd000b01710058
:10480000c551de000d0378005402070003f0a1003b
:104810000cf0a70003f0a000460137001b18b800f9
:104820008502400006834800e0834b0060044c0092
:10483000070037001b18b8000603400087834800b4
:10484000faff37001b18b8008703400008844800af
:10485000e0844c0060054d00000006001b18b80005
:104860000804400089844800faff37000108a300cb
:104870002d013a005800be005801be00e3ff37008a
:104880000008a30028013a0009047800f9ff370066
:10489000889fbe008a9fbe008c1f7800970007008b
:1048a0009e00330003866c006450e1002e0032004d
:1048b0006420e100330032006150e1002f0032003b
:1048c0006120e1003100320085855500eb07b00022
:1048d00009002000080420000500370008044400f7
:1048e00089844c000a0031000603430087834b0093
:1048f0000001530081815b00f8ff33000203be001a
:104900000800a0000804440089844c00f6ff390028
:10491000c639dd008301730001003200130020005e
:104920008904d1000884d3000998a300050032004f
:104930000800a7000300a0008904d1000884d30068
:104940008b05e8008904d1000884d3000001eb0046
:104950000281d2008100070001f0a1000cf0a70045
:1049600001f0a000760037006420e10078003200fa
:104970000801be000200be00f7ff37006120e10021
:10498000730032006000b800f3ff37000000200021
:1049900001f82700f0ff37000001be009500070076
:1049a0000470a70003f0a1006509b10016003200f1
:1049b0000d0035006828e10006003500f0ff2f00eb
:1049c000f1ff27000300e00013003b000100280076
:1049d0000000050000004000818048008502e900d9
:1049e000fcff3a0008003700f88f420002003c004c
:1049f0008000eb00000005008100d1000080d300a2
:104a00008502e800fcff3a000300e00002003b00e2
:104a100060001000e0801800000006000001be00e9
:104a2000740007000470a70003f0a10003f8a300be
:104a300013003a006509b10010003200090035008a
:104a40006928e1000200350001002800000005008f
:104a500000004000818048008502e900fcff3a0028
:104a600000000600f88f4200050035008100d100eb
:104a70000080d3008502e800fcff3a000000060039
:104a80008000eb000000050004002000000037005b
:104a9000889fbe008a9fbe00841f78001700070011
:104aa0004f00780011003300f0ff2f00838f6c005f
:104ab00006003b00040565000a00a7000800370057
:104ac00009f0a6001000200008003700820f5400f3
:104ad000838f5c00030039001000200001003e00bd
:104ae0000000200009f0a7000000ea004f05be000a
:104af0004f04be000000e000000006000004be00fd
:104b00003c0007000003be000405be000200be001a
:104b100038000700844f7500000006000200be0048
:104b20006450e100050036006420e1000200360018
:104b30000968a30001003a000800be000160a0005f
:104b40004f0678004f05be004f04be00000006006f
:104b5000f0ff2f00f1ff2700f9ff37008100200050
:104b6000618055000b003d000b00200061fe2f000e
:104b70000100e1001d0034008281710061016400c8
:104b80008904d1000884d3000000e800faff3a004d
:104b900071002000610064000300700002006000ea
:104ba0000900320061044400e0844c000988a5003b
:104bb000050032008b05e8006808e10002003a00b9
:104bc0008904d1000884d300f20f20000258e100cc
:104bd00005003d00c75ddd00f907b2008980750062
:104be00008007800000006000bf827008b00780012
:104bf00000000500c70ade00f107b200f50fb200a1
:104c000008003200e1cf4200020032000170a00033
:104c100024000500810f7000010032000408050027
:104c200044000500810f700002003a0014000500e6
:104c30008502e9000000400081c04800fcff3b0005
:104c40000170a00024000500800078005002be0022
:104c50005003be004439de00f700b200f37f2000ad
:104c600003016100090032000218e10016003a0059
:104c700085017200830173008381730000082000a6
:104c800015003a0040002000130037008501720033
:104c9000830173008381730005003a0004a8be00fd
:104ca00006a8be00100020000b0037000201e9003a
:104cb0000402420085824a0006034b0087834b00b2
:104cc0000748a300f9ff32000740a00004a8be0077
:104cd00006a8be00200020008000980092009800e6
:104ce00000000600680447000294be000094be0065
:104cf000fc0447008694be008494be00090078003e
:104d0000d1ff070008007800cfff07009900780066
:104d1000814f70000b003b000800be0064010700db
:104d20004f00b10003003700f3ff2700f2ff2f0010
:104d30006110b9004f06be004f05be004f04be0013
:104d40000080fa0000000600889fbe008a9fbe0017
:104d50008c9fbe00820578000004be00a5ff0700fe
:104d60000800be006420e1000700390002003a009c
:104d7000f1ff2700f0ff2f000160a00012022000c9
:104d800022bf8800550037006120e10003003a008f
:104d90000b00a70001f823005000370001f0a1002c
:104da0000200210093642400a1fb07000800be005c
:104db00004003500b2fd2000930c24004a010700d6
:104dc0000004be000005eb000b00a6004f0dde0046
:104dd00001f0a1000004be0032982f0023ea230056
:104de00095fb07000001eb0003f023000b00a70078
:104df00003f82300c5fb0700e7fe07000000a7003b
:104e00000a00a2003dfc07000b00e0000300320096
:104e10000200200003f02300bbfb070001f0a2000a
:104e20000006be00020020009304240082fb07005d
:104e30000801be00b5fb0700809fbe000c00be004d
:104e400022a22a00d3a723007bfb07004f01be004c
:104e5000aefb07000004be0001f0a100020020002c
:104e60000398230072fb07000800be0019003500fc
:104e70000001be0070fb07000006be00b2c529009d
:104e8000e36223006cfb070022222b00f3942b002b
:104e90009efb07000c01be0067fb0700e2732800c1
:104ea00083c0230099fb07000c01be0062fb0700d2
:104eb00042aa2a00a3e22b0094fb07000c01be00cb
:104ec0005dfb07000801be005bfb07000801be0098
:104ed0008efb07000a00a70001f0a2004f06be00eb
:104ee0004f05be004f04be0000000600889fbe00b4
:104ef0008a9fbe008c9fbe000004be003dff0700dd
:104f00000800be00890678006420e100080039002e
:104f1000040032000160a0001202200022bf8800bd
:104f20005300370091fc2300b0fd20004e003700f5
:104f30000006eb0009f0a10003f8230002002000a6
:104f40000800be003afb07000600340001f8230009
:104f5000000020000801be004dfe07000004be0056
:104f60002c0020000800be0093e82300320a230032
:104f70002ffb0700120034000801be00d1fd230002
:104f8000703d2b0061fb07000005be00b3f323005a
:104f9000f27a26000800be0027fb070003f8230072
:104fa0000200200058fb07000801be0057fb070065
:104fb0000a01be0036fe07000004be000c06e80031
:104fc0000800be0001f0a1000200200003982300a9
:104fd00017fb07000800be00160035000801be00e0
:104fe00015fb07000005be0032cd2c0043fb23005b
:104ff00046fb0700809fbe001269280003d52b00e6
:105000000a00be000cfb0700620f210013ef2b000b
:105010003efb07000a01be0007fb07004f01be0070
:105020001bfe07000801be0003fb07000801be00cd
:1050300036fb07000c00e0000b0032000c10a7004c
:1050400001f0a200b2fd200093fc23006260e100a9
:105050000400320022a9200063f023000c10a700f6
:1050600063f8230029fb07000df0a70001f0a20060
:105070004f06be004f05be004f04be0000000600f4
:10508000889fbe00830478000300e0002c003500f8
:1050900003003c0000827000040271002600320010
:1050a00036432000c50020008383cf000a0039006a
:1050b0000541b1008283cf00070039000541b100ee
:1050c0008183cf00040039000541b1008083cf0007
:1050d000010039000541b10085c353006022b800ca
:1050e000120032000a003b008482720061026000fc
:1050f0008301d1000281d3008180d3000080d300de
:105100000603e8008743e800f7ff3a00070037008e
:10511000000040008180480002014900838149006d
:105120000603e9008743e900f9ff3a000b00070096
:1051300009f0a70003f0a0004f04be000000060025
:1051400060001000e080180060011900e081190083
:10515000d3ff3b00033e2c00f7ff37001800200070
:1051600057002000080453000d003d0006002000f9
:1051700097fc2f000740e1001e003400848272007b
:10518000610260008301d1000281d3008180d300dd
:105190000080d3000804e800f8ff3a004700200030
:1051a0006104600005047400040464000d00320012
:1051b00061004000e080480060014900e081490052
:1051c00003b8a500070032000603e8006538e100d7
:1051d00004003a008301d1000281d3008180d30012
:1051e0000080d300f87f20000830e1000300350084
:1051f000080378006000b8006011b8004433dd0097
:10520000f300b2008301730000000600889fbe0017
:105210008a9fbe008c9fbe000404be000605be002f
:10522000809fbe00829fbe00310007000406780008
:105230000800be000a01be002d00070084067800a9
:105240004f03be004f02be008d4f76007fb0970027
:1052500013003300f0ff2f008b8f6b0006003b0024
:105260000d0666000c00a7000a00370007f0a60034
:10527000100020000a003700880f5200898f5a0062
:105280008a0f5b008b8f5b00030039001000200049
:1052900001003e000000200007f0a7000000ea0027
:1052a0004f06be004f05be004f04be0000000600c2
:1052b000e48240001078a30007003200640240003e
:1052c0001178a3003400be001401be0004003200b7
:1052d0000330a700000006003500be001501be0027
:1052e0000330a00000000600040020001200370078
:1052f00005ff270005826100070032000428e10055
:1053000001003200240005000600070001003a00f9
:10531000440005000408050002000700f9ff3a00f8
:10532000140005006f826100810270008502710027
:105330008502720000000600889fbe008a9fbe00a2
:105340008c1f78004f26dd00ecfd0700f3fd3300d5
:105350006120e100430032006250e10041003e0064
:105360003e0039006420e1003c0032000582550017
:105370000f003b000402e80038003a00800f5300a1
:10538000818f5b00350034000800be0003f0a100ef
:1053900001f0a60003f0a0000cf0a7005bfa0700e4
:1053a000e7fd37000603430087834b000c464600a9
:1053b0000005530081855b00020033000a03be0034
:1053c0000c00a0000402e900f6ff3b008505780010
:1053d0000602430087824b0004003a006000b800d8
:1053e00009f0a70001f0a000d5fd3700000252002f
:1053f00081825a000704e0000400330006034300e2
:1054000087834b008b05e900faff37000905780018
:105410000604be000203be006011b800cffd070005
:10542000e00f5200e08f5a000700350002003c00f8
:105430000c08a300040032000601be0003f0a00027
:105440000cf0a70031fa07000a85680001f0a100fe
:105450000af0a70001f0a000b9fd37000800be0067
:10546000b7fd3700100220000cf0a60020bf880016
:10547000b7fd3700020ab900001bb9000200b800ee
:10548000810042008100430000000600839f680005
:105490000100e00002003d0060001000e080180004
:1054a0000300e00002003d0060011100e0811900ee
:1054b00041fc07004f00e00002003b0060001000cc
:1054c000e08018000000060060001000e080180076
:1054d00060011900e081190000000600881f7800b3
:1054e000000478005001be004000be0000004200f1
:1054f00081804a0002014b0083814b00009cbe006a
:105500000294be00dc000700030031004800900058
:105510000000e800400498004f04780000000600f6
:10552000889fbe00000478008004eb005001be009c
:105530004000be00d000070001003100190020002b
:1055400004005000858058000601590087815900e9
:10555000009cbe000294be0048009000090050006c
:10556000400498004f04be00000006001200fa003c
:10557000889fbe008a9fbe008c1f78000205be0077
:105580000004be00f4b79f0085bf9f0096bf9f0038
:10559000a7bf9f000000eb00e0b79f00d0b79f00bf
:1055a000c0b79f00b0b79f00a0b79f000006eb00f8
:1055b0005fb197006fb097008000d0000000e0005e
:1055c00015003d00e1b79f00010078000200e000f7
:1055d00001003d000000a000ac00070001003d00fc
:1055e0000000a000af00070001003d000000a00087
:1055f000b200070001003d000000a000810007008c
:1056000001003d000000a000b20007007c805700b0
:10561000b2ff070014003700e1b79f0001007800d7
:105620000200e00001003d000000a000970007001c
:1056300001003d000000a0009a00070001003d00ad
:105640000000a0009d00070001003d000000a00038
:105650006c00070001003d000000a0009d00070055
:105660007c805700aeff07006fb097000000e0009d
:105670000700350010002000010020006011b80074
:1056800008047000898470000a0571008b85710020
:105690000c06e800f0032000800f5600c4ff340021
:1056a0006fb097000000e00006003d007fb2970059
:1056b0008fba97001fbb9700afbb97007c80570045
:1056c00086ff07000802be000a03be006fa897000d
:1056d0000000e00004003a002fb29700bfb297002c
:1056e0004fb39700dfb397000400be000601be0071
:1056f0004f0678004f05be004f04be000080fa0040
:1057000000000600881f780018002000881f78001d
:1057100096ff07008f87e9004f047800000006001d
:10572000801feb0091ff07008f87e9000000060053
:105730000800fa00889fbe008a9fbe008c1f780078
:105740006e00070005003d00430007003000070021
:105750000c003d00330007000b003700e00f520043
:10576000e08f5a00e00f5b00e08f5b0006003d0019
:105770000400be000601be0053ff07000205be0084
:105780000004be001c0020002c000700ddff070005
:105790000c00e000010032004bff07004f067800cc
:1057a0004f05be004f04be000080fa000000060056
:1057b0000800fa00889fbe008a9fbe008c1f7800f8
:1057c0004e00070002003d001c00200022000700e0
:1057d0000f00070001003d0012000700170007003e
:1057e000cfff07000c00e0000100320036ff070089
:1057f0004f0678004f05be004f04be000080fa003f
:105800000000060090b79f000100d00080b79f0005
:10581000e00f5400e08f5c00e00f5d00e08f5d0062
:10582000000006000800be000a01be0026ff0700b7
:105830000205be000004be00000006000802be0013
:105840000a03be005fb09700efb097007fb19700ea
:105850008fb99700000006001bff0700010007003a
:1058600000000600b0b79f00c1b79f00d2b79f00ed
:10587000e3b79f00000006000400e1000588e10096
:105880000690e1000798e10000000600c0b79f0005
:105890000200d000b0b79f00afb097000100e00059
:1058a00000000600b0b79f000100d000a0b79f0025
:1058b0009fb097000100e00000000600a0b79f0025
:1058c0000100d00090b79f008fb097000100e0006a
:1058d0000000060080b79f000804d0008984d20031
:1058e0000a85d2008b85d2005fb29700efb2970095
:1058f0007fb397008fbb970000000600d9ff070019
:105900000605be000404be000006eb00e00f5000d8
:10591000e08f5800e00f5900e08f590000000600aa
:10592000889fbe008a9fbe008c9fbe000404b80002
:105930000506b8008904460060854e000606b800da
:105940000a054600e0854e000706b8008b054600b4
:10595000040eb800890446000a854e00050eb80002
:105960000a0546008b854e00060eb8008b054600e2
:105970000416b8000a0546008b854e000516b800cf
:105980008b054600041eb8008b0546000800be00cb
:105990000a01be004f06be004f05be004f04be0008
:1059a000000006000800fa00889fbe008a9fbe0023
:1059b000170007000605be000404be00e00f5200f9
:1059c000e08f5a00e00f5b00e08f5b0008003d00b5
:1059d0000400be000601be00bbfe07000205be00bb
:1059e0000004be000f000700b7fe07000800070014
:1059f0000802be000a03be000a000700c8ff070035
:105a00004f05be004f04be000080fa0000000600f3
:105a1000e0b79f00f1b79f0082bf9f0093bf9f0038
:105a2000000006006fb09700ffb097000fb9970015
:105a30009fb9970000000600809feb00f3fd070070
:105a40008f87e9000000e000000006002600fa0051
:105a5000889fbe008a9fbe008c9fbe000004780015
:105a60000000e00003003200104078000004e00075
:105a70000f003a00881f7800606b2800801f7800b4
:105a800010072000e91c07000003eb00e5042000dc
:105a90001407200053052000926e2800d102200038
:105aa000206f2800ae1c0700e487570018407800dc
:105ab0008000eb00210f98008005eb002b17980069
:105ac0001b1798000005eb000a179800880478005f
:105ad0000004e0001200320098407800d0c2b30009
:105ae00080cf50002a023200a0c3b30080cf500004
:105af00023023200e0c2b30080cf50001c0232000b
:105b00000100fb0002ea07000000e0000100320093
:105b10008b05e800d94078000104e000efff3a006f
:105b2000e10f55000d023c009e1190000300e000c3
:105b3000c5013200e28f5100bf013a00ae10900063
:105b4000e18f5000b8013c000b00e000b2013a00c8
:105b50006055b8003a0f98004b0f98000a06be0037
:105b60008000eb00710f9800610f9800510f9800b2
:105b70000802780088047800184078000004e000eb
:105b80000f003200ea4f50000d0032009e119000cd
:105b90000300e000a3003200a0c3b300994f10003f
:105ba000760032008900e800810478001140780016
:105bb0000004e00002003200ea4f5000f3ff3a0018
:105bc000890f520063003a000a00be0001f0a100f4
:105bd000020020000327240013f807000000e00063
:105be00054003d003e089000ce08900001f0a10056
:105bf00002002000032724000bf807000000e0004b
:105c000043003d002e0890000000e000010032003b
:105c10000df0a2006011b8000c00be0004f80700ef
:105c20000000e00029003d009288280083c823007e
:105c30003e089000ce089000fff707000004be0069
:105c4000422b2a00139923000a00be00faf707002e
:105c50000001be000800be002cf807000001be00d5
:105c60000c00be0028f807000006be0001f0a100ed
:105c700002002000433b2400ebf707000000e00097
:105c800006003c000c00be004f06be004f05be00e3
:105c90004f04be000080fa00000006000c00be00a9
:105ca00077f80700809fbe00829fbe00a16f28008a
:105cb000811f7800500820005c1c0700f0ff2f00b7
:105cc000f1f72700ea875700efff37009288280096
:105cd00083c823003e089000ce089000d6f7070046
:105ce0000004be00422b2a00139923000a00be00c4
:105cf000d1f707000001be000800be0003f807004e
:105d00000001be000c00be0000f80700d6ff3700ff
:105d10003e089000ce08900059f80700809fbe0012
:105d2000829fbe0083722800831f780040082000f5
:105d3000e1ff37000a00be0051f80700809fbe0057
:105d4000829fbe00a1762800811f780030082000c5
:105d5000d9ff3700891f7800841f7800c07a280097
:105d6000801f780020082000301c0700f0ff2f0063
:105d7000f1f72700e6875700c3ff3700e28f510095
:105d80000c003a00a20020008000eb000400780024
:105d900069e90700cf80de0058f807000006be0062
:105da0000902e80084007800100020001017980015
:105db0007dff37009e109000e18f500011003a00e7
:105dc000a20020008000eb00040078005ae90700e0
:105dd000cf80de0049f80700300f9800410f98008f
:105de0000902e8006011b8008000eb0004007800b0
:105df000e4e907006cf807000005be00090278001e
:105e00006fff3700837e2800831f7800b0072000d3
:105e1000061c0700f0ff2f00f1f727008f87e9002d
:105e200099ff37000e1090000000e000d300320010
:105e3000194178000200fb00cf80de0069005000ad
:105e4000e0805800e3062000830f5000e08f5800e8
:105e5000be003e000060010052ff3700bb0037006b
:105e6000ba003700b9003700b8003700b700370074
:105e7000b6003700b5003700b4003700b300370074
:105e8000b2003700b1003700b0003700af00370074
:105e9000ae003700ad003700ac003700ab00370074
:105ea000aa003700a9003700a8003700a700370074
:105eb000a60037003bff3700a4003700a3003700df
:105ec000a2003700a1003700a00037009f00370074
:105ed0009e0037009d0037009c0037009b00370074
:105ee00030ff3700990037002eff37002dff3700b5
:105ef0009600370095003700940037009300370074
:105f00009200370091003700900037008f00370073
:105f10008e0037008d0037008c0037008b00370073
:105f20008a00370089003700880037008700370073
:105f30008600370085003700840037008300370073
:105f4000370037004c003700320037007f00370041
:105f50007e0037007d0037007c0037007b00370073
:105f60007a003700790037006000370029003700d9
:105f70007600370075003700740037007300370073
:105f80002400370071003700700037006f003700c1
:105f9000200037006d0037006c0037006b003700c1
:105fa0006a00370069003700680037006700370073
:105fb0006600370065003700640037006300370073
:105fc000170037002c003700120037005f00370041
:105fd0005e0037005d0037005c0037005b00370073
:105fe0005a003700590037004000370009003700d9
:105ff0005600370055003700540037005300370073
:106000000400370051003700500037004f003700c0
:10601000000037000902e80084007800e2fe370043
:106020007e0890000000e0000b003a006011b8000c
:106030008000eb000400780052e90700daf707005f
:106040000005be000902e80084007800130020006b
:10605000730f9800d4fe37000a00be0088f70700cf
:10606000809fbe00829fbe0001812800811f7800b2
:10607000e007200010ff37005e0890000000e000fd
:1060800012003a000484540008017800840078006b
:106090000e007800fce907000e044400004ceb0001
:1060a0006011b8008000eb000e00780035e90700b1
:1060b000bdf707000006be000902e8008400780072
:1060c00013002000530f9800b7fe37000c00be00ed
:1060d0006bf70700809fbe00829fbe00838428006c
:1060e000831f7800c0072000f3fe37006e08900081
:1060f0000000e0000c003a006011b8008000eb00e6
:10610000040078001fe90700a7f70700300f980088
:10611000410f98000902e800840078001300200075
:10612000630f9800a0fe37003e089000ce08900054
:1061300053f70700809fbe00829fbe0000882800a2
:10614000801f7800d0072000dbfe370000cdb300b1
:10615000004041008900e800e94f500092fe3600ff
:106160000200fb00801f7800801f7800808b2800d1
:10617000801f7800f0072000fbfe3700ae10900073
:106180000100e00020003200e0c2b300994f10008f
:1061900084fe3a00e28f50000c003a00a20020007a
:1061a0008000eb000400780063e80700cf80de0089
:1061b00052f707000006be000902e80084007800dc
:1061c000130020002317980077fe37002e10900050
:1061d000e10f500008003a006011b8008000eb00a9
:1061e00004007800e7e807006ff70700300f980019
:1061f000410f980001ff3700018f2800811f7800b0
:106200000008200002ff370093912800831f7800c8
:1062100010082000fefe3700f0942800801f780050
:1062200050072000fafe370093992800831f78005a
:1062300040072000f6fe3700f09d2800801f780000
:1062400030072000f2fe37000b00e0000e003a009d
:10625000ae1090000100e000070032002e10900008
:10626000e20f50003afe320071a22800811f780030
:1062700070072000e6fe3700c3aa2800831f7800bd
:1062800060072000e2fe370071af280008007800a8
:106290008de907000000e0002c003200e1af28008b
:1062a0000800780088e907008004780031b02800f1
:1062b0000800780084e90700200f98000a00e00039
:1062c000130032000900e00002003a000000e00084
:1062d0000f0032000900e0000a0032001900fb0044
:1062e000801f780080b02800801f78009007200071
:1062f000ce1a0700f0ff2f00f1f72700e4875700c0
:1063000061fe3700ae0990001300fb00f4ff370078
:106310000900e000020032000000e00003003a0043
:10632000130020000317980009fe37001000fb003f
:10633000801f78001900fb00801f7800f1b528004d
:10634000811f7800a007200087fe370003bb2800cc
:10635000831f780080072000adfe37008a1f780079
:1063600091c32800811f780020072000e0ff37003c
:106370002e1090000000e80020179800e5fd37007f
:106380009e1190008301e80013179800e1fd37008b
:106390000a05e800dffd37005400fa00889fbe00c0
:1063a0008a9fbe008c9fbe000004be0002067800db
:1063b0000305780084057800e17c21009140780095
:1063c00070c4b30080cf500089003200e17c21000e
:1063d000914078006340500080cf5000840032002c
:1063e0000102200010002000320a07000000e00037
:1063f0007f0032000a00e000ba0032000c00e0002a
:10640000aa0032000800e00088003a000900e0001d
:106410007e0032008a1f78008a1f78008c1f780067
:106420001904e00077003a00b0cd2800801f780002
:10643000891f7800c5cd2800851f7800d21a070073
:10644000ec87570001c2b30031679800416798009c
:10645000c0c7b300507f9800617f98008002eb00b6
:10646000152f98006044b800fd0320008e8646007a
:106470006f0064002d0032008a0f54002b003200a0
:1064800024002000e78f540001003c000002eb00d4
:106490006348b800000042000e004000ec407c0061
:1064a0000181fb00c411de00b5cc2800e3c17a00f5
:1064b000334898006f01610062c17a004248980039
:1064c00002c2b3005248980002c15000e0c5b300b8
:1064d000804f510012003e0081f67c000804e80065
:1064e0008904e8008a0f5400e1ff3a00f08f54005d
:1064f000dfff3200708014006300b9000400500018
:106500000081e8006348b900000047000400400033
:106510006b00400001022000f9e80700d4ff3700bb
:10652000e0c2b30080f67c00ecff37000800e0001a
:1065300010003400a0c0b30080f67c0000042000ee
:106540000e004000090040000048eb000e007800fb
:10655000f2e80700000178008e00780010002000ab
:10656000e90507001e2890000000e800102f9800a1
:106570008004eb008a0f54001d0031000b00e00086
:106580000e0032001e299000110009000b81d80076
:106590008000fd000000e00008003a000800e00074
:1065a0000e00320090c72800dce8070000017800e8
:1065b00091c7280010002000d3050700881f78002d
:1065c000881f7800e3d02800831f78000e00780031
:1065d0009ae90700e6875700a9ff3700a0c72800ff
:1065e000cee8070000017800a1c72800f1ff3700be
:1065f0004f06be004f05be004f04be000080fa00eb
:106600000000060090d1280088ff37008a1f78001c
:106610008a1f78008c1f7800c3d12800831f780060
:10662000591a0700e887570086ff37000808a300bb
:10663000170032000900e0000e0032008a1f7800c7
:106640008a1f78001904e00008003a00b0cd280045
:10665000801f7800891f7800a2d42800821f78004c
:10666000491a0700ea87570076ff370090d12800c3
:10667000f7ff37008a1f78008a1f780010d628009d
:10668000801f7800401a0700e68757006dff37002b
:106690000818a3006bff32008a1f78008a1f780059
:1066a000d3d72800831f7800f6ff370002d92800cf
:1066b000821f7800b0082000dc1907000003eb00ff
:1066c000e5042000b408200053052000d2da280099
:1066d000c1192000206f2800a11907008f87e90049
:1066e00048ff370050db2800801f7800261a07007b
:1066f0008f87e900beff37000000fa00889fbe00c8
:106700008a1f780080047800010478000000e0000f
:10671000600032000800e0004f0034000800e00094
:106720004b0032009940780000c2b30080cf500087
:106730003e003200e9cf50003c0032001a00200039
:10674000d0c2b30080cf500036003200b0c2b300d8
:1067500080cf5000300032000800e0000600320018
:106760001940780001c2b300814f5000210032006f
:10677000e94f50001f0032006033b8000804e90000
:10678000e10f44001100320005cdb300194278003a
:1067900005404200e94f50000c003e006a31b8004d
:1067a0006a38b900808141000400fb000003b10099
:1067b000cf80de0002034000838348008904e800a4
:1067c0000804e900e10f4400f0ff3a006151b9000c
:1067d0000230b80003b2b900048240000791b9004a
:1067e000820042004f0578004f04be000080fa008e
:1067f000000006008904e8000804e900deff32001a
:1068000019407800814f5000faff3200e94f5000e4
:10681000f8ff3200d8ff37008904e8000804e900d7
:10682000cdff37000085eb00fbff37008904e8004f
:106830000804e900060032009940780080cf50003b
:10684000faff3200e9cf5000f8ff3200bbff3700fb
:1068500099407800b9ff3700881f7800c1dc280014
:10686000811f780070082000701907000803780065
:10687000650520007408200053052000b2de2800c2
:10688000512a2000206f280035190700e48757009f
:10689000a2ff370010df2800801f7800600820006a
:1068a000621907000003eb00e504200064082000e3
:1068b00053052000b2de2800112a2000206f280096
:1068c000271907008f87e90092ff37001600fa00aa
:1068d000889fbe008a9fbe008c9fbe006007980004
:1068e0007107980002067800030f9800840578006d
:1068f0000400e0009f0032000c00e00004003200c1
:10690000eb0f460002003500eb0f56000e0034007e
:106910008c1f780031e12800811f7800900820004a
:10692000421907000c037800250520009408200078
:106930005305200002e3280081372000206f280043
:1069400007190700e48757008c0678000c00e00068
:10695000860035006e009000fe009000e00f5000b1
:10696000e08f58007a0035008000eb00210f98007e
:106970006e049000fe0490000c00e000350035002d
:106980000d05e900090033000a00e00020003a008c
:106990002e0a90000400e0001d003200d0c2b300b7
:1069a000804d78000a05e900f7ff3b00e00f540036
:1069b000e08f5c000b003a000e0a90000400e0003b
:1069c000020032000040eb0080f57e000b007800f2
:1069d0004f06be004f05be004f04be000080fa0007
:1069e000000006008c1f78006e009000fe009000f2
:1069f000809fbe0061e32800811f7800a00820006e
:106a00000a1907000000eb00e8875700f0ff370085
:106a1000e00f5400e08f5c0003003a0000c3b300b5
:106a200080757d00dfff3700a200200003002000fa
:106a30000800be00c0e707000203be000002be005f
:106a400001c3b3000140430080757d000404be0013
:106a5000d4ff37000002eb00140f98002e089000be
:106a600000855600e00f150012003d00a200200036
:106a7000030020000800be00afe707000203be00cd
:106a80000002be0001c3b300014043009e08900015
:106a900080707f000404be00e00f5200e08f5a00b7
:106aa000040032008100e800110f98008a8f500026
:106ab000eeff3500e00f5400e08f5c00c9ff3a00a4
:106ac0000005eb000d00e0000d003400d3c2b30060
:106ad0002e0a90008400470002c2b3000a00e000c2
:106ae0000d003a002e0890000000e0000a0032007d
:106af000834d78000a05e8008d0f5500f7ff35003b
:106b00008e0890000100e000b0ff32000040eb0072
:106b100080757d00adff37002e0a900004005500ff
:106b20001e0a9000840f500004003c000a0052002e
:106b30006140780080757d00eeff37000e08900000
:106b40000000e000eeff3a0082757d00e9ff3700ab
:106b500011002000210f98006e009000fe009000b0
:106b600060041000e084180083ff37008c06ea0000
:106b700078ff3700b0e62800801f780080082000ea
:106b8000aa1807000003eb00e50420008408200099
:106b90005305200002e3280041372000206f280021
:106ba0006f1807008f87e90053ff37000800fa00cd
:106bb000889fbe008a9fbe008c9fbe00000f780099
:106bc0001107980022079800330798000404be00bc
:106bd0000605be000000e000560032001e019000d5
:106be0000200e000450032000801be003eb89700f8
:106bf000ceb8970044f407000004be002e019000b8
:106c0000be0190000a00be0040f4070052a32f000e
:106c1000e3c0230008f407000ef507000001be00e2
:106c20000800be0004f4070092872100a328240076
:106c300001f407000006be002e019000be01900086
:106c40000a00be0030f4070092872100a328240028
:106c5000f9f307000004be000c01be000c00be00ea
:106c6000f5f307000005be000801be000800be00e5
:106c7000f1f307000001be000a00be0023f4070084
:106c8000f6f407001e0178000089be000c01be006a
:106c90000800be0026f5070012ee2200532624004d
:106ca000e5f307000001be0000002000412b240096
:106cb00015f407000004be006011b800dcf3070003
:106cc0000000e00005003d0002002000433b2400de
:106cd0000800be000df407000004be001e00900076
:106ce0000888be000000eb004f06be004f05be0046
:106cf0004f04be000080fa000000060080e8280073
:106d0000801f7800e0082000481807000003eb000f
:106d1000e5042000e40820005305200032eb2800a1
:106d200041152000206f28000d1807008f87e9000b
:106d3000adff370010ec2800801f7800d00820003d
:106d40003a1807000003eb00e5042000d4082000f7
:106d50005305200032eb280001152000206f280089
:106d6000ff1707008f87e9009cff37000400fa0037
:106d7000889fbe008a9fbe008c9fbe0000067800e0
:106d8000810578000205e9000200e00006003a00f3
:106d90000000eb004f06be004f05be004f04be00d2
:106da0000080fa00000006009c4678001b80fb0073
:106db000000f78000d80fb0010079800f5e6070033
:106dc000800478001e04780008007800f1e60700cf
:106dd000808f54000a003a000000eb000d04e00030
:106de000ecff32000c06e8008b05e8000a00780092
:106df0000a05e9000000e000ebff3a00e4ff37007d
:106e00001e009000e3e60700800478000800780088
:106e1000e0e6070000805400deff37000200fa00c1
:106e2000889fbe008a9fbe008c9fbe0080057800b0
:106e3000010578001b4678001a84fb000c80fb00db
:106e4000000f7800d3e607008004780088067800f9
:106e500008007800cfe60700808f54000b003a004e
:106e60000000eb000c04e000030032008b05e8009a
:106e70000a05e800efff37004f06be004f05be00d1
:106e80004f04be000080fa00000006001e007800db
:106e9000c0e60700000478000d007800bde607009a
:106ea00000005400f4ff37000000fa00889fbe0085
:106eb0008a9fbe0000047800810578008204780073
:106ec000030578000000e000020032001004e0003a
:106ed00007003a00004deb00800ceb000000eb00d7
:106ee0004f05be004f04be000080fa0000000600ff
:106ef000afe60700000444001804e000f5ff32008c
:106f00008b00780008007800bae607000000440013
:106f1000800c7800104d7800190078001004e00013
:106f2000020032000048eb00990ce80008007800ed
:106f3000ebff37000000fa00810278008000eb00d0
:106f400000027800104078000004e00006003200e3
:106f50000000fb007f09b800820040005440780028
:106f60000004e000faff3a00110009008580d80013
:106f70008000fd000080fa00000006001600fa0004
:106f8000889fbe008a9fbe008c1f780066010700a4
:106f900020402d00801f7800010f2900811f7800fc
:106fa000f9170700b1192900e04921009bff0700ec
:106fb000e48757000000e0005301320050a4800035
:106fc00061a48000809fbe00211a2900811f7800e3
:106fd000ed17070020c0b300004f78000001eb0060
:106fe0008e007800100020005c010700000478008b
:106ff000e68757000000e0003a013500e10f540039
:10700000fb003200d0c4b300cef7b7001000200060
:10701000d0a5880070a4800081a48000809fbe005d
:10702000111f2900811f7800d7170700e687570036
:10703000acd22100dc37ef00de37ef00007d20000e
:10704000010020001007980021079800b2bc8000c2
:10705000c3bc8000c00320000014b8000098b90031
:10706000808444000800be004ef4070030079800fa
:10707000410798005207980063079800e00f5400fa
:10708000e08f5c00d1003500e057e200cd003a000f
:10709000e17c21009140780080c4b30080cf500093
:1070a000c8003200004feb00e17c210091407800e5
:1070b00070c4b30080cf500094003200e17c210006
:1070c00091407800d0c4b30080cf50008d003200d2
:1070d0000104200020002000f60607000000e00068
:1070e0006a003200b614e20037003a001e24a00005
:1070f0000e81e8008e0078003000200017010700a4
:10710000000478000000e000260035000800e000e0
:107110000d0032001e80fb000018a3000a003200a0
:10712000e17c21009140780070c4b30080cf500012
:107130001a003200e17c210091407800d0c4b300f5
:1071400080cf500007003200e0be8000f1be80001a
:1071500061004000e0804800e0be8800f1be880089
:10716000c9ff3700004eeb008001eb001200200049
:10717000a1d22100020078001d02070030c0b30038
:107180009c4f1000f0ff3a00200020001905070076
:1071900080c4b300cef7b700ebff3700251d070012
:1071a000e4ff37000003eb008002eb0000027800f0
:1071b000d304200032242900b10f200080242900ac
:1071c000e7160700d1ff3700740907007007980021
:1071d000010f9800120f9800230f9800f8bd80004f
:1071e00009be80000800be00eef30700e00f540067
:1071f000e08f5c00200035000002be000203be00ec
:107200007e0090008e0890001e099000ae0990004c
:10721000e7f3070040f407000005be0082ad8000e0
:1072200093ad80000201500083815800b0a580001a
:1072300001002000800f5100818f5900abff390001
:10724000007121009d2407000000e00003003a00c7
:107250008aad88009bad8800a4ff3700801f7800ae
:10726000f8242900881f780090322000ef160700cc
:10727000e4875700f6ff37006022b80006002000c0
:10728000071f24004af40700dbff37000810200026
:10729000881f7800479f2100a6002000a57e2100be
:1072a000540020004100200072a4800083a48000cc
:1072b00020002000540307008f87e9000000e00051
:1072c00088ff320020002000801f780091272900cd
:1072d000811f780050042000d416070026002000eb
:1072e000d5042000540420008501780032242900b0
:1072f000210d20008024290099160700e4875700fb
:1073000078ff37001e14a00071ff37000104200031
:1073100010002000670607000000e00002003200b5
:107320001e14a00065ff37003e029000ce029000c0
:107330005e039000ee039000887021003800be00cc
:107340002801be001af407000004be000205be00ba
:10735000120907000002be000203be000800be00c2
:107360000a01be008ff407000000e00053ff3d005b
:1073700001042000100020002d0407000000e000a0
:10738000e7ff320010002000801f7800212a29002a
:10739000811f780070192000a41607001600200035
:1073a000d5042000741920008501780032242900ba
:1073b000910b20008024290069160700e4875700fc
:1073c000d7ff37003f0907002fff37006022b800c2
:1073d00006002000071f2400f5f30700300798007f
:1073e00041079800520798006307980026ff37006e
:1073f000800c200001002000100798002107980051
:107400008e81e80008017800a1d2210008007800f0
:1074100077010700e10f50000e003200a82d29006f
:10742000881f780000192000801607000003eb0079
:1074300005192000d404200084017800322429009a
:10744000d108200080242900451607008f87e90015
:10745000f7fe370078b98800b214e2001900320054
:10746000acd2210030c0b3009c4f10000d003200a0
:1074700070c4b300cef7b70070a4800081a4800070
:10748000809fbe0050a4800061a48000809fbe0049
:10749000d1302900811f7800bb160700ea8757000a
:1074a000e4fe370080c4b300cef7b700d8a588004b
:1074b00042022000e134290008007800120207008f
:1074c000dcfe370080c4b300cef7b700d8a5880033
:1074d0002202200031372900080078000a02070044
:1074e000d3fe37000003eb0080027800d4042000b4
:1074f0008401780032242900c1062000802429005c
:1075000017160700bdfe370068392900881f78006c
:107510009d16070080c4b300cef7b70010c0b300bb
:10752000e0f7b700c9ff37000000fa00e0c4b3007d
:10753000cef7b700351607004a080700cd17070039
:107540009515070089060700250707002908070089
:107550000000eb000080fa00000006000200fa00c4
:10756000889fbe008a9fbe008c9fbe00800178006d
:1075700001047800820478000000e900e70f500061
:107580005a003e00114178000204e0005000320031
:107590008041eb00034f78000006eb007bc5b30091
:1075a0000900e000060032001900be00e9c55500e0
:1075b000e00f5000e08f580001003200e6c54500a2
:1075c0001dc0b3000045eb000218a30031003a00d3
:1075d0000228a30021003a000c00e0001d003a0040
:1075e0000a04e00010003a0070c5b30080cf5500d7
:1075f0001400320040c5b30080cf55000a003a00a5
:107600000d01fb001900be00000707003901100042
:10761000a98118004240a900030034008046eb0015
:1076200018417800e8ff37001e4c78000c00780005
:107630004f06be004f05be004f04be000080fa009a
:1076400000000600d4e2a8000140fe00d4e2a90038
:10765000f3ff3700db070700f3ff370001042000ca
:1076600020002000930507000000e0000700320022
:107670009215e200d8ff32001e4178000224a000db
:10768000024f78000c06e800d3ff37000a45e800f7
:10769000d1ff3700010420001000200085050700fd
:1076a0000000e000080032005815e200040032003b
:1076b0001e4078000014a000004f78000c06e8007f
:1076c00018417800c2ff37000a45e800fcff370088
:1076d000623d2900821f7800c0032000d3150700f7
:1076e0000080eb008f87e900d1ff3700831f78000f
:1076f000503f2900801f7800b0032000cb15070001
:107700000080eb00e4875700c9ff37000400fa004f
:10771000889fbe008a9fbe008c9fbe000004780038
:107720008105780002057800030f78000000e90069
:10773000e10f50009d003e000b00e0008d00320084
:10774000e10f55007c00360001042000080078009d
:10775000580507000000e0006800320075c5b3005e
:107760001e0178000200e000060032001200be0098
:10777000e9c25200e00f5000e08f580001003200d3
:10778000e6c24200a00320000040b800435121009f
:107790008304400084532100040040009046780098
:1077a0000a04e9000006eb000045eb0012c0b3003c
:1077b0004240a9002a003400590090008800780057
:1077c000800f540001003400800078000100e000c8
:1077d00033003400ee814400930078003145780096
:1077e00081097800090a90004900900000004200d9
:1077f000808f500001003900840978008a5d78008c
:107800000c06e8000804e9002104200091407800fb
:107810008180fb00c508de0001007800d4f7b700c6
:1078200000ceb3004260b700590090000000e900ac
:10783000d0049800c508dd0042c0bf007f40600052
:107840000140700042e0b7008d4f55001200320039
:107850000800e000100034000800e000d6ff3c0003
:107860009ed7bf000018a30009003a000c00780062
:107870008d4f5500010032000c00ea004f06be009b
:107880004f05be004f04be000080fa000000060055
:107890004c070700f5ff3700804deb00f0ff370085
:1078a000e0c4b30080cf5200edff320069404000d9
:1078b00080cf52000d0032000201fb009e017800d3
:1078c0001300be0015079800500607001e0278003e
:1078d00034011000a48118009e0290004240a900cb
:1078e000dfff34000041eb00dbff3700d4e2a800eb
:1078f0000140fe00d4e2a900d7ff3700881f7800be
:1079000000432900801f780000042000471507006d
:1079100008037800d504200004042000330520006b
:1079200032462900d10e2000d04629000c15070050
:10793000e487570089ff37008a1f780064472900d1
:10794000841f7800f0032000381507000a03780030
:1079500065052000f403200033052000324629008d
:10796000810e2000d0462900fd140700e48757004f
:1079700075ff3700234a2900831f7800e0032000a9
:107980002a1507000003eb00e5042000e4032000b3
:107990003305200032462900410e2000d046290040
:1079a000ef1407008f87e90065ff3700881f780014
:1079b00020002000801f7800124d2900821f7800cf
:1079c000d0032000191507000803780025052000c2
:1079d000d40320003305200032462900010e200088
:1079e000d0462900de140700e687570052ff370013
:1079f0000400fa00889fbe008a9fbe008c9fbe00d4
:107a0000000478000106780082047800030f7800f3
:107a10000000e900e10f5000aa003e000c00e00069
:107a20009a0032000900e0008900320001042000c1
:107a3000080078009f0407000000e0007500320095
:107a400070c5b300204798009e0078000100e00058
:107a5000080032001100be00e2c4b30022479800c3
:107a6000e00f5000e08f58000200320043c5b30021
:107a700023479800a00320000040b8004451210093
:107a800004054000890578008006eb0010c0b300b3
:107a9000304798000900e0002e0034005a009000a2
:107aa0000b047800808f550001003400000478003a
:107ab0000800e0003f0034000a089000ca0090006f
:107ac00001004000fa00900081045000890f54002a
:107ad0002b003400090178000c007800d4e3070083
:107ae00009004600090154008a089000d0e307000d
:107af0000a08900008004000090050007005980036
:107b00000806460088864600888555002104200026
:107b1000914078008180fb00c508de0001007800fc
:107b2000d4f7b70000ceb3004260b7005a0090000f
:107b30000800500050059800c508dd0042c0bf0095
:107b40007f4060000140700042e0b7000b00e000a1
:107b5000d2ff3c009ed7bf000018a30006003a00e9
:107b60000d0078004f06be004f05be004f04be005a
:107b70000080fa000000060092060700f8ff3700b8
:107b8000080178000c007800a9e30700fa009000d3
:107b900088804000710598000a0990004a00900012
:107ba00000004100808f5000d5ff39007205980019
:107bb000d3ff3700e0c4b300ae40900080cf500048
:107bc000e4ff32006940400080cf50000d003200d9
:107bd000be4190000301fb001e0278001400be00ad
:107be0008a0507001e02780034011000a4811800e5
:107bf0004240a900d7ff34000040eb003047980016
:107c0000d2ff3700d4e2a8000140fe00d4e2a90070
:107c1000ceff3700881f780004512900841f7800a8
:107c2000400420008114070008037800d5042000d8
:107c3000440420003305200032542900311620006e
:107c4000d046290046140700e48757007cff370020
:107c5000801feb00d3542900831f780030042000dc
:107c6000721407000003eb006505200034042000b7
:107c70003305200032542900e1152000d0462900a8
:107c800037140700e487570068ff37009257290030
:107c9000821f780020042000641407000003eb001a
:107ca000e50420002404200033052000325429007c
:107cb000a1152000d0462900291407008f87e9006c
:107cc00058ff3700881f780020002000801f7800b0
:107cd000815a2900811f78001004200053140700e6
:107ce0000803780025052000140420003305200037
:107cf0003254290061152000d046290018140700cd
:107d0000e687570045ff37000200fa00889fbe0053
:107d10008a9fbe008c9fbe000006be0082057800d0
:107d2000ba14e2000b003200e17c2100914078009f
:107d300040c4b30080cf5000060032000102200092
:107d400010002000db03070018c0b3000000e000b3
:107d500001003a000044eb000c00e900e10f500084
:107d60000a0036000804e0009e003a000c03780088
:107d7000250520001404200033052000725e290030
:107d8000411d2000d0462900f51307000d00e0003a
:107d9000830032000b00e0000a003a000804e00013
:107da00078003a000003eb00650520003404200051
:107db00033052000725e2900011e2000d0462900f4
:107dc000e7130700010220000c007800b903070048
:107dd0000000e0000a003a000804e00062003a00f7
:107de0000c037800650520004404200033052000c2
:107df000725e2900711e2000d0462900d8130700aa
:107e0000a00320000060b80062522100020540007b
:107e10000000eb00000f78000b00e000360032009d
:107e2000ca0090005a009000008050004240a90013
:107e3000490034000b047800808f550001003600a3
:107e4000000478000a08900001004000ea01900058
:107e500083045000890f5400310034000901780078
:107e60008d00780003007800f1e207000a08900016
:107e70000901540089804600ede207000a089000dd
:107e80000800400009005000600598008886460000
:107e9000888555001e01780008014100020f780016
:107ea00021042000914078008180fb00c508de009d
:107eb00001007800d4f7b70000ceb3004260b700ed
:107ec0005a0090000800400050059800c508dd00e9
:107ed00042c0bf007f4060000140700042e0b70038
:107ee000e10f56000c003200e20f5600080032008d
:107ef0000b00e000caff3a001e0078004f06be00eb
:107f00004f05be004f04be000080fa0000000600ce
:107f10008720a800f6ff37008540a800f4ff37004f
:107f2000080178008d00780003007800c0e20700a7
:107f3000ea00900088804000610598000a099000de
:107f40004a00900000004100808f5000cfff3900b0
:107f500062059800cdff3700d4e2a8000140fe0082
:107f6000d4e2a900e2ff37008c1f7800205f2900cf
:107f7000801f780040042000ac130700e4875700fe
:107f800097ff3700801feb0062622900821f780094
:107f900030042000a5130700e487570081ff370055
:107fa0000804e00009003a000003eb00e5042000ab
:107fb0002404200033052000725e2900a11d20004a
:107fc000d04629006613070072ff3700206529009c
:107fd000801f780020042000941307008f87e90099
:107fe000f1ff37008c1f780020002000801f7800f0
:107ff00022682900821f7800100420008b130700dc
:10800000e687570059ff37000600fa00889fbe0038
:108010008a9fbe008c9fbe00800478000205be00cf
:10802000010f7800140798000506780026079800cd
:10803000870678000000e900e10f5000eb003e00e9
:108040000a01be00e206b1000380b10020192c0035
:1080500011002000800f5100818f5900d4003e0094
:108060009e0078000100e900e60f5000c1003e00cc
:108070009e0090000100e900e60f5000ae003e00b7
:108080000c00e0009e003200ae0090000100e00015
:108090008c0032000d00e0007c003200ceb897006a
:1080a0000100e0006a003200a00320000048b80090
:1080b0000250210002044000180890000006b2009f
:1080c0005f003a00080078001c0009000018eb006f
:1080d0000a01be000900780009030700e1ff2f0034
:1080e0000000e0002d003a002c1498001c149800a9
:1080f0000c1498003d1c98002d1c98001d1c980025
:10810000ae009000610c98004eb997007214980070
:10811000a0c0b300007c9800e18f54002d00320015
:10812000e28f540023003a001622ef008f00a900ce
:108130008f20a9008700a9008720a9002e40900069
:1081400067416000a0c0bf0081cfb3000140600064
:1081500002407000a0e0b7009e40780067c1600058
:108160004411dd00a0c0bf00f1c8b30001406000b1
:1081700002407000a0e0b70000002800b0108800a6
:1081800000402800c01088008f00a8008f20a800a1
:1081900010062000100c98008000eb000100780011
:1081a0004f06be004f05be004f04be000080fa001f
:1081b00000000600891f7800226c2900821f7800c9
:1081c00000042000191307008080eb00e4875700ab
:1081d000f2ff37000c22ef008d20a9008d40a9008e
:1081e0008520a9008540a9002e40900067416000cd
:1081f0004411dd0098c0bf00f1c8b3000140600029
:108200000240700098e0b7009e40780067c16000af
:1082100099c0bf0081cfb3000140600002407000f0
:1082200099e0b70000002800601088000040280096
:10823000701088008d20a8008d40a800d4ff370062
:10824000891f7800706f2900801f7800dcff3700dd
:10825000801feb0022722900821f7800200420007a
:10826000f21207000003eb00650520002404200043
:108270003305200012752900e1242000d046290092
:10828000b7120700e487570087ff3700b075290051
:10829000801f780020042000e41207000003eb0098
:1082a000e504200024042000330520001275290075
:1082b000a1242000d0462900a91207008f87e900d9
:1082c00076ff3700801feb0072782900821f78004c
:1082d00020042000d51207000003eb0065052000f4
:1082e0002404200033052000127529006124200099
:1082f000d04629009a120700e487570065ff37002f
:10830000607b2900801f780020042000c71207002e
:108310000003eb00e50420002404200033052000c6
:108320001275290021242000d04629008c12070054
:108330008f87e90054ff3700811f7800227e2900d3
:10834000821f780020042000b81207001e0390004e
:108350002505200024042000330520001275290083
:10836000e1232000d04629007d120700e487570052
:1083700043ff3700811f7800f2822900821f7800b6
:1083800020042000a91207001e0378002505200004
:10839000240420003305200012752900a1232000a9
:1083a000d04629006e120700e487570030ff3700df
:1083b0008a9fbe00d2872900821f780020042000f7
:1083c0009a1207000a0378002505200024042000e3
:1083d000330520001275290061232000d0462900b2
:1083e0005f120700e68757001dff3700891f7800de
:1083f00020002000801f7800c18b2900811f780099
:1084000010042000891207000903780025052000c8
:1084100014042000330520001275290021232000b8
:10842000d04629004e120700e687570004ff3700a8
:108430000000fa00889fbe008004780001047800e4
:108440000000e900e10f500059003e00000220004a
:10845000800f54001100320000042000800f5400ef
:108460000e003200881f7800b08f2900801f78002e
:10847000200420006d120700080378002505200065
:10848000240420003305200052932900712e20007f
:10849000d046290032120700e4875700a0032000cd
:1084a0000048b80022512100020040001008a3003b
:1084b0003c003200880078000102b2001000640025
:1084c000880f50002a003200e18f54001d00320056
:1084d000e28f540013003a000100e0000d0032006a
:1084e0008720a9001942a80019e2a8008f20a8003f
:1084f000a00320000048b8002251210002004000e3
:10850000100874000000eb004f04be000080fa0069
:10851000000006008700a9001822a9008f00a8000b
:10852000f3ff3700891f780040942900801f7800ee
:10853000000420003d1207000080eb00e487570094
:10854000f1ff37000100e000050032008540a9007e
:108550000f42a8000fe2a8008d40a800e4ff3700fa
:108560008520a9000e22a9008d20a800e0ff370079
:10857000e09729000100e00001003a00709829000e
:10858000801f7800891f7800f2982900821f7800e8
:1085900000042000251207000080eb00e68757004a
:1085a000d9ff3700891f7800709c2900dfff370052
:1085b000891f780020002000801f780022a0290059
:1085c000821f7800100420001812070009037800a9
:1085d00025052000140420003305200052932900b3
:1085e000312e2000d0462900dd110700e687570014
:1085f00096ff37000000fa00881f7800000478001a
:108600000000e900e10f50002a003e00e10f540095
:108610001d003200e20f540013003a001622ef0052
:108620008f00a9008f20a9008700a9008720a9003a
:1086300080cfb300a060b600f0c8b300a060b60061
:108640001822ef00a00320000040b80022512100b2
:10865000020040000008eb000000eb004f0478002f
:108660000080fa0000000600881f780060a429003e
:10867000801f780000042000ec1107000080eb0050
:10868000e4875700f5ff37000c22ef008d20a9008a
:108690008d40a9008520a9008540a900f0c8b3003d
:1086a0009860b60080cfb3009960b6000e22ef004c
:1086b000e4ff3700881f780020002000801f78002a
:1086c000c2a72900821f780010042000d7110700dc
:1086d000080378002505200014042000330520003d
:1086e000c2ab290081352000d04629009c1107002b
:1086f000e6875700c5ff37000000fa00889fbe00dc
:1087000080047800010478000000e900e10f5000c7
:108710003d003e0000022000800f54001100320096
:1087200000042000800f54000e003200881f7800e3
:1087300070ac2900801f780020042000bb110700c6
:1087400008037800250520002404200033052000bc
:1087500022b02900d1392000d0462900801107001d
:10876000e4875700e18f54001d003200e28f54006f
:1087700013003a000858a3000e0032008f20a90011
:108780008720a9001942a90019e2a900a00320002e
:108790000048b80022512100020040000881ea0090
:1087a000100861000000eb004f04be000080fa00da
:1087b000000006008f00a9008700a900f3ff370022
:1087c000891f780022b12900821f78000004200050
:1087d000961107000080eb00e4875700f2ff370096
:1087e0000858a300050032008d40a9008540a9006b
:1087f0000f42a9000fe2a900e4ff37008d20a90075
:108800008520a900e1ff3700891f780020002000a3
:10881000801f7800d2b42900821f78001004200045
:1088200082110700090378002505200014042000a8
:108830003305200022b0290091392000d0462900bc
:1088400047110700e6875700b2ff3700809fbe0040
:10885000829fbe00849fbe00861f78000000fa0041
:108860008041eb00d4c2bf000080fb004700de0067
:108870008082fb00d4e2a9008540a90000ab800003
:1088800011ab800061004000e080480000ab880030
:1088900011ab88006a15e2001b003200d6002000f0
:1088a00082ab800044ab80000f22ab0014003a0082
:1088b00071ab800011407800ea4f50001d0032007b
:1088c0008041eb000080fb00801088008100e80000
:1088d00071ab880004004100808f50000100390016
:1088e00072ab88006a35ed0020ab800031ab8000b0
:1088f00061004000e080480020ab880031ab880078
:108900006a15e200e8ff3a00c728dd00d4c2bf00c4
:108910000074a10001407000d4e2b7000080fa00aa
:108920004f0378004f02be004f01be004f00be0053
:10893000004006000304e000e1ff3a0013c0b3006a
:1089400086108800e8ff3700809fbe00829fbe002f
:108950000000fa00d4c2bf000080fb004700de0028
:108960008081fb00d4e2a900d4c2a8008520a90020
:1089700070aa800081aa800061004000e080480069
:1089800070aa880081aa88000e22ab00070032007e
:10899000d0a98000e1a9800061004000e08048008b
:1089a000d0a98800e1a988004c35a8000e02ab00d0
:1089b0000c0032000e42ab00180032004c55a800eb
:1089c000f0a9800001aa800061004000e08048001a
:1089d000f0a9880001aa8800901080000e02ab0068
:1089e000f4ff3a000e22ab00020032000e22a90072
:1089f0004c35a900d4c2a900c718dd00d4c2bf00fd
:108a00000074a10001407000d4e2b7000080fa00b9
:108a10004f01be004f00be00004006004c55a900ab
:108a2000c1aa8000b0aa8000808f500013003100de
:108a30004c95a900d1aa8000901080008058780041
:108a4000d1aa8800f2aa8000b0aa800000004100ec
:108a5000808f500001003900d2aa880090aa8000bf
:108a6000a1aa800061004000e080480090aa880030
:108a7000a1aa88005835ec00d8ff370010aa800062
:108a800021aa800061004000e080480010aa880010
:108a900021aa88004c95a800d2ff3700809fbe0015
:108aa000829fbe00841f78000000fa00d4c2bf007d
:108ab0000080fb004700de000082fb00d4e2a9003a
:108ac0008720a900d0ac8000e1ac800061004000ac
:108ad000e0804800d0ac8800e1ac8800a415e2003a
:108ae0001500320013ad800052ad80001922ab009a
:108af0000f003a0040ad8000b080fb00d11088002c
:108b000040ad880083004100810f50000100390012
:108b100042ad8800f0ac800001ad800061004000f3
:108b2000e0804800f0ac880001ad8800a435ed007d
:108b3000a415e200edff3a00c720dd00d4c2bf005b
:108b40000074a10001407000d4e2b7000080fa0078
:108b50004f0278004f01be004f00be0000400600eb
:108b6000809fbe00829fbe000000fa00d482a80051
:108b7000d4c2bf000080fb004700de008081fb0004
:108b8000d4e2a9008700a90040ac800051ac80006d
:108b900061004000e080480040ac880051ac880093
:108ba0001822ab0007003200a0ab8000b1ab800000
:108bb00061004000e0804800a0ab8800b1ab8800b5
:108bc0008635a8001802ab000c0032001842ab003a
:108bd000180032008655a800c0ab8000d1ab8000e1
:108be00061004000e0804800c0ab8800d1ab880045
:108bf000e01080001802ab00f4ff3a001822ab002e
:108c0000020032001822a9008635a900c718dd002d
:108c1000d4c2bf000074a10001407000d4e2b700cc
:108c2000d482a9000080fa004f01be004f00be00b0
:108c3000004006008655a90091ac800080ac800001
:108c4000808f5000130031008695a900a1ac8000f0
:108c5000e010800080587800a1ac8800c2ac800091
:108c600080ac800000004100808f5000010039007e
:108c7000a2ac880060ac800071ac80006100400054
:108c8000e080480060ac880071ac88009235ec0050
:108c9000d8ff3700e0ab8000f1ab800061004000fe
:108ca000e0804800e0ab8800f1ab88008695a80022
:108cb000d2ff37000000fa000001be000000e9000a
:108cc000e10f50000a003e00a00320000010b80091
:108cd0002251210002004000030178000200a000a0
:108ce0001000610011002000820f500001003200ce
:108cf0008000eb00010078000080fa000000060010
:108d00000000fa00889fbe008a9fbe008c9fbe00b4
:108d1000000678000205be000000e900e10f5000e7
:108d20004d003e000a01be00e206b1000380b10022
:108d300020192c0011002000800f5100818f590054
:108d400036003e00f2bd800003be80006a10b8000d
:108d50006a19b900828040007051b800705ab90099
:108d60008481410014ee07000004be00a200200030
:108d70000300200020ee07001dc0b300e40f5000e8
:108d8000e08f580001003e008046eb00a20020006a
:108d9000030020000800be0007ee07000d81fb0065
:108da000000141008201e900a00320000060b8003a
:108db000c4502100040140000a89be000251210074
:108dc0000200400003087800e10f56001100320055
:108dd000e20f560007003a00f31088000000eb0095
:108de0004f06be004f05be004f04be000080fa00d3
:108df000000006008c1f780024b92900841f780029
:108e000000042000091007000080eb00e4875700f1
:108e1000f3ff3700a3108800f0ff37008a9fbe00e1
:108e2000b4bc2900841f780020042000ff0f070035
:108e30000a037800250520002404200033052000c3
:108e4000e2c02900f1552000d0462900c40f0700d8
:108e5000e6875700bbff37008c1f780020002000fa
:108e6000801f7800c2c12900821f780010042000f2
:108e7000ee0f07000c0378002505200014042000e5
:108e800033052000e2c02900b1552000d04629005a
:108e9000b30f0700e6875700a2ff37000000fa0073
:108ea000889fbe0000047800814478000000e9003b
:108eb000e10f50001c003e00010420000800780073
:108ec0007cff07000000e00008003200a003200043
:108ed0000040b80082532100020040000948780099
:108ee0004f04be000080fa0000000600881f7800d2
:108ef000f0c52900801f780040042000cb0f070038
:108f000008037800d5042000440420003305200025
:108f1000b2c92900213e2000d0462900900f070049
:108f2000e4875700e9ff3700881f78002000200001
:108f3000801f7800e2ca2900821f780010042000f8
:108f4000ba0f07000803780025052000140420004c
:108f500033052000b2c92900d13d2000d0462900a8
:108f60007f0f0700e6875700d3ff37000000fa00a5
:108f7000b214e2002000320052a4800063a48000fa
:108f8000c0122000801f780047af2100062020007b
:108f9000457f2100640020003100200010002000e7
:108fa00019fc07008f87e9000000e00002003a008a
:108fb0000080fa000000060010002000801f7800ea
:108fc00060cf2900801f780050042000970f070011
:108fd00016002000d5042000540420003305200092
:108fe00042d22900b1542000d04629005c0f07006e
:108ff000e4875700eeff370032a4800043a48000ce
:10900000dfff37000c00fa00889fbe008a1f78003f
:10901000d4a2a8008025200001002000008fbe00ff
:1090200071b980000810200001005400e10f5000c9
:10903000630034000005eb0001015400a3d22100bd
:10904000838040008e01780010002000aff90700f7
:109050000000e0000f003c000b003500e4d22900c6
:10906000841f780000322000700f07008f87e9000e
:10907000d4a2a9000a0078004f0578004f04be0072
:109080000080fa00000006002e37b5000085eb00d6
:10909000f7ff37002e37b4001a002000bf01070089
:1090a000200798003107980042079800530798005e
:1090b00084702100009abe000292be00b8bc8000fd
:1090c000c9bc80000800be0036ec0700e00f540069
:1090d000e08f5c00350035000002be000203be00d8
:1090e0002e009000be0090004e019000de01900026
:1090f0002fec070043ed070080b9880091b9880084
:1091000070b9800072d22100820040002e37ef003b
:109110008001eb0001007800a4d22100848f500070
:109120000600390042c2b300904f11001d0032000a
:109130000000e900840f5000fbff31000300e00055
:1091400011003200838050008100e800027121008c
:109150000300780011130700000478000000e0000d
:10916000c3ff3200e30f40000500320094d4290011
:10917000841f7800f03220002c0f07008f87e90051
:109180000885e900baff370023d72900831f78003c
:10919000e0322000250f07002e37ef00eaff2f00f6
:1091a000b2ff370080017800e4ff37006022b8008a
:1091b00006002000071f24007dec0700c6ff3700d3
:1091c00080da2900801f780040332000170f070045
:1091d0008000eb002e37ef008f87e90095ff370006
:1091e0000000fa00b0a48000c1a4800080b888000c
:1091f00091b88800d0a48000e1a48000a0b88800c5
:10920000b1b888000080fa00000006000800fa00eb
:10921000889fbe008a1f78000004be000205780007
:109220009e57e200400032000a00e00027003a00aa
:1092300011c1bf000078a30003003200d4e2a800ef
:109240000140fe00d4e2a90054010700487a210041
:109250003802be002803be0016ed07006022b800e9
:1092600006002400f708240014ed0700009fbe004c
:109270000297be00b8bc8000c9bc80000800be00d8
:10928000c8eb0700e00f5400e08f5c000a003500d7
:109290000002be000203be003e00be002e01be0062
:1092a000c3eb0700d7ec07004f0578004f04be0062
:1092b0000080fa00000006006022b80006002000ce
:1092c000071f24003aec0700f1ff37000800be003a
:1092d000230007000000e00005003a002f0107000e
:1092e000487a2100009cbe000294be00d6ff3700e1
:1092f00024dd2900841f780060192000cb0e0700b0
:109300000003eb00d5042000641920003304200082
:10931000c2de2900a104200010df2900900e070002
:109320008f87e900edff370090df2900801f78006c
:1093300050192000bd0e07000003eb00d5042000eb
:109340005419200033042000c2de2900e10320006c
:1093500010df2900820e07008f87e900b2ff370077
:109360000000fa00889fbe000004be009e57e20085
:1093700036003200e00f5400e08f5c00250034001e
:1093800011c1bf000078a30003003a009ed7bf00c0
:109390000018a3000d00320000e22900801f7800b1
:1093a000a0192000a10e07000003eb00d504200047
:1093b000a419200033042000c2e429006109200020
:1093c00010df2900660e07008f87e9000821ef00f3
:1093d0000621ef00d4bc8000e5bc80000821b80065
:1093e00009a0b9000080410005c2b9008401400015
:1093f000620888007308880011e1a80030c0b3003b
:109400009ef7b7000000eb004f04be000080fa009a
:109410000000060060e52900801f78005019200038
:10942000820e07000003eb00650520009419200060
:1094300033042000c2e429000109200010df2900c4
:10944000470e07008f87e900cdff3700f0e72900be
:10945000801f780090192000740e07000003eb00b5
:10946000d50420009419200033042000c2e4290010
:10947000b108200010df2900390e07008f87e900ae
:10948000bcff3700809fbe00829fbe000000fa0034
:1094900011e1a900d4c2bf000080fb004700de003c
:1094a000d4e2a90084e0a90002bd800013bd8000c1
:1094b00061014100e081490002bd880013bd8800c0
:1094c00051c0b3008000fd009ef7b7008000fd0092
:1094d0004700dd00412d2000914078000174a1007b
:1094e00080c0700001007800d4e2b7000080fa006c
:1094f0004f01be004f00be00004006000000fa0011
:10950000889fbe000004be009e57e2001f0032008c
:109510000800be0092ff07000000e0000d003a00c6
:1095200011c1bf000078a30006003200d4e2a800f9
:109530000140fe00d4e2a90011c1bf000078a300e1
:10954000faff3a000000eb004f04be000080fa0072
:1095500000000600b0ea2900801f78008019200072
:10956000320e07000003eb00d50420008419200010
:109570003304200032ed29006107200010df2900ac
:10958000f70d07008f87e900e5ff370090ed290010
:10959000801f780070192000240e07000003eb00e4
:1095a000d5042000741920003304200032ed290076
:1095b000c106200010df2900e90d07008f87e900b0
:1095c000d3ff37000000fa0011e1a9000821ef00e5
:1095d0000621ef000e21ef0070088000600888006f
:1095e00050c0b3009ef7b7000000eb000080fa0007
:1095f000000006000000fa001221ef009008800031
:10960000800888000821ef000621ef000e21ef00fe
:10961000700880006008880080cfb3009760b600b3
:1096200097c0bf00f1c8b300014060000054a00023
:1096300097e0b7008cc0a9008ce0a80084c0a90006
:1096400084e0a9001061a80011a1a900f0ccb3002a
:109650001061b60050c0b3009ef7b7000080fa005a
:10966000000006000000fa0000002000211c20007d
:10967000f0bd880001be8800b0bc8800c1bc880075
:10968000303327000100200010be880021be880072
:10969000d0bc8800e1bc8800300a200030be8800c1
:1096a000c837ef00020007000080fa000000060043
:1096b0000000fa002021ef0000098000f008880077
:1096c0001621ef001421ef001c21ef00e0088000bc
:1096d000d0088800f0c8b3009e60b6009fc0bf00ed
:1096e00081cfb300014060000014a0009fe0b700ec
:1096f0008ea0a9008ec0a80086a0a90086c0a900df
:109700001e61a8001fa1a900f0ccb3001e61b60025
:109710000080eb00d0088800e00888001fe1a80066
:1097200030c0b300ccf7b7000080fa00000006009c
:109730000000fa0086c0a900ca37ec000080fa00d9
:10974000004006000000fa00cc57e2000a00320098
:10975000a008800001002000b20880000300200063
:10976000c011dd0002002000020070008380700044
:109770000080fa00000006000003eb00d504200082
:10978000341320003304200022f02900d1092000e6
:1097900090f02900720d0700edff37000800fa0075
:1097a000889fbe008a1f7800cc57e2003c00320040
:1097b00042c0bf000080fb004505de000a007800c3
:1097c000d4f7b70000ceb3004260b700a80880000d
:1097d00009002000b008800001002000c000dd006a
:1097e0000000200000047400818474000800be00a2
:1097f0006cea0700009fbe000297be00e00f540015
:10980000e08f5c001f00350058be80006140b90049
:1098100064ea07000800e000150035006022b80087
:1098200006002000071f2400a4eb07000002be0072
:109830000203be003e00be002e01be00dcea0700af
:10984000c552dd0024042000144278007f426200eb
:10985000054272000002fd0042e0b7000002fd0078
:109860004f0578004f04be000080fa00000006009b
:109870006022b80006002000070f2400ccea070091
:10988000e6ff37006022b80006002000071f240012
:10989000c7ea0700009fbe000297be00daff37004c
:1098a0000003eb00d5042000341320003304200013
:1098b00012f12900310b200090f02900280d07003b
:1098c000bbff37003c00fa00889fbe008a9fbe00a5
:1098d0008c9fbe00b214e200b805320050a4800094
:1098e00061a48000809fbe0040352b00801f78005f
:1098f000a50d0700a1c0b3001000200067fd070000
:10990000e68757001d00200031362b00e04921007a
:1099100042f507000000e000a105320082002000af
:10992000a1362b0010002000f7f807000e00780089
:10993000180009000018eb008001eb002203200052
:109940008e0078001000200070f70700a0c0b30060
:109950002077980012002000210320008e80400014
:1099600002007800e8f807000e0478001e40780036
:109970000004e00005003200e84f50006b053200a3
:10998000584078000004e000fbff3a000e04780025
:10999000f9c3b300184078000004e0000900320069
:1099a0000080fb005ada07000000e0005d053a0085
:1099b00018407800894f5000020032000804e80087
:1099c000f4ff3700ed4f5000cfff32000004e000fd
:1099d000cdff32000045eb000006eb002c1f980085
:1099e000330320008e814100420320000e0141001c
:1099f00011c52a00080078002bf507000004780044
:109a00000000e000c0ff32002e1890000800500057
:109a10008004e9000001eb00321f98008000eb0099
:109a2000680ab80040232b000002420009017800b8
:109a30008800780014007800ccf407000000e000f3
:109a400036053a000a45e8003e1990006810b80053
:109a500043232b00030640000201e800321f980058
:109a60008200780030022000800f5100ecff3600a9
:109a70000a04e00024053200e14f55001d053c00ba
:109a80002e1c9000080278003c4090000081fb00f2
:109a90000300200091032000810f5100e08f590046
:109aa00006053e0002600100400037000305370054
:109ab00064003700a0003700d4003700ff043700ef
:109ac000fe00370006013700fc043700480137006c
:109ad0007f013700a4013700f40137001e02370070
:109ae000f6043700f5043700080137003b02370061
:109af0006e023700f10437009e023700ef04370092
:109b0000ce023700f0023700f1023700f2023700d0
:109b1000f7023700e9043700e8043700e7043700ac
:109b2000e6043700e5043700f8023700e3043700a5
:109b30002d0337005603370081033700ee0337004b
:109b40001e0437003a043700dc0437007204370083
:109b5000a50437000e003700d8043700d7043700bb
:109b6000d6043700a3043700d4043700d3043700e9
:109b7000d2043700d1043700d0043700cf043700b7
:109b8000ce043700cd043700cc043700d0043700b2
:109b900022402d00821f780033372b00831f78006e
:109ba000f90c0700e487570057ff370040c4b300a3
:109bb000cef7b7005c0f070080c4b300cef7b70044
:109bc00041a68000006f8000808f50000f0032009f
:109bd000801f7800811f780022382b00821f7800b8
:109be000d00e2000910c0700066f80006505200054
:109bf000d40e200023052000023d2b00e11320009d
:109c0000d03d2b00560c0700e6875700f4072000d4
:109c1000f30f2000220b20006148210080572f0005
:109c2000b21b0700130e0700f4072000f30f2000fb
:109c30008257200021de200000002f00ab1b070010
:109c400031ff3700330320008e81410042032000a2
:109c50000e01410011c52a000800780092f40700a7
:109c60000000e0001b003200a20020008000eb009a
:109c7000b1d907000004be000001be00e206b10039
:109c80000380b10020192c0011002000800f51002a
:109c9000818f590007003600889fbe009c1f780006
:109ca000403e2b00801f7800b70c0700e887570064
:109cb00015ff370058a4880069a48800f407200025
:109cc000f30f200042002000a1482100c0572f00c0
:109cd000861b070072a4800083a48000829fbe00c0
:109ce00050a4800061a48000809fbe00a1402b0092
:109cf000811f7800a40c070052a4800063a4800098
:109d000010002000fefb0700007d20000100200065
:109d1000571b070070c4b300cef7b700ea8757009f
:109d20000000eb004f06be004f05be004f04be0012
:109d30000080fa0000000600330320008e814100fd
:109d4000420320000e01410011c52a0008007800de
:109d500055f407000000e0001d003200a2002000c2
:109d60008000eb0074d907000004be000001be00b3
:109d7000e206b1000380b10020192c001100200080
:109d8000800f5100818f590005003600889fbe006a
:109d90009c1f7800423e2b00821f7800c2ff3700d4
:109da00078a4880089a48800f4072000f30f20001d
:109db00042002000e148210000582f004b1b070003
:109dc00072a4800083a4800020002000ccfb070048
:109dd00070a4800081a48000809fbe0052a48000f7
:109de00063a48000829fbe00a3402b00831f7800e5
:109df000650c070070c4b300cef7b700007d2000eb
:109e0000010020001a1b0700c4ff370033032000a5
:109e10008e814100420320000e01410011c52a003d
:109e20000800780020f407000000e0001400320071
:109e3000a20020008000eb003fd907000004be0014
:109e40000001be00e206b1000380b10020192c0021
:109e500011002000800f5100818f5900cbff3e0080
:109e600038a4880049a48800f4072000f30f2000dc
:109e7000420020006148210080572f001b1b070073
:109e800030a4800041a48000809fbe00e1452b00eb
:109e9000811f78003c0c0700803e2000010020005c
:109ea000f31a070032a4800043a4800010002000b1
:109eb00093fb0700e687570093fe370072a48000eb
:109ec00083a48000829fbe0050a4800061a4800013
:109ed000809fbe00a1402b00811f7800c4ff370087
:109ee000f2012000d1472b001000200086f7070068
:109ef000007d200001002000dd1a07001000200076
:109f0000bcf907000000fe002e1a90003303200069
:109f10008e814100420320000e01410011c52a003c
:109f200004007800e0f307000000e00029003200a0
:109f30009040780090c7b30080cf500021003200dd
:109f400090c5b30080cf50001e00320010c3b30094
:109f500080cf50001b00320040c7b30080cf5000bc
:109f60001800320040c5b30080cf50001500320009
:109f70007140400080cf50001200320050c4b30046
:109f800080cf50000f003200bc34ef0032002000c0
:109f9000d1492b00100020005bf707005201200080
:109fa000114a2b001000200057f70700f40720008b
:109fb000f30f200022002000c14b2100e05a2f00a7
:109fc0001eff3700eda5880022002000714b2b00fa
:109fd000f0ff370000cb2a00801f78009c1f78001c
:109fe000a14b2b00811f7800e70b0700b1ff370062
:109ff000330320008e814100420320000e01410006
:10a0000011c52a0008007800a7f3070000047800b3
:10a01000624e2b000000e000280032003fda07000b
:10a02000301f9800e60f50001f003c000001e900bf
:10a03000321f98008204780011003b0088007800ed
:10a04000e049210081da0700f4072000f30f200027
:10a0500082002000e149210000592f00a31a0700c7
:10a06000e1492100811f7800024f2b00821f7800f8
:10a07000c50b0700e077ef00ae75ef00c9fe3700b3
:10a0800068c07c000080fb0075da070000f47c00eb
:10a090003e1890000001e900321f98008204780009
:10a0a000f7ff3b00e5ff3700881f78009c1f780012
:10a0b00010512b00801f7800cbff3700821f7800e3
:10a0c0009c1f7800a34b2b00831f7800c6ff37002e
:10a0d000330320008e814100420320000e01410025
:10a0e00011c52a00080078006ff30700b1d82a00d4
:10a0f0000000e000170032000001eb008000eb00e0
:10a100005eda0700ef0f5000e08f580005003600c0
:10a11000809fbe009c1f780063542b00831f780033
:10a12000e1fe37006f00600030a58800f4072000d2
:10a13000f30f200022002000614a210080592f00e7
:10a140006a1a0700a614f800a0572b00801f780099
:10a1500093fe3700811f78009c1f7800a24b2b00d4
:10a16000821f7800a0ff3700330320008e8141005a
:10a17000420320000e01410011c52a0008007800aa
:10a1800049f30700000478000000e00045003200b9
:10a190002eee07000005be00f2ff2f00f3f72700a8
:10a1a000a3e607000000e00006003a00881f7800e0
:10a1b000e3fb2a00831f78009c1f780060592b0066
:10a1c000b8fe37002e189000330320008e81410026
:10a1d000420320000e01410011c52a0032f307009e
:10a1e000000478000000e0002c00320017ee0700a9
:10a1f000401f9800511f9800f2ff2f00f3f727002f
:10a200008be607000000e00021003200baa48800bd
:10a21000cba488004e199000de199000d2a48800cb
:10a22000e3a48800f4072000f30f20004200200080
:10a230006149210080582f002c1a0700f4072000e4
:10a24000f30f200042002000a1492100c0582f0038
:10a25000261a0700d0a48000e1a4800008e70700c8
:10a26000809fbe00829fbe00b0a48000c1a4800079
:10a2700003e70700809fbe00829fbe00935b2b0018
:10a28000831f7800400b0700f28757009efd3700c0
:10a29000881f7800d3fd2a00c6ff3700d1fd2a00b1
:10a2a000acff3700b1f72a00aaff370033032000c4
:10a2b0008e814100420320000e01410011c52a0099
:10a2c00008007800f8f20700000478000000e000c1
:10a2d0001f003200dded07000005be00f2ff2f0079
:10a2e000f3f7270052e607000000e00006003a00fe
:10a2f000881f7800e2fb2a00821f78009c1f7800ec
:10a3000063592b0085ff3700baa48800cba48800ce
:10a31000f4072000f30f20004200200061492100d3
:10a3200080582f00f1190700b0a48000c1a480005c
:10a33000d3e60700809fbe00829fbe00105e2b0008
:10a34000801f7800100b0700ea8757006efd37006a
:10a35000e0fb2a0020ff3700330320008e814100fc
:10a36000420320000e01410011c52a0008007800b8
:10a37000cdf20700000478000000e000c7ff3200c3
:10a38000b2ed07000005be00f2ff2f00f3f7270033
:10a3900027e607000000e000bdff3200daa48800d5
:10a3a000eba48800f4072000f30f200042002000f7
:10a3b000a1492100c0582f00cc190700d0a480006b
:10a3c000e1a48000aee60700809fbe00829fbe0031
:10a3d000d15f2b00811f7800daff370033032000a4
:10a3e0008e814100420320000e01410011c52a0068
:10a3f00008007800acf207000000e00029003200fd
:10a400009040780090c7b30080cf50002100320008
:10a4100090c5b30080cf50001e00320010c3b300bf
:10a4200080cf50001b00320040c7b30080cf5000e7
:10a430001800320040c5b30080cf50001500320034
:10a440007140400080cf50001200320050c4b30071
:10a4500080cf50000f003200be34ef0032002000e9
:10a46000d1492b001000200027f60700b201200080
:10a4700091612b001000200023f60700f407200054
:10a48000f30f200022002000e14b2100005b2f0091
:10a49000eafd3700fda5880022002000714b2b004b
:10a4a000f0ff370002cb2a0004ff370033032000ff
:10a4b0008e814100420320000e01410011c52a0097
:10a4c0000800780078f207000000e000c1fe3200ca
:10a4d0009040780090c7b30080cf50002100320038
:10a4e00090c5b30080cf50001e00320010c3b300ef
:10a4f00080cf50001b00320040c7b30080cf500017
:10a500001800320040c5b30080cf50001500320063
:10a510007140400080cf50001200320050c4b300a0
:10a5200080cf50000f003200c034ef003200200016
:10a53000d1492b0010002000f3f50700a2012000f4
:10a5400051632b0010002000eff50700f4072000f6
:10a55000f30f200022002000014c2100205b2f007f
:10a56000b6fd37000da6880022002000714b2b009d
:10a57000f0ff3700330320008e81410042032000aa
:10a580000e01410011c52a000800780046f20700bc
:10a590000000e000c3ff32009040780090c7b30095
:10a5a00080cf50002100320090c5b30080cf500012
:10a5b0001e00320010c3b30080cf50001b003200d9
:10a5c00040c7b30080cf50001800320040c5b30030
:10a5d00080cf5000150032007140400080cf500005
:10a5e0001200320050c4b30080cf50000f00320080
:10a5f000b034ef0032002000d1492b0010002000c1
:10a60000c1f507009201200001652b001000200019
:10a61000bdf50700f4072000f30f20002200200002
:10a62000014b2100205a2f0084fd37008da58800a2
:10a6300022002000714b2b00f0ff37004c232b0031
:10a64000a0662b00801f780061672b00811f7800b7
:10a65000b2672b00821f780033682b00831f7800bd
:10a66000490a07000001eb00321f9800e8875700f5
:10a67000380220002c4090000004e00007003a005f
:10a68000680646000200e800301f980000017800cc
:10a69000880f5000f7ff36009bfc37003c0090000d
:10a6a000801f7800ac009000811f78009c1f78000c
:10a6b00033682b00831f7800330a0700e8875700b0
:10a6c0003e199000eeff3700fb0b07008efc3700b1
:10a6d000f30707008cfc3700c834ef00c2052000e8
:10a6e00041692b001000200087f50700f8ff3700b4
:10a6f00080f1290089d807000001780081f1290044
:10a700001000200080f507007ffc37003303200095
:10a710008e814100420320000e01410011c52a0034
:10a7200008007800e0f1070003cb2a000000e000f9
:10a73000290032009040780090c7b30080cf5000cd
:10a740002100320090c5b30080cf50001e003200bf
:10a7500010c3b30080cf50001b00320040c7b300cd
:10a7600080cf50001800320040c5b30080cf5000a9
:10a77000150032007140400080cf500012003200be
:10a7800050c4b30080cf50000f003200ba34ef0045
:10a7900032002000d1492b00100020005af507009c
:10a7a000b2012000116f2b001000200056f50700a9
:10a7b000f4072000f30f200022002000a14b21000d
:10a7c000c05a2f001dfd3700dda5880022002000a3
:10a7d000714b2b00f0ff3700831f78009c1f78001f
:10a7e000a04b2b0033fe3700330320008e81410045
:10a7f000420320000e01410011c52a000800780024
:10a80000a9f107000000e0001f0032000001eb008a
:10a810008000eb0099d80700421f2000820f5000f3
:10a82000e08f580006003600809fbe00431f2000c6
:10a83000831f78009c1f7800d0702b00c0fe37006b
:10a84000a0a58800f4072000f30f200022002000bc
:10a85000414b2100605a2f00a4180700a0a58000da
:10a860000000e00005003200801f780041742b00da
:10a87000811f7800e2742b0039fe370002022000ad
:10a8800011772b009eff370090de2a00d2fd3700a3
:10a89000330320008e814100420320000e0141005d
:10a8a00011c52a00080078007ff1070093de2a0016
:10a8b0000000e000c8ff32000001eb008000eb0068
:10a8c0006ed80700e10f4000e08f58000a00360004
:10a8d000809fbe00f2ff2f0003002000829fbe0079
:10a8e0009c1f780023792b00831f7800a60907009e
:10a8f000ec87570004fc370020a68800f4072000ee
:10a90000f30f200022002000414c2100605b2f004b
:10a910007618070020a680000000e0000500320045
:10a92000801f7800a07c2b00801f7800e1742b0032
:10a93000acfd3700b2012000a17d2b0070ff370075
:10a94000330320008e814100420320000e014100ac
:10a9500011c52a000800780053f1070000047800b0
:10a960000000e00062003200c04c21001f0009001e
:10a970000018eb0062002000617f2b0008007800c7
:10a98000faf007000000e0004d0032000001eb008b
:10a99000321f980008007800e0d70700e84f500009
:10a9a0003b003e008004eb000085fb00e00f15003b
:10a9b00007003d0068c07c000080fb0028d807002d
:10a9c00000f47c008904e8008a8f5400f9ff350008
:10a9d0003e1890006800b800c24c21000200400000
:10a9e0000a01780088007800a7d707002e18900089
:10a9f000330320008e814100420320000e014100fc
:10aa000011c52a0028f10700000478006e75900037
:10aa10003e1890000001e800321f9800e70f510037
:10aa200002003c000800e000daff3a00e14f450078
:10aa30000d0032000a40e80038f5b700f4072000a6
:10aa4000f30f200002042000c14c2100e05b2f0026
:10aa50002618070038d5bf000080fb00801f780053
:10aa6000d07f2b00b9fd37009c1f780043822b005c
:10aa7000831f780044090700f30f20000204200020
:10aa8000e15b2f00c04c2100ab18070045fc3700ec
:10aa900082002000821f7800881f78003e189000f6
:10aaa000801fe8009c1f7800f0842b00801f780036
:10aab0003509070000c5eb00ea875700dbff3700c8
:10aac0003875ef00f4072000f30f20000204200087
:10aad000c14c2100e05b2f000418070071882b0097
:10aae000811f7800280907008f87e90086fb37005f
:10aaf000438a2b0038ff3700330320008e8141004a
:10ab0000420320000e01410011c52a000800780010
:10ab1000e5f007000000e000260032000001eb0035
:10ab20008000eb00d5d707000004be00e00f500006
:10ab3000e08f5800050032006a005000e0805800a5
:10ab4000eb0f4000e08f580012003e00b8a58800cf
:10ab5000f4072000f30f200022002000614b2100a9
:10ab6000805a2f00e1170700b0a580000000e00028
:10ab700005003200801f7800e28a2b00821f7800d7
:10ab8000e3742b0050fd370072012000518b2b0025
:10ab9000dbfe3700889fbe00809feb00a0002000f6
:10aba000801f78009c1f7800d18c2b00811f7800bb
:10abb0004eff370092de2a0040fd370033032000ad
:10abc0008e814100420320000e01410081902b0044
:10abd00008007800b4f0070000047800b3902b0060
:10abe0000000e000fcfe3200c0502100150009000a
:10abf0000018eb00b202200088007800c05021004d
:10ac000021d70700f4072000f30f2000c202200024
:10ac1000c1502100e05f2f00b4170700c150210090
:10ac2000811f7800a2912b00821f7800dcfb370087
:10ac3000d0932b000800e000e7fc32009840780039
:10ac4000f0c2b30080cf50000f003200c0c5b30087
:10ac500080cf50000c00320000cdb30000c0400097
:10ac6000e94f500008003600f0c9b30000c04000b2
:10ac7000e94f500004003600f0cbb30000c04000a4
:10ac8000f94f50001f003e009840900000c2b300f2
:10ac900080cf500016003400f0c7b30080cf5000c2
:10aca000130032001800fb004800dd008100fb00ab
:10acb00001007000c0a58800f4072000f30f2000f9
:10acc00022002000814b2100a05a2f008717070087
:10acd000ae189000114090000000fb00801f78002b
:10ace0001100fb00801f780090942b00f1fc3700ce
:10acf00062962b00821f78009c1f780083982b009f
:10ad0000f1fc3700c19a2b00811f78009c1f78004e
:10ad100082982b0012fd3700330320008e81410002
:10ad2000420320000e01410011c52a0008007800ee
:10ad30005df0070093ff2a000000e000a6fe32004d
:10ad40000001eb00410320008e8040004bd707003c
:10ad50000004be002e1890009040780060c6b3003a
:10ad600080cf50001200320060c4b30080cf50008a
:10ad70000f00320098a48800a9a48800889fbe0014
:10ad8000d39d2b00831f7800209f2b00801f78000d
:10ad90007d080700e8875700f4072000f30f200024
:10ada000420020002149210040582f00a3fb37001a
:10adb0000800be0051e4070052b82e00130524001d
:10adc000b3e60700f4e6070090a48800a1a4880079
:10add000889fbe00d19d2b00811f780002a02b0010
:10ade000821f7800eaff3700a002200090150700bc
:10adf000c5fa3700330320008e8141004203200052
:10ae00000e01410011c52a000800780026f0070055
:10ae100000047800c1a02b000000e000cdfc32004f
:10ae20009040780040c6b30080cf50001c00320034
:10ae300040c4b30080cf50001900320000c7b300f7
:10ae400080cf50000700320000c5b30080cf500013
:10ae500004003200881f78009c1f780083a12b001b
:10ae600099fc37008000200030a6880002072000ef
:10ae7000321f9800e201200011a42b0010002000d6
:10ae8000a1f30700f4072000f30f200022002000a8
:10ae9000610320008e804000805b2f0067fb37003d
:10aea0004000200030a6880042062000321f980093
:10aeb000e201200001a62b00f0ff37000080fb001c
:10aec000801f7800f1a72b00811f780034fb37002a
:10aed000cfd7bf0000c0ea00cff7b70031aa2b00e0
:10aee00001003a0061aa2b00811f7800a0aa2b0064
:10aef00096fc37008e1f780072ab2b00821f780003
:10af000013ac2b0070fc37008e1f780020ad2b0097
:10af1000801f780011ac2b0032fc37003e199000e6
:10af2000cdfa370018407800a6fa37008e0f54008b
:10af30000f0032000804e900281f9800080278007a
:10af4000184078000004e0008efa3200a44190001e
:10af5000034a78002e1890000002e800241f980091
:10af60001404e000f9ff3a001840780085fa370031
:10af70000e0278002e1f98001e04e000faff320037
:10af800014419000024a78002e1890000002e80058
:10af9000241f98001404e000f9ff3a00f2ff370084
:10afa000a1ad2b00811f7800f707070010c0b30088
:10afb000e0f7b7008f87e90058fa370030a4800027
:10afc00041a4800047fa37003000fa00889fbe0095
:10afd0008a9fbe008c1f7800800578000000e0008a
:10afe000650132008004eb006e8545000904d00045
:10aff00042ca2b00020444001800780047d607001c
:10b00000000178008a00780018007800e4d6070074
:10b010000000e000540132008904e800f98f540078
:10b02000f2ff3600ca1520000b054500f8844500e4
:10b030003b0c9000d0c7b300994f10003b01320089
:10b040005bf892000004a000d0fd9a00194078003f
:10b050000080fb00010020007c005000e0805800d0
:10b06000f2052000820f5000e08f58006a003e0079
:10b0700000600100ed003700ec003700660037008b
:10b0800065003700640037006d003700620037004c
:10b0900061003700570037005f0037005e0037005f
:10b0a000e20037005c0037005b0037005a003700d1
:10b0b0005900370058003700570037005600370056
:10b0c0009b00370054003700530037005200370010
:10b0d00051003700500037004f0037004e00370056
:10b0e0004d0037004c0037004b0037004a00370056
:10b0f000490037004800370051003700460037004c
:10b10000450037008a00370043003700420037000f
:10b1100041003700400037003f0037003e00370055
:10b120003d0037003c0037003b0037003a00370055
:10b130003900370038003700370037003600370055
:10b140003500370034003700330037003200370055
:10b1500031003700300037002f0037002e00370055
:10b160002d0037002c0037002b0037002a00370055
:10b170002900370028003700270037002600370055
:10b1800025003700a90037002300370022003700d0
:10b1900021003700200037001f0037001e00370055
:10b1a0001d0037001c0037001b0037001a00370055
:10b1b0001900370018003700170037001600370055
:10b1c0001500370014003700130037001200370055
:10b1d00011003700100037000f0037000e00370055
:10b1e0000d0037000c0037000b0037000a00370055
:10b1f000090037000a01780088007800090078000b
:10b20000e60a07000000e00003003a005bf8920045
:10b210000014a000d0fd9a005bf89200620060006c
:10b220000000cf000000e9004f00de004f0678006c
:10b230004f05be004f04be000080fa00000006006b
:10b240005980fb0069d607000000e00018003a00b2
:10b250008000eb0009007800ef010700008dbe00c0
:10b26000f2ff2f00f3f7270071e207000000e00073
:10b27000e9ff3200e9844400110020000900780051
:10b28000e50107002005980031059800f2ff2f0026
:10b29000f3f7270066e207000000e000deff32005f
:10b2a0005bf892000034a000d0fd9a00d7ff370071
:10b2b00082002000890078000e00780072d5070017
:10b2c0000046eb000c4f98008000eb000e00780069
:10b2d000b7000700008dbe00f2ff2f00f3f7270034
:10b2e00053e207000000e000cbff3200e984440095
:10b2f00078044700920020000800be0062d50700d5
:10b300001c6798001100200008007800a8000700c2
:10b310002005980031059800f2ff2f00f3f7270071
:10b3200043e207000000e000bbff3200b7ff370038
:10b330008904e80069449000f0c2b300804f5400d3
:10b340001d003200a0c7b300804f54001a00320025
:10b3500080c6b300804f5400afff3a0021002000a8
:10b3600009007800e4ec0700005d9800f74f5000fa
:10b37000a9ff3e008984e800210020000900780030
:10b38000ddec0700105d9800b8c3b300804f540097
:10b39000a1ff39008984e80021002000090078001d
:10b3a000d5ec0700205d9800804f54009aff3900cb
:10b3b000e3844400beff370021002000090078002c
:10b3c000cdec0700705598000040e900fe4f50009a
:10b3d00091ff3e008984e8002100200009007800e8
:10b3e000c5ec0700005d9800f74f50008aff3e0053
:10b3f0008984e8002100200009007800beec0700e5
:10b40000105d9800b2c3b300804f510082ff390035
:10b41000a0c7b300804f5400e5ff3a005bf89200ec
:10b420000044a000d0fd9a00e1ff37005bf89200d5
:10b430000024a000d0fd9a006b489000d5010700c1
:10b440006a00b900000478007b489000d101070031
:10b45000000444006140b900a8e20700008dbe006e
:10b460000b509000cb0107006a00b900000478007f
:10b470001b509000c7010700000444006140b90060
:10b480009ee20700020020000327240000e50700d9
:10b490000001be001a00be001ce20700008dbe00c5
:10b4a0002b509000bb0107006a00b900000478002f
:10b4b0003b509000b7010700000444006140b90010
:10b4c0008ee2070002002800b35b2400f0e40700ce
:10b4d0000001be001a00be000ce20700008dbe0095
:10b4e0001b509000c60107000000e00003003a0076
:10b4f0001a00be0001f0a200008dbe003b5090007b
:10b50000bf010700000478002b509000bc01070029
:10b51000800078000900e80008417800c6010700b3
:10b52000200598003105980038ff37005bf892003d
:10b530000074a000d0fd9a00a1032000090078004b
:10b54000b0d5070000017800100020000200e000e4
:10b5500036ff320002805400000044000004e9007d
:10b560008204e800b6fe37005bf892000064a00099
:10b57000d0fd9a00abfe370080cd2b00801f7800f5
:10b5800040002000290607000003eb00e50420002e
:10b59000440020001304200042d02b00610320004f
:10b5a00020d12b00ee0507008f87e9008dfe3700c4
:10b5b0000200fa00889fbe008a9fbe008c9fbe00da
:10b5c00080057800010478000000e00002003200ed
:10b5d0001004e0000d003a0090d12b00801f78008d
:10b5e00010012000110607000003eb00e504200015
:10b5f000140120001304200012d42b009118200005
:10b6000020d12b00d60507008f87e9000800e00055
:10b6100058003a00210020000b00780036ec0700ab
:10b6200000017800000f78000000e0004f003500b6
:10b63000f4ff2f00f5f72700a0052000800f510030
:10b640003f003c008b85e800210020000b007800c3
:10b6500029ec070000047800000178000000e000f9
:10b6600040003500f4ff2f00f5f72700b00320005d
:10b67000800f510032003c00e3854500210020008e
:10b680000b0078001cec0700000578006140b90051
:10b690001ae207000004be006150b90017e207007b
:10b6a00002002000832c240079e407000001be0082
:10b6b0000800be0095e107000006be0001f0a100f1
:10b6c000020020000327240057e107000000e000eb
:10b6d00021003d001e0178006110b90007e207005b
:10b6e0000004be0002002000032724000c00be005e
:10b6f00067e407000001be000800be0083e1070008
:10b700000004be0001f0a10002002000432b240031
:10b7100045e107000000e0000f003c00ab40900056
:10b72000e0c4b30080cf50000400320009f0a20052
:10b730006540400080cf500007003a000802be007c
:10b740000400be004f06be004f05be004f04be0001
:10b750000080fa0000000600f4ff2f00f5f7270034
:10b76000f7ff37000001ea00beff37000001ea00e2
:10b77000afff3700310020000b007800deeb070040
:10b7800000017800000f78000000e0004400350060
:10b79000f4ff2f00f5f72700400b2000800f510029
:10b7a000e7ff3c00e3854500210020000b00780006
:10b7b000d1eb070000047800000178000000e000f1
:10b7c00035003500f4ff2f00f5f72700b003200007
:10b7d000800f5100daff3c00e38545002100200086
:10b7e0000b007800c4eb0700000578006140b90049
:10b7f000c2e107000004be006150b900bfe10700cc
:10b8000002002000832c240021e407000001be0078
:10b810000800be003de107000006be0001f0a100e7
:10b820000200200003272400ffe007000000e000e2
:10b83000c9ff3d001e0178006110b900afe10700ab
:10b840000004be0002002000032724000c00be00fc
:10b850000fe407000001be000800be002be1070056
:10b860000004be0001f0a1000200200043332400c8
:10b87000ede007000000e000b7ff3c00ab409000a7
:10b8800050c4b30080cf5000acff320009f0a200da
:10b8900072404000a7ff37000001ea00c9ff3700ef
:10b8a0000001ea00baff37000000fa00889fbe00de
:10b8b0008a9fbe008c1f78000005be000204be00f7
:10b8c000040678000200e00045003200e48f5400d6
:10b8d000340036000c00e0002b003a000a01be00e4
:10b8e00000002000412b240007e1070002fc2f008c
:10b8f000938b2400d0e0070027e4070032fa2700ea
:10b90000b30020000cd407000203be000002be00fa
:10b9100010c2b300004c4200920522000300200038
:10b920000600be0004d407000203be000002be00f1
:10b9300011c2b3000140420010449800b20520003b
:10b94000030020000600be00fbd307000203be0078
:10b950000002be0011c2b300014042002044980022
:10b9600001404300304498000040eb004044980000
:10b97000080078004f0678004f05be004f04be0057
:10b980000080fa000000060002002000433324007b
:10b990000a00be00dde0070002fc2f0093832400b4
:10b9a000d4ff3700891f7800e1d42b00811f780075
:10b9b000100120001d05070009037800e5042000a0
:10b9c0001401200013042000f2d72b006121200075
:10b9d00020d12b00e2040700e4875700bdff3700a9
:10b9e000c0d82b00801f7800100120000f05070031
:10b9f0000003eb00e50420001401200013042000e4
:10ba0000f2d72b002121200020d12b00d4040700e5
:10ba10008f87e900adff37000000fa00889fbe0065
:10ba20000004be000000e000030032001040780077
:10ba30000004e0000e003a0030db2b00801f78008d
:10ba400010012000f90407000003eb00e5042000ca
:10ba50001401200013042000b2dd2b00b1242000cb
:10ba600020d12b00be0407008f87e9001840780022
:10ba70000000fb00b40520000480b90052442f00f0
:10ba8000020040006101b900184090000000fb0076
:10ba9000cf80de0002004000838048000401b8002f
:10baa0000488b9008081410056442f00f7ff2f0021
:10bab0000201430083814b00284090000000fb00fe
:10bac000cf80de0002004000838048000401b800ff
:10bad000048ab900848141000201430083814b0044
:10bae000384090000000fb00cf80de0002014000e3
:10baf000838148001202b1000380b1000900e00018
:10bb000017003a000200be00fce0070002fc2f0014
:10bb1000938b24005ee307000001be0000002000bc
:10bb2000412b240078e007000004be0001f0a100d2
:10bb300002002000432b24003be007000000e0004f
:10bb400004003c000800be004f04be000080fa0064
:10bb500000000600f0ff2f00f1f72700faff370082
:10bb60000200be00e5e0070002fc2f0093832400e2
:10bb700047e307000200200043332c0063e0070086
:10bb80000004be0001f0a1000200200043332400a5
:10bb9000e9ff37000000fa000041780000cdb30053
:10bba00000404100e94f500006003e000280fb00cb
:10bbb00002fd2f0082004000010078000080fa00a2
:10bbc00000000600f0cbb30000404100e94f5000f8
:10bbd00003003e000280fb00f2fb2f00f5ff370060
:10bbe00000cbb300004041008000eb00e94f500063
:10bbf000f1ff3e000280fb0002fb2f00edff37004b
:10bc00000000fa008040780000cdb30000c0400082
:10bc1000e94f50000400360042062000c0c4b300c3
:10bc200080cf500001003a000001eb0002007800d4
:10bc30000080fa00000006000000fa00889fbe00a5
:10bc40008a9fbe008c9fbe0000047800814478006b
:10bc5000824678000000e0004900320098c04400ad
:10bc6000fcc5500002c3b30002c04000e94f5000c1
:10bc70003d003e0000cbb30080c545001840900059
:10bc80007c455000b0c3b300804f55000200360021
:10bc900040ccb30000454500284090007c46500051
:10bca0000b00fb00cf80de0094e007000004be0024
:10bcb0000b04e000270035000a00fb00cf80de0007
:10bcc0008ee007000a04e0001e003500020020009c
:10bcd00003272400eee207000001be000800be00ba
:10bce0000ae007000004be000c00fb00cf80de006d
:10bcf00082e007000c04e0000e003500020028007e
:10bd0000b35b2400e2e207000001be000800be00b1
:10bd1000fedf07000d04e0000100320001f0a20088
:10bd20004f06be004f05be004f04be000080fa0063
:10bd3000000006000200200003382400f3df0700a3
:10bd4000eeff37000200200003382400efdf070079
:10bd5000deff37000200200003382400ebdf07007d
:10bd60000004be00d4ff370062c2b30002c040002e
:10bd7000e94f5000c1ff3e0080457800bfff37000b
:10bd800080de2b00801f7800c00120002704070000
:10bd90000003eb00e5042000c40120001304200090
:10bda00022e12b001129200020d12b00ec030700f9
:10bdb0008f87e900a9ff37000000fa000200200089
:10bdc00003e823009cdf070014e307001002b00023
:10bdd0000080fa00000006000000fa00004278002f
:10bde000f6022000a2b12b008001eb0045c32b001e
:10bdf000850f510009003100924f520011003200ae
:10be000012409000804f5200070032006301410051
:10be10008301e800850f5100f7ff39000600780024
:10be20000080fa00000006002240900080cf500001
:10be3000f6ff3a0010022000030040000003ea0071
:10be4000f6ff37002240900080cf5000ecff3a0010
:10be50001602200003034300f0ff37001000fa0031
:10be6000889fbe008a9fbe008c9fbe00800678001f
:10be7000410798000000e00073013200ce009000fe
:10be80000100e00069013200c0152000008046007a
:10be90005007980029de2000e0ff2f00ce00900020
:10bea000800878000006eb0048a68000e00f140030
:10beb00018003100095990008280fb0040032000e7
:10bec000808f50003b0132006e003c000080e90092
:10bed000808f5000460032000000e800808f500044
:10bee000140032000280fb00801f7800e4eb2b007e
:10bef000841f780050032000cc030700e48757001c
:10bf000048a680000c06e800fc844400880f560018
:10bf1000e8ff3900ce029000808aeb0030a6800056
:10bf20004f06be004f05be004f04be000080fa0061
:10bf300000000600195890000080fb000058a30084
:10bf400028003a000048a3000d00320009007800e4
:10bf500072d2070000017800e680460009007800f0
:10bf600082eb07000000e000e5ff3a004e00900081
:10bf70000c087800195890006f006000e8ff370047
:10bf8000668446000800780064d20700000178004b
:10bf9000880078000900780074eb07000000e000da
:10bfa000d7ff3a00195890000068a3000a00320039
:10bfb000e94090008180fb005d4890000000d100c6
:10bfc0006f006000808f5000cdff3a00ce009000df
:10bfd0008c087800e7ff37004e0190000c097800cc
:10bfe000e4ff3700ce0290008c0a7800e1ff3700b2
:10bff000195890000080fb000058a3001e003a0072
:10c000000048a300090032000900780043d207006d
:10c0100000017800ee8046000900780053eb07002d
:10c020000000e000b6ff3a00ebff37006e844600e8
:10c030000800780039d207000001780088007800f5
:10c040000900780049eb07000000e000acff3a006f
:10c05000195890000068a300e2ff3200e940900008
:10c060008180fb005d5090000000d1006f006000f7
:10c07000808f5000a2ff3a004e0290000c0a780018
:10c08000bcff370060032000808f5000a900320001
:10c09000470035000000e800808f500091ff3a0013
:10c0a0005df892000018a30096ff3200b214e2007f
:10c0b0003a00320082b8800093b88000a0b88000b7
:10c0c000b1b88000de02900025029000b502900019
:10c0d000849fbe005e0290001403be000002be00fa
:10c0e0008e00780064004700b0ea0700e48757003c
:10c0f0000000e00023003a001e05be001901be004a
:10c100000a00be00c8de07000000e0007cff35002a
:10c1100039019000c90190000a00be00c4de07008a
:10c120000000e00076ff3c002e009000be00900072
:10c13000600798007107980069019000f90190006c
:10c14000b9de07000000e0006dff3500190d90001a
:10c15000a90d90006011b8000a00be004ae2070075
:10c160000000e0009cff32000a01be006e0090005b
:10c17000fe009000aede07000000e00060ff3c0023
:10c1800092ff370045ef2b00851f78003003200019
:10c19000260307008f87e90059ff3700b2a480000b
:10c1a000c3a48000d0a48000e1a48000c5ff3700b4
:10c1b0005df892000018a30052ff32001940780089
:10c1c0008080fb00e48f5000520032002c003c00c5
:10c1d000e28f50001a00320010003c00e18f500046
:10c1e000060032000080fb00801f780075f12b00f4
:10c1f000851f7800200320003fff37005e0290007b
:10c200001400be0039019000c901900086de0700cd
:10c210000000e0003bff340072ff3700de029000b8
:10c2200025009000b500900069019000f901900090
:10c230007dde07000000e00032ff34004bff3700d6
:10c24000de0290001500be0039019000c901900087
:10c2500075de07000000e0002aff34005e01900058
:10c2600022009000b200900069019000f901900056
:10c270006dde07000000e00022ff34007eff370083
:10c28000e68f50001b003200e58f50001400340090
:10c29000e78f500009003200e88f5000d1ff3a00cc
:10c2a000de0290001500be0039019000c901900027
:10c2b0005dde07000000e00012ff34005e01900028
:10c2c00022009000b200900069019000f9019000f6
:10c2d00057de07000000e0000aff3d0066ff370060
:10c2e0005e0190001200be0039019000c90190006b
:10c2f000f7ff3700de0290001500be003901900004
:10c30000c90190004ade07000000e000fdfe3d008c
:10c31000eaff3700de0290001500be0039019000f0
:10c32000c901900042de07000000e000f5fe3d007c
:10c33000caff37005df892000018a300f1fe32003a
:10c340005e0090001005be001901be000a00be008c
:10c3500037de07000000e000eafe3c0069019000c3
:10c36000f90190000a00be002fde07000000e00087
:10c37000e4fe3500de00900021059000b10590003c
:10c3800039019000c90190000a00be0026de0700b6
:10c390000000e000dbfe350019099000a9099000bb
:10c3a0000a00be0022de07000000e000d5fe3c00cf
:10c3b00009ff37005df892000018a300d1fe32009b
:10c3c00069029000f902900039019000c9019000c3
:10c3d000de00900021009000b1009000809fbe0020
:10c3e0005e0090001003be008e00780064004700dd
:10c3f000eee90700e48757000000e00007003a007c
:10c400001901be002e009000be00900008de07005b
:10c410000000e000bafe3c00effe370041ef2b00c9
:10c42000811f78001003200059ff370032f52b00e0
:10c43000821f7800e00220007c020700100020002c
:10c440008f87e900b6fe3700f0f72b00801f7800d9
:10c45000d0022000f8ff37000000fa00889fbe00dd
:10c460008a9fbe008c9fbe000004be00820578003b
:10c470000000e0007c0032000900e0006c003200a7
:10c480000b08a3005b003a00fc0720000c007800ba
:10c4900032e0b7004d0320009d467800f00f2000e9
:10c4a00034e0b7000005eb008b05d100e08f1500ec
:10c4b00049003100183b88000c00780064e7b700a1
:10c4c00040042400003b88002104200091407800b3
:10c4d0008180fb00c508de0001007800d4f7b700ba
:10c4e00000ceb3004260b70050c5b30066e7b700a6
:10c4f000a0cab30066e7b70061e7a800c508dd0081
:10c5000042c0bf007f4060000140700042e0b700c1
:10c510006007e200feff350019017800020cbb0045
:10c5200040002400003b8800210420009140780056
:10c530008180fb00c508de0001007800d4f7b70059
:10c5400000ceb3004260b70050c5b30066e7b70045
:10c55000a0cab30066e7b70061e7a800c508dd0020
:10c5600042c0bf007f4060000140700042e0b70061
:10c570006007e200feff350018007800820f5000cf
:10c5800010003200821f7800801f7800881f78001a
:10c5900090fa2b00801f780050172000230207001c
:10c5a000180378006505200054172000630420005c
:10c5b00022002c002119200000012c00e8010700b6
:10c5c000e88757000884e8008984e8000a05e80045
:10c5d0008b0f5500b7ff39000d00780034e0b7002d
:10c5e0004f06be004f05be004f04be000080fa009b
:10c5f000000006008b1f780080012c00801f78004f
:10c6000080052000090207000b0378006505200063
:10c61000840520006304200022002c00a1142000c7
:10c6200000012c00ce010700e487570096ff370079
:10c63000c0042c00801f780080052000fb0107004b
:10c640000003eb00e50420008405200063042000c3
:10c6500022002c006114200000012c00c001070002
:10c660008f87e90086ff370000072c00801f7800c5
:10c6700080052000ed0107000003eb00e504200029
:10c68000840520006304200022002c0021142000d7
:10c6900000012c00b20107008f87e90076ff370008
:10c6a0005000fa00889fbe008a9fbe008c1f780051
:10c6b00080572000801f7800c1012000811f780072
:10c6c00020032000801f7800c814f80041092c00c6
:10c6d000811f78002c020700ea875700c814e20087
:10c6e00012003a0030a68000d10d2c00e40f50005b
:10c6f00004003200210e2c00e80f5000010032002f
:10c70000710e2c00811f7800900e2c00801f780085
:10c710001d020700e48757004f0678004f05be0052
:10c720004f04be000080fa0000000600f1112c004a
:10c73000811f780040122c00801f7800c1122c004d
:10c74000811f780030132c00801f78000e02070034
:10c75000d1142c00811f7800210e2c0030a68000ff
:10c76000e80f500001003200d10d2c00811f78002d
:10c7700060152c00801f7800030207008005eb0085
:10c7800028de2000ee875700c814e200e2ff3200e6
:10c7900074054700890220008e844400cc032000e9
:10c7a0000e0646000e007800090009000018eb0094
:10c7b0000a007800090009000018eb000900780061
:10c7c000090009000018eb000c00780009000900be
:10c7d0000018eb00085990008280fb004003200005
:10c7e000808f5000ba0032004f003c000080e9000a
:10c7f000808f5000260032000000e800808f50003b
:10c8000023003200004eeb00804ceb00004deb00ab
:10c81000004feb00985890008c1f7800891f78001b
:10c820008a1f78008e1f780001007800000fb20088
:10c83000801f78000280fb00c1000700801f780085
:10c84000185890006f006000210e2c00e80f500077
:10c8500004003200d10d2c00e40f50000100320022
:10c86000710e2c00811f780011162c00811f78009a
:10c87000c5010700f08757008b05e8007c044400e1
:10c8800040a68000808f5500c6ff3900a2ff370008
:10c89000985890000180fb000058a300030032006c
:10c8a000a0022000000f7800dbff37000048a30043
:10c8b00018003a000068a3000d00320068409000a4
:10c8c0000080fb00801f7800881f78006100200036
:10c8d000811f7800f0172c00801f78000e00780070
:10c8e000d6d00700e887570008599000c9ff3700e5
:10c8f000881f780061002000811f780080182c00bc
:10c90000801f78000e007800ccd00700e687570023
:10c91000f5ff3700881f780061002000811f780034
:10c92000e0182c00f6ff370060032000808f5000d5
:10c9300045003200280035000000e800808f5000dc
:10c94000b0ff3a001800be004ddd0700809fbe001a
:10c95000829fbe0050192c00801f78000e007800c6
:10c96000b6d0070038009000c800900044dd0700f2
:10c97000809fbe00829fbe00311a2c00811f78006c
:10c980000a007800add0070068009000f800900021
:10c990003bdd0700809fbe00829fbe00101b2c0065
:10c9a000801f780009007800a4d0070018089000c4
:10c9b000a808900032dd0700809fbe00829fbe0065
:10c9c000d11b2c00811f78000c0078009bd0070041
:10c9d0008f02b100c4ff37001880fb000000d000b8
:10c9e000c1ea2b00e09f7800901c2c00801f78008b
:10c9f0000e00780091d0070038009000c800900029
:10ca00001fdd0700809fbe00829fbe00311d2c00ed
:10ca1000811f78000a00780088d007006800900025
:10ca2000f800900016dd0700809fbe00829fbe00c8
:10ca3000201e2c00801f7800090078007fd007009e
:10ca4000f8875700a8ff37001800be000cdd07006c
:10ca5000809fbe00829fbe00011f2c00811f7800b6
:10ca60000e00780075d0070038009000c8009000d4
:10ca700003dd0700809fbe00829fbe0000202c00c7
:10ca8000801f78000a0078006cd0070068009000d2
:10ca9000f8009000fadc0700809fbe00829fbe0075
:10caa00001212c00811f78000900780063d0070065
:10cab00018089000a8089000f1dc0700809fbe00d5
:10cac000829fbe0000222c00801f7800beff37002e
:10cad0001800be00eadc0700809fbe00829fbe00f7
:10cae000f1222c00811f78000e00780053d007003f
:10caf00038009000c8009000e1dc0700809fbe0075
:10cb0000829fbe00301d2c00801f78000a00780034
:10cb10004ad0070068009000f8009000d8dc0700b9
:10cb2000809fbe00829fbe00211e2c00811f7800c6
:10cb30000900780041d00700fe8757006aff3700e0
:10cb40000000fa00800178000082eb000001eb0099
:10cb50006410b80085e62b0005004000908f51005e
:10cb60000b0032000201e800ea0f5100f8ff360026
:10cb7000207e2100e10f4200030032006420b80053
:10cb800062e62b00600079000080fa0000000600d9
:10cb900002027800f6ff37000000fa00410320008f
:10cba00091407800f00f200034e0b70022de200032
:10cbb00000002f0077050900305978000100780047
:10cbc00034e0b7000080fa00000006000000fa0020
:10cbd000881f78004803200018447800f30f2000d5
:10cbe0008001fd0034e0b7008001fd0090cf070018
:10cbf0000800780034e0b7004f0478000080fa00a5
:10cc0000000006000400fa00889fbe008a9fbe0054
:10cc100081057800a2002000110009000280d800e0
:10cc200021479800110009000280d80011479800a0
:10cc3000110009000280d800014f7800d4a2a8009a
:10cc4000a00f200001002000890f0700d4a2a90036
:10cc5000a00f200001002000850f0700d4a2a8002b
:10cc6000a00f200001002000810f0700d4a2a9001e
:10cc7000a00f2000010020007d0f0700d4a2a80013
:10cc8000a00f200001002000790f0700d4a2a90006
:10cc9000a00f200001002000750f0700d4a2a800fb
:10cca000a00f200001002000710f0700d4a2a900ee
:10ccb000c05d2000010020006d0f07000005eb00a3
:10ccc0008e044500194078000004e0001e00320088
:10ccd0000004eb000c003200d4a2a800401f20008a
:10cce00001002000620f0700d4a2a900401f20000d
:10ccf000010020005e0f07000804e8001980fb0017
:10cd0000800f5400f4ff3500c05d200001002000ba
:10cd1000570f07000a05e800e20f5500e8ff34004e
:10cd20000b00e00004003200c05d20000100200084
:10cd30004f0f0700c1ff37004f05be004f04be0074
:10cd40000080fa0000000600d4a2a800007d2000a8
:10cd500001002000460f0700d4a2a900eaff370017
:10cd60000200fa00889fbe008a9fbe008c9fbe0012
:10cd7000000f7800810678000206780083057800ad
:10cd8000840478000505780006047800010220007c
:10cd900010002000c7ef07000000e0001200320082
:10cda000ba14e20010003200e17c210091407800ca
:10cdb00040c4b30080cf50000b003200881f7800c1
:10cdc0008a1f7800891f78008b1f78008c1f7800dd
:10cdd0008d1f78009e1f7800c0232c00801f7800d4
:10cde00069000700f0875700e1a58000090078007e
:10cdf00084ff07000000fe004f06be004f05be0086
:10ce00004f04be000080fa00000006000000fa0097
:10ce1000d422ef00f0f02f0090168800d4a2a900d1
:10ce2000d4e2a9000080fa00000006000000fa0029
:10ce3000881f780000047800ba14e2000a0032006b
:10ce4000e17c21009140780040c4b30080cf5000c5
:10ce500005003200010220001000200095ef0700bd
:10ce60000000e0000a003a00301f2000800f54004c
:10ce7000030036004f0478000080fa00000006002e
:10ce80008000eb00080078005eff0700f9ff370024
:10ce90004eb897000000e0002d003200823e2000d6
:10cea000110009000284d800301f2000808f50003c
:10ceb00021003600a235210000272c0005000900c2
:10cec0003059780058002000a235210002024400a9
:10ced0006108b8008001eb00320020007be607000b
:10cee00063044400a135210001004400a1c3b30044
:10cef00001587800fac05000015878000048eb0053
:10cf00000884e800c112200088805000a23521006a
:10cf100002004400e80157004eb9970069cf0700ae
:10cf20000004440008017800a13521001000200011
:10cf300075eb0700cfff3700a235210060272c00da
:10cf4000060009003059780068002000deff370035
:10cf5000d1272c00811f7800c0122000b3ff0700ea
:10cf600008037800e5042000c41220000305200017
:10cf700082292c0051042000e0292c0078ff0700b2
:10cf80008f87e900c5ff37000000fa00ba14e200fd
:10cf900017003200e17c21009140780040c4b300ca
:10cfa00080cf50001200320001022000100020004b
:10cfb00040ef07000000e0000d0032004eb897007f
:10cfc0000000e0000c003200c0122000e801570011
:10cfd0004eb9970080007800a035210039cf0700b6
:10cfe00000017800a13521001000200046eb070069
:10cff0000080fa0000000600602a2c00801f7800e4
:10d00000d012200089ff07000003eb00e504200098
:10d01000d412200003052000222c2c00e107200060
:10d02000e0292c004eff07008f87e900e6ff37005c
:10d030000c00fa00889fbe008a9fbe008c1f7800fb
:10d04000000478000000e000880032000081eb005e
:10d050006602440063002000c810dd003480fb003d
:10d06000808070004810de000000d00002ef280031
:10d0700002004000108168008301e900e18f410057
:10d08000f5ff3a006e02440063002000c810dd0086
:10d090003480fb00808070004810de000000d0006b
:10d0a00006ef280006004000108168008301e900b7
:10d0b000e18f4100f5ff3a008201780078024400d8
:10d0c000380990000201e900e10f41000b00320035
:10d0d000c818dd003480fb00808070004818de0036
:10d0e0000000d00003ef280003004000908168009a
:10d0f0000201e900e10f4100f5ff3a0058489000b5
:10d100000000d1006f4f60000040eb001047980016
:10d1100020479800030578008e0178002200200047
:10d12000c850dd003380fb00808070004850de0076
:10d130000000d00004ef28000400400010856800c3
:10d140000201e900e10f4100f5ff3a000206780014
:10d150000b8020008000eb00520920002b00900083
:10d16000800f55003f0032008100e800e685450051
:10d17000828f5000f9ff360088f1070020079800e1
:10d18000310798004207980053079800f8bd8000c7
:10d1900009be80000800be0002dc0700e00f54005a
:10d1a000e08f5c002a0035000002be000203be00d2
:10d1b0002e009000be0090004e019000de01900015
:10d1c000fbdb070054dc07000002be00e10f460055
:10d1d000100032001b01be00a0a58000000041002d
:10d1e000e080490012002000840f5000858f580015
:10d1f00002003e00848dbe000001eb0002007800ba
:10d200004f0678004f05be004f04be000080fa00b4
:10d2100000000600e36e80006618b800468020001b
:10d22000060140000a097800028020000200400048
:10d230000488be008301e800e36e880050092000e6
:10d24000808f5100ecff3400dc2def00eaff370047
:10d250006022b80006002000071f240054dc0700ed
:10d26000d1ff370001067800c3ff3700a02c2c0047
:10d27000801f780050192000ecfe07000003eb002f
:10d28000e50420005419200043042000122f2c0034
:10d29000a1032000c02f2c00b1fe07008f87e900fa
:10d2a0006aff37000800fa00889fbe008a9fbe0010
:10d2b000000578000000e000020032001004e000e9
:10d2c0000d003a0040302c00801f780050192000db
:10d2d000d6fe07000003eb00e504200054192000ef
:10d2e0004304200012342c00210b2000c02f2c00fe
:10d2f0009bfe07008f87e9008085eb000004eb00b0
:10d30000190320006c40b80082b8200002004000e1
:10d31000820020008a00780021ce07000000e00093
:10d32000400032000804e800890f5400f5ff340083
:10d330001af10700009fbe000297be00f8bd8000f2
:10d3400009be80000800be0096db0700e00f540015
:10d35000e08f5c002e0035000002be000203be001c
:10d360003e00be002e01be0091db0700eadb070095
:10d370000004be00e18f4500120032006c58b80076
:10d3800044b8200084014000a400200005002000d3
:10d3900033004200a3804a0012002000880f500092
:10d3a000898f580002003e008889be000001eb0012
:10d3b000020078004f05be004f04be000080fa0056
:10d3c00000000600f06e80006c00b80085b82000f8
:10d3d00005004000820020008a0078002acd070066
:10d3e000f26e80006c10b80043b8200003004000cb
:10d3f0000888be000201e800f26e880010032000d9
:10d40000800f5100e9ff3400de2def00e7ff370009
:10d410006022b80006002000071f2400e4db07009c
:10d42000cdff370088057800c1ff37000000fa0003
:10d430000002be000201e900e10f41000a003200d3
:10d44000c820dd003580fb00808070004820de00b1
:10d450000000d00060807900008268000201e900cd
:10d46000e10f4100f6ff3a00040078000080fa0066
:10d47000000006000000fa00f30f20004200200028
:10d4800081572f00604821002b0e0700f30f20006a
:10d4900042002000c1572f00a0482100260e07009f
:10d4a000f30f20004200200001582f00e048210027
:10d4b000210e0700f30f20004200200041582f00ea
:10d4c000204921001c0e0700f30f2000420020001d
:10d4d00081582f0060492100170e0700f30f20002c
:10d4e00042002000c1582f00a0492100120e070061
:10d4f000f30f20008200200001592f00e049210095
:10d500000d0e0700f30f20002200200081592f008c
:10d51000604a2100080e0700f30f200022002000bf
:10d52000415b2f00204c2100030e0700f30f200069
:10d5300022002000215a2f00004b2100fe0d070081
:10d54000f30f200022002000415a2f00204b210021
:10d55000f90d0700f30f200022002000615a2f0070
:10d56000404b2100f40d0700f30f200022002000a3
:10d57000815a2f00604b2100ef0d0700f30f2000b0
:10d5800022002000a15a2f00804b2100ea0d070045
:10d59000f30f200022002000c15a2f00a04b2100d1
:10d5a000e50d0700f30f200022002000e15a2f00b4
:10d5b000c04b2100e00d0700f30f200022002000e7
:10d5c000015b2f00e04b2100db0d0700f30f200073
:10d5d00022002000215b2f00004c2100d60d070007
:10d5e000f30f200022002000615b2f00404c21003f
:10d5f000d10d0700f30f200022002000815b2f00d7
:10d60000604c2100cc0d070031a6800000052000f1
:10d61000808f5000260032000600360040062000b1
:10d62000808f5000030032006c004000808f50005b
:10d630001f0032004000200030a68800f30f2000b9
:10d6400022002000a15b2f00804c2100ba0d0700b2
:10d65000f30f200002042000e15b2f00c04c2100ea
:10d66000b50d07000001eb006810b800c34c2100a5
:10d67000030040001004e000030032000201e80053
:10d68000e70f5100f8ff34000200780038f5b700ca
:10d69000ae75ef00f30f2000c2022000e15f2f0003
:10d6a000c0502100a40d07000080fa000000060011
:10d6b00080002000e0ff37000000fa00881f78009b
:10d6c000e17c21009140780070c4b30080cf50000d
:10d6d0000a003200e17c2100914078006340500054
:10d6e00080cf500005003200010220001000200011
:10d6f00070ed07000000e00003003a004f047800de
:10d700000080fa0000000600c0a5800080007800bc
:10d71000f107b200811f78004800de00801f78000a
:10d72000b614f800c414f800b414f80070a4800013
:10d7300081a48000809fbe0050a4800061a480006e
:10d74000809fbe0030a4800041a48000809fbe0066
:10d7500090a48000a1a48000809fbe00d0a480007f
:10d76000e1a48000c6d90700809fbe00829fbe0052
:10d77000b0a48000c1a48000c1d90700809fbe0072
:10d78000829fbe00a614f800e1492100811f7800a5
:10d7900062002000821f7800200b2000801f78008c
:10d7a00021402d00811f780022352c00821f780037
:10d7b000f5fd07006f03b100b014e200580032001d
:10d7c00080422c00801f7800c1502100811f78000a
:10d7d000b2422c00821f7800ebfd070038d5bf0055
:10d7e000c1442c0001003a00d1442c00811f780074
:10d7f0000080fb00801f780040452c00801f7800cf
:10d80000e1fd07000004eb00ec87570038d5bf00ae
:10d810000080fb00e00f100014003d000000e90054
:10d82000c1442c00800f54000100320071462c00ce
:10d83000811f78006840b800c24c2100821f400060
:10d8400080002000801f780091462c00811f780006
:10d85000cdfd0700e88757000804e80038d5bf0071
:10d860000080fb00800f5400ecff350030a68000e4
:10d8700001472c00e40f50000400320051472c00f7
:10d88000e80f500001003200a1472c00811f7800f2
:10d89000c814f800be14e2001f003200c0472c007c
:10d8a000801f7800bc14e20019003200c0472c0031
:10d8b000801f7800c214e20013003200c0472c0021
:10d8c000801f7800c014e2000d003200c0472c0019
:10d8d000801f7800ba14e20007003200c0472c0015
:10d8e000801f780002482c00821f7800a6fd0700e8
:10d8f000f087570081ff370060512c00f8ff370098
:10d9000060512c00f2ff370060512c00ecff370013
:10d9100060512c00e6ff370060512c00e0ff37001b
:10d9200090512c00a7ff37000000fa00889fbe002e
:10d930008a9fbe008c1f780051012000a0d22100d8
:10d940009100070000057800f50f50000800320034
:10d950000003780065052000c41a2000730520002c
:10d9600002522c007103200090522c00fcfc070096
:10d970005100200080d321005fe307000004be00b7
:10d9800000067800cbd221004200200041532c0039
:10d990000b007800dccc07000000e0003100320012
:10d9a0005200200091532c000b007800d6cc0700c9
:10d9b0000000e00017003a000800e00002003a0012
:10d9c000e02def00dcff37008800780020de20002b
:10d9d00030000700880f5000080032000003780074
:10d9e00065052000d41a20007305200002522c0087
:10d9f000b104200090522c00d9fc0700c201200085
:10da0000110009000286d80000017800026f88002a
:10da1000c9ff3700a2002000f1532c000b00780052
:10da2000b9cc07000000e000090032000a037800ca
:10da300065052000e41a20007305200002522c0026
:10da40008300780090522c00c5fc0700baff370015
:10da50004f0678004f05be004f04be000080fa005c
:10da600000000600880078006048210009000700d7
:10da7000880f5000b0ff32000003780065052000d9
:10da8000c41a20007305200002522c00110420004b
:10da9000ecff37000000fa00889fbe008a9fbe009e
:10daa00000057800010478000000e0002d0032003d
:10dab0000800e00022003200880478008005eb00b6
:10dac0000800e0001000340001102000a0d2210066
:10dad0002d00070000047800e40f50000f00340010
:10dae0006404540008017800c1d221000a007800c3
:10daf000cfcb070008054500888545008884540081
:10db00004240a900f0ff3c000b0078004f05be002a
:10db10004f04be000080fa000000060000037800f9
:10db200065052000d41a200073052000a2542c00a3
:10db30003108200090522c0089fc0700e8ff3700d4
:10db40000003eb0065052000c41a200073052000c7
:10db5000a2542c002107200090522c0080fc0700ca
:10db6000d5ff37000003eb00e5042000c41a2000b5
:10db700073052000a2542c00d106200090522c00e6
:10db800077fc0700caff37000800fa00889fbe0034
:10db90008a9fbe008c9fbe000005be000000e00012
:10dba00075003200e48f55006a0036005c002000ea
:10dbb000615bb80004d420000430b8006331b900c0
:10dbc0000281400004bab9008400410032a4800000
:10dbd00043a4800078da07002007980031079800f6
:10dbe000e90f5000e08f580004003c00a000200026
:10dbf000010020002007980031079800800c2000c9
:10dc000001002000008fbe008a86e8002800200066
:10dc10008e017800080178008a007800100020004a
:10dc200073e70700880f50000800320000037800f7
:10dc300065052000e41a20007305200082552c00a1
:10dc4000610c200090522c0045fc07009a80fb00dc
:10dc5000c808dd001a4090000080fb00808470003e
:10dc60008b8f540032003e000984e900e401470034
:10dc7000080178008d007800100020005ce70700a4
:10dc8000880f50000800320000037800650520006e
:10dc9000041b20007305200082552c00210d20005c
:10dca00090522c002efc07000080eb0003ef2800b0
:10dcb000090178008a007800dcfd07000000e00020
:10dcc000150032000c06e90012002000f1512c0072
:10dcd000020078000ce807000c00e000cbff3c00dd
:10dce0000003eb0065052000f41a200073052000f6
:10dcf00082552c00d10e200090522c0018fc0700f9
:10dd00000000eb004f06be004f05be004f04be00f2
:10dd10000080fa000000060012002000e1512c00f3
:10dd200002007800f8e7070009007800f5ff3700e7
:10dd30000903780065052000f41a2000730520000f
:10dd400082552c00b10c200090522c0004fc0700de
:10dd5000c5ff37000003eb0065052000d41a200042
:10dd60007305200082552c00e10a200090522c00ff
:10dd7000fbfb07008dff37000003eb00e5042000ec
:10dd8000c41a20007305200082552c00810a20004f
:10dd900090522c00f2fb070082ff37000000fa00cf
:10dda000889fbe008a9fbe008c9fbe000004780042
:10ddb00001057800820678000000e000b70132001b
:10ddc000e90f5500a60134000d00e0009601320075
:10ddd000630644001c41780070c4b300804f5100ba
:10dde000d700320020c5b300804f510004003a0034
:10ddf0009c4090006540500080cf50000b003200e6
:10de00000040eb00c05e980000c0eb00b05e9800e0
:10de1000d1ff2f00010078004f06be004f05be0065
:10de20004f04be000080fa0000000600ac409000e5
:10de30006a40500080cf5000f1ff3a008a00e900ac
:10de40000800e800a30107008080eb000000e0006c
:10de5000f0ff3500c10220000c00780069cb0700fc
:10de60000006e8001c80fb006a00b9001c4190001d
:10de70000041410070415100825e98002c409000aa
:10de80000080fb006a00b9003c4190000041410065
:10de900070415100925e98004c4090000080fb0061
:10dea0006a00b9005c41900000414100704151009e
:10deb000a25e9800c10220000c00780051cb070040
:10dec0000006e8009c40780010c4b30080cf5000ea
:10ded0009900320060c5b30080cf5000940032003a
:10dee0000040eb00b05e9800c10220000c007800fa
:10def00044cb0700000478000006e8001c81fb000a
:10df00006a11b9001c4090000080fb000200400034
:10df10000021b100cf80de00f8d707000005be0069
:10df2000630444006011b8008000eb000800780032
:10df300094c907001cd807000004be00c1022000dd
:10df40000c0078002fcb07000006e800928828001c
:10df500083c823000800be0037d707000001be00b9
:10df60000a00be0069d707000001be00808ebe0017
:10df700030c5b3009c4f100069003200c102200080
:10df80000c0078001fcb0700000478000006e800b2
:10df90001c81fb00400620000091b9001c4090004d
:10dfa0000080fb006a00b900000141002c40900095
:10dfb0000080fb000001410000b32e000001410081
:10dfc0006110b900cdd707000005be00640444000d
:10dfd0006011b8008000eb000800780069c90700f4
:10dfe000f1d707000004be00c10220000c00780039
:10dff00004cb07000006e8009288280083c82300ad
:10e000000800be000cd707000001be000a00be00d9
:10e010003ed707000001be00a0069800b106980098
:10e0200070c5b3009c4f100038003200c1022000c0
:10e030000c007800f3ca07000006e8006011b80081
:10e040008000eb000c0078004ec90700d6d707000f
:10e05000e0069800f1069800c10220000c0078004c
:10e06000e8ca07000006e8006011b8008000eb0075
:10e070000c00780043c90700cbd70700800e98003a
:10e08000910e9800c10220000c007800ddca070044
:10e090000006e8001c80fb006a00b9001c419000eb
:10e0a0000041410070415100f25698002c40900010
:10e0b0000080fb006a00b9003c4190000041410033
:10e0c00070415100e25698004c4190000281fb00e3
:10e0d0006a11b9005c4090000080fb000200400023
:10e0e000015c200001004000a00e9800000020000c
:10e0f00001082000c0069800d106980030c0b30087
:10e10000c05e98008000eb0042ff37000200be00b6
:10e1100001f0a200a0069800b1069800c3ff3700e6
:10e120000200be0001f0a200808ebe0093ff370007
:10e1300000c0eb006bff370010c0b30069ff370071
:10e140001c409000824f500026ff3a00ac409000e7
:10e1500010c4b30080cf500022ff3a008a00e900cb
:10e160000800e800db0007008080eb000000e00012
:10e1700028ff3500c10220000c007800a1ca07006a
:10e180000006e8001c80fb006a00b9001c419000fa
:10e190000041410070415100825e98002c40900087
:10e1a0000080fb006a00b9003c4190000041410042
:10e1b00070415100925e98004c4090000080fb003e
:10e1c0006a00b9005c41900000414100704151007b
:10e1d000a25e9800c10220000c00780089ca0700e6
:10e1e000000478000006e8001c81fb006a11b900f9
:10e1f0001c4090000080fb00020040000021b100a4
:10e20000cf80de003dd707000005be006304440058
:10e210006011b8008000eb0008007800d9c8070042
:10e2200061d707000004be00c10220000c00780086
:10e2300074ca07000006e8009288280083c82300fb
:10e240000800be007cd607000001be000a00be0028
:10e25000aed607000001be00808ebe0030c5b30000
:10e260009c4f10006c003200c10220000c007800ae
:10e2700064ca0700000478000006e8001c81fb0067
:10e28000400620000091b9001c4090000080fb0077
:10e290006a00b900000141002c4090000080fb00a2
:10e2a0000001410000b32e00000141006110b900df
:10e2b00012d707000005be00640444006011b800d6
:10e2c0008000eb0008007800aec8070036d70700d2
:10e2d0000004be00c10220000c00780049ca0700fb
:10e2e0000006e8009288280083c823000800be00ca
:10e2f00051d607000001be000a00be0083d6070009
:10e300000001be00a0069800b106980070c5b300d9
:10e310009c4f10003b003200c10220000c0078002e
:10e3200038ca07000006e8001c40780001c3b300ab
:10e33000814f50003100320001405000b05e980023
:10e34000c10220000c0078002eca07000006e80079
:10e35000c10220000c0078002aca07000006e8006d
:10e36000c10220000c00780026ca07000006e80061
:10e370006011b8008000eb000c00780081c8070035
:10e3800009d70700c0069800d1069800c1022000f6
:10e390000c0078001bca070090409000d0c4b30066
:10e3a00080cf50000d0032000040eb00f056980086
:10e3b000e05698000000eb00a00e9800000020003e
:10e3c00001082000e0069800f1069800800e9800f1
:10e3d000910e980010c0b30049ff37004d00900027
:10e3e000dd00900052b82e001305240012d607005d
:10e3f000c0069800d1069800ebff370000c0eb0084
:10e40000ceff37000200be0001f0a200a006980077
:10e41000b1069800c0ff37000200be0001f0a20064
:10e42000808ebe0090ff3700a0562c00801f780021
:10e43000e00420007dfa07000003eb00e504200063
:10e44000050278008501780072592c002103200014
:10e45000305a2c0042fa07008f87e9005cfe370033
:10e460008a1f7800a15a2c00811f7800f004200038
:10e470006efa07000a03780065052000f404200006
:10e48000e304200072592c00e1022000305a2c00d5
:10e4900033fa0700e48757004bfe3700505d2c002d
:10e4a000801f7800d004200060fa07000003eb0012
:10e4b000e5042000d40420008501780072592c0066
:10e4c000a1022000305a2c0025fa07008f87e900ae
:10e4d0003bfe37000000fa00889fbe000004be002b
:10e4e0000000e00045003200e58f540034003400a5
:10e4f000090044008000e900888f50002e00390098
:10e5000011417800a0c2b300804f510006003200d4
:10e510008100e900888f5000270039001141780000
:10e52000804f5100faff3a008081eb00a0c2b30097
:10e53000804f510018003a000041eb0008007800bd
:10e54000810f54000300310030416900810f5000f9
:10e55000fdff39000280fb00c401de00e9cf51005d
:10e5600013003e000343b0006f416100e94f5100ca
:10e570000d003e000243b0001140900080cf5100da
:10e5800004003a002140900088815000804f5100e3
:10e5900001003200e3ff2f00030078004f04be00ab
:10e5a0000080fa00000006007243b000f2ff37005e
:10e5b0007343b000ecff370011417800daff3700f9
:10e5c000891f780020602c00801f7800d032200046
:10e5d00016fa07000003eb00e504200034022000d7
:10e5e0007304200072632c0041122000305a2c006a
:10e5f000dbf90700e4875700bdff3700c0642c003b
:10e60000801f78003002200008fa07000003eb00aa
:10e61000e5042000340220007304200072632c0003
:10e62000f1112000305a2c00cdf907008f87e90046
:10e63000adff3700c401fa00889fbe008a9fbe006c
:10e640008c9fbe008e0678000e007800be00090088
:10e650000018eb00abd22100802520000100200033
:10e66000309799004197990071b9800008102000f7
:10e6700001005400e10f500074023400d1c0b30017
:10e680001000200005ea070071b980000101540064
:10e69000a3d2210083804000631a20008e814100b4
:10e6a0001000200019e40700000478000000e000da
:10e6b00010003c000800e0000b003500246e2c0028
:10e6c000841f780000322000d8f907000000eb001a
:10e6d0008f87e9004f06be004f05be004f04be0005
:10e6e0000080fa00000006002e37b5000080eb0025
:10e6f000f8ff37002e37b40028ec0700609f990020
:10e70000719f990002a7990013a7990084702100b6
:10e71000009abe000292be00b8bc8000c9bc800056
:10e720000800be009fd60700e00f5400e08f5c0099
:10e73000410235000002be000203be006e98910047
:10e74000fe9891000ea191009ea1910098d607001d
:10e75000acd7070080b9880091b9880070b98000f3
:10e7600091d22100010440008b1f780002702c0020
:10e77000821f780004fa07000005eb000b00780008
:10e78000e4875700888f550006003e0041c2b30061
:10e7900090cf1000260232000000e800880f5000e1
:10e7a000fbff36002e37ef000a00e0001a023200ad
:10e7b0000a0054000006e80078824600049f990091
:10e7c00052002000d1702c000a0078004ec90700ca
:10e7d0000000e000ba0132003200200031712c004c
:10e7e0000a00780048c9070071712c000000e000a1
:10e7f000aa013a00c21520000d0141008c007800ea
:10e800000a00780065fd0700000478000000e000c1
:10e810000600320014732c00841f7800f0322000b0
:10e8200082f907000880e900a9ff37005df892002f
:10e830003040b300d0fe9a00631a20008e81410060
:10e8400002102000a1d2210010002000afe3070039
:10e850000000e00004003c00a3ff3500206e2c0007
:10e86000801f780097ff370070b9880071d22100af
:10e87000010440000000eb0010449800aad22100df
:10e880008a1f780022762c00821f7800bef90700cc
:10e8900052002000d1702c000a0078001ac907002d
:10e8a000e48757000000e000d7013200320020006a
:10e8b00031712c000a00780013c907000000e00045
:10e8c00022003a000a0054000006e800e217200087
:10e8d0000e0141008c0078000a0078002ffd07002f
:10e8e0000000e000c2013a002e589300e14f5000b2
:10e8f000b8013200e34f5000a70132002e37ef007d
:10e90000631a20008e81410002102000a1d2210054
:10e91000100020007de30700000478000000e00004
:10e9200064ff340070b9880052002000d1702c00c0
:10e93000a0d22100f4c807000000e0005a01320014
:10e9400040c2b3009b4f100052013200a0d2210000
:10e95000f2c7070000017800a1d2210010002000ba
:10e96000e9e40700c014e200030032007df09200e9
:10e97000e14f40004401320071b98000a0d2210073
:10e98000d4fe0700509f99000000e00038013500d8
:10e990002e37ef000000eb00804d9800a0d2210040
:10e9a00040fa07000000e00027013a000d0078005f
:10e9b000ba0707000000e0001e013a00a0d22100c3
:10e9c000ca1920000e0545006011b80005c2b30049
:10e9d000d6c2b3000200e0000f013a009040780078
:10e9e000d4c2b30084cf50000801320085cf50005c
:10e9f0000401320085cf500005003200e58f510040
:10ea00000200340012002000065d7800105d7800de
:10ea10008301e8000000e800e78f510002003c009d
:10ea2000e20f5100ebff3400e10f5100f20034001f
:10ea3000004deb00ab4890001b489000e6f4070047
:10ea4000000178000000e000e0003500f002200046
:10ea5000109f9900229f99006d299100fd29910036
:10ea600062979900739799000200be00cad7070009
:10ea7000000678000000e000c3003500e404200038
:10ea8000349f9900cf80de001cd507000001be0036
:10ea90006e909100fe9091009bd40700f8d407007f
:10eaa0006022b80006002000e704240003d7070016
:10eab0003dd5070060979900719799000d3491003a
:10eac0009d3491000800be00b3d707008005780090
:10ead0000000e0009d00350051042000419f990096
:10eae0006158b90005d507000001be000800be004e
:10eaf00085d40700e2d407006022b8000600200099
:10eb0000e7042400edd6070027d507000004be0067
:10eb10006d309100fd3091009fd70700000578000f
:10eb2000509799000000e00002003a008a16200089
:10eb30005a9799002d309100bd30910096d707006b
:10eb4000809fbe0072d32100821f7800de99910061
:10eb5000ed9f51004d309100dd3091008ed70700c0
:10eb6000801f78008a1f78002e9a9100841f7800f9
:10eb70004e989100801f78000800be00c0d40700a6
:10eb8000809fbe00829fbe008b1f78009e989100e0
:10eb9000811f78003e999100821f78006e9091004d
:10eba000fe909100b6d40700809fbe00829fbe00f9
:10ebb0008c1f7800c31920008e9f410064762c00c2
:10ebc000841f78000e9891001cc80700b00e9800b2
:10ebd000cf02b100a11a20008e8040000e00780004
:10ebe0009ef4070000047800e40f50004500320056
:10ebf00011003c00e20f500005003e00c17a2c00dd
:10ec00000e007800400407000000eb00b1fe370062
:10ec1000881f7800f17c2c00811f7800daf807004b
:10ec2000d1802c000e007800c90407000080eb00a2
:10ec3000e4875700a7fe3700e80f5000f4ff3a00c2
:10ec40000e007800faf80700e10f500029003200aa
:10ec50005e909100e10f400021003200801fe8002b
:10ec60007c00b800c2df2000e01f790013832c0075
:10ec7000831f7800c4f80700e6875700b1842c0092
:10ec80000e0078002004070002102000a1c221001d
:10ec90000e007800f5000700800478000000e00016
:10eca0000b00320000017800a1c2210020002000ea
:10ecb000b6020700890f5000d3ff3200801f780092
:10ecc000c0842c00801f7800aff80700d7ff370002
:10ecd000801feb0024862c00841f7800faff370089
:10ece00010892c00801f7800a7f807008f87e900a3
:10ecf000e2ff3700818a2c000e0078000204070032
:10ed00007afe37005e909100e10f40000a00320069
:10ed1000801fe8007c00b800c3df2000e09f79007e
:10ed2000b48b2c00841f780097f80700e687570003
:10ed3000b1842c00f0ff3700528d2c00821f780028
:10ed400091f807008f87e900f9ff37007005200070
:10ed5000409f99006158b90068d407000801be00bf
:10ed6000e9d3070046d407006022b800060020005f
:10ed7000e704240051d607008bd407000004be002e
:10ed80008b05ea0062ff370033052000339f9900ae
:10ed9000cf80de0059d407006e919100fe91910062
:10eda000d9d3070036d407006022b800060020003f
:10edb000e704240041d607007bd407006097990040
:10edc000719799000c06ea003cff3700bb489000a1
:10edd0008181fb00139f990000c2b30080cf5000d7
:10ede000020032000201ea001aff3700c4052000c9
:10edf000149f9900fbff37000040eb0070fd9f005f
:10ee00000cff3700e28f5100fafe340012002000a0
:10ee1000045d7800fefe37009040780086cf5000f9
:10ee2000fbfe320085cf5000f9fe32000201e800ff
:10ee3000f6fe3700d2022000c18e2c001000200008
:10ee4000b1e3070029fe3700a4d22100841f780017
:10ee5000a0002000801f7800a1912c00811f780065
:10ee600049f807000080eb00e687570019fe3700dd
:10ee7000d3932c00831f780043f807002e37ef0050
:10ee80000080eb0012fe370032962c00821f7800c3
:10ee9000f9ff37002e37ef00e1972c00811f780033
:10eea000e032200008fe37002e37ef00509a2c0089
:10eeb000801f7800e0322000dcf707008f87e90030
:10eec00065004500020120008000eb00ebc6070052
:10eed0000004be000080eb006a015600ea04450011
:10eee0008900780028050700800f540025003a00ab
:10eef000a1d221000900780007000900b05878006d
:10ef000082002000e1032000a0d221008dc707006d
:10ef10000000e000190032000048eb00a0d2210000
:10ef2000e0f807000000e0000d003a000d00780056
:10ef30005a0607000000e000beff3a00d0c7b30049
:10ef4000104d980069045600e9004500080178005a
:10ef50000e989100b6c60700b80e98001dff370046
:10ef6000a1d22100811f7800a2002000821f78001a
:10ef7000a3912c00831f7800b9ff3700804d9800c3
:10ef8000e6ff3700e09c2c00801f7800f032200064
:10ef9000a6f70700baff37007e8191008e899100a5
:10efa000e2369900f33699005e809100ee80910080
:10efb000c0369900d13699009e889100813e990013
:10efc0004e519300a2f69a00de519300b3f69a00d8
:10efd0004afe37003e809100ce809100a036990015
:10efe000b13699009e589300f1f69a0043fe37001f
:10eff00014732c00841f7800f03220008bf7070078
:10f000008f87e9003dfe370013a02c00831f780096
:10f01000f0322000a8ff3700c3a22c00831f780025
:10f02000e032200081f70700e0ff2f00a8fd370045
:10f0300000057800dbfd37006022b80006002000e4
:10f04000071f2400dad40700bafd3700811f7800bb
:10f05000b0a62c00801f78004033200073f7070013
:10f060002e37ef00e487570084fd37001401fa00c3
:10f07000889fbe008a9fbe008004780081057800ca
:10f08000020578000000e000bb0032000b00e00049
:10f09000ab00320010032000800f550099003600ad
:10f0a0000e0378000004eb008000eb000001eb0091
:10f0b00003c4b30002804400604890000004e000f4
:10f0c00001003a00110020000100e0008b00320036
:10f0d000034b78000201e8000603e8000804e8009a
:10f0e000e50f5100f3ff340059509000005b7800a9
:10f0f0000804e8008000eb000001eb0003c4b3004b
:10f1000002804400604090000004e00001003a00ea
:10f11000110020000100e00076003200034b78006f
:10f120000201e8000603e8000804e800e50f5100ca
:10f13000f3ff340059489000004b7800a9d89200a2
:10f140000104e00002003a001604a000a9d89200d1
:10f150000603e8000804e8008003eb000104e00077
:10f16000200032008000eb000001eb00683ab8009c
:10f1700003c4b3000400410009004000205892007d
:10f180000004e00001003a00110020000100e0004e
:10f1900056003200034b78000201e8000603e80045
:10f1a0000804e800e50f5100f2ff34000480440039
:10f1b00010609200004b7800a9d892000180fb00fb
:10f1c0000000e900808f5300450032008703e8000b
:10f1d0000603e8000804e8000180fb00808f53006c
:10f1e000e0ff350030c0b300005b780000cfb30013
:10f1f000005b78000884e8003909900002004400b0
:10f200000080e8008a0f50002c003100f880440094
:10f210000600780006c60700390890000004440084
:10f220000b03780001ccb300015b7800005beb00be
:10f230000000eb000001eb00e00f14000e003d00a9
:10f2400001427800fbc04000c5cdb300d7cdb3006c
:10f25000e2417f0084cf51001400320081cf510081
:10f260000e003200034b78000201e8000603e800bc
:10f27000880f5100f6ff35008000440000ccb30039
:10f28000005b7800004beb00638040004f05be0040
:10f290004f04be000080fa0000000600034b780017
:10f2a0000000e800076b7800efff3700014b7800a3
:10f2b0000000e800056b7800ebff3700801f780046
:10f2c0008a1f780010aa2c00801f780030052000cb
:10f2d000d6f607000080eb00e6875700ebff37000b
:10f2e0001604a000a9d89200b8ff3700004bd00048
:10f2f000a9ff3700004bd00089ff3700004bd0003a
:10f3000074ff37008a1f780030ae2c00801f780011
:10f31000f0042000c5f607000a0378006505200008
:10f32000f40420004305200032b12c00713d200080
:10f3300030b22c008af60700e487570058ff3700e8
:10f34000b0b22c00801f7800e0042000b7f6070060
:10f350000003eb00e50420000502780043052000cf
:10f3600032b12c00313d200030b22c007cf6070079
:10f370008f87e90047ff3700c0b52c00801f780059
:10f38000d0042000a9f607000003eb00e5042000ec
:10f39000d40420004305200032b12c00f13c2000b1
:10f3a00030b22c006ef607008f87e90037ff370078
:10f3b0000200fa00889fbe008a9fbe008c9fbe009c
:10f3c00000047800010f7800020578000000e000da
:10f3d000e00032000a00e000d00032001e00780099
:10f3e0000000e000be003200220020006e06450052
:10f3f0008c0478000a007800be0009000018eb00b9
:10f400000884e8008005eb008006eb001e00780011
:10f410000000e0001e003200e30f510095003200b2
:10f4200049003c00e10f510037003200e20f51006b
:10f430002d003a008b05e800e68f550020003400cf
:10f44000804ceb0098407800714698008005eb00f6
:10f45000660645008c0478007c4090000000d100d6
:10f460006f00600011003a00120020008d06e800d5
:10f470000804e8009e007800818f560004003100e7
:10f48000e70f510002003200e80f5100e2ff3a009e
:10f490004af892000080fb004f06be004f05be00f8
:10f4a0004f04be000080fa0000000600d0b82c0017
:10f4b000801f7800b4f607008f87e900eaff370065
:10f4c0009840780000c4b30080cf500004003200a0
:10f4d0000180fb000000d100805c7800e3ff370072
:10f4e000805ceb00e1ff3700821f7800c0ba2c007f
:10f4f000801f7800d00520004cf607001000200087
:10f50000e4875700e4ff37008b05e800e68f5500dd
:10f51000ebff3400804ceb00984078007146980077
:10f520008005eb001880fb00420020000008a300cb
:10f53000ceff3a00ac1120000a0646008c04780089
:10f5400032002000c9ff3700e50f510043003200b0
:10f55000e40f51002c003400e60f5100e2ff3a00a6
:10f560009841780000ccb30080cf510023003200d6
:10f570009e0078000100e900808f560015003200df
:10f58000ba089000f00f2000808f500006003e0067
:10f59000835c78003a0890000000e800300d980085
:10f5a0008b05e800b1ff3700811fe80020be2c006a
:10f5b000801f7800600620001cf60700804ceb00de
:10f5c00081c0b30041fd9a0082002000e48757000b
:10f5d000a6ff370090c22c00801f78005006200044
:10f5e00012f60700804ceb0081c0b30041fd9a0089
:10f5f000820020008f87e9009cff3700804ceb00e1
:10f600007200200099ff37001840780020fd9a0012
:10f61000720020001880fb00e10060000d00320045
:10f620000018a30009003200c00ab20004003a002a
:10f6300030c0b30040fd9a00520020008bff37001d
:10f6400020c0b30040fd9a0088ff370010c0b3000f
:10f65000fcff370041fd9a0084ff37009840780096
:10f6600031fd9a00f80445008005eb00620020009f
:10f670007eff37008b05e800e68f550090ff3400d1
:10f68000804ceb0018407800704698008005eb0035
:10f690002ad892000040e80020dd9a00e74f500091
:10f6a00008003e001880fb000008a30002003200a2
:10f6b000420020006dff3700680646008c04780089
:10f6c0006aff370081002000811f7800b0c62c003f
:10f6d000801f780090052000d4f50700b8ff3700a0
:10f6e000801feb0061cb2c00811f7800800520007b
:10f6f000cef507000003eb0065052000840520001f
:10f7000043052000e2cd2c006148200030b22c00df
:10f7100093f50700e487570033ff3700d1ce2c0064
:10f72000811f780070052000c0f507000003eb0082
:10f73000e50420007405200043052000e2cd2c00e4
:10f740002148200030b22c0085f507008f87e900a2
:10f7500022ff3700a0d12c00801f78006005200018
:10f76000b2f507000003eb00e5042000640520006b
:10f7700043052000e2cd2c00e147200030b22c00f0
:10f7800077f507008f87e90012ff37000000fa00c5
:10f79000889fbe008a1f78008004780001057800e9
:10f7a000020478000000e900e10f50002a003e004a
:10f7b0000a00e0001a0032000800e00009003200f0
:10f7c000080178008a007800090078004ee10700ff
:10f7d000080078004f0578004f04be000080fa0052
:10f7e00000000600801feb0060d42c00801f780012
:10f7f000000620008df507000003eb0065052000e2
:10f800000406200043052000a2d62c0051562000fb
:10f8100030b22c0052f50700e4875700e8ff3700ac
:10f8200050d72c00801f7800f00520007ff50700de
:10f830000003eb00e5042000f40520004305200050
:10f84000a2d62c001156200030b22c0044f507003f
:10f850008f87e900d8ff3700891f7800200020003b
:10f86000801f7800c0d92c00801f7800e0052000a0
:10f870006ef507000003eb0025052000e4052000dd
:10f8800043052000a2d62c00d155200030b22c0018
:10f8900033f50700e6875700c5ff37000200fa007e
:10f8a000889fbe008a9fbe008c9fbe0080057800a6
:10f8b00081067800020578000000e900e10f5000a1
:10f8c00078003e000d00e000680032000a00e00011
:10f8d000570032006044b80010c0b30010479800d1
:10f8e0000cccb3008a8f54004c0031008001eb0037
:10f8f000120020008e0078000b0078003ce007002a
:10f90000e10f500040003a00e10f540026003200a1
:10f910000800e00021003200e20f540017003a0016
:10f920009e407800d0cdb30080cf50001000320050
:10f93000c0cdb30080cf50000a0032001800200074
:10f940001e4090000004e000e6ff3a000900780045
:10f950004f06be004f05be004f04be000080fa00f7
:10f96000000006008cf67c008904e800f3ff3700f5
:10f9700000c0e90080f67c00fbff3700881f78009c
:10f98000d0dc2c00801f78007006200027f50700cf
:10f990000080eb00e4875700edff37009e4f160014
:10f9a000e7ff3a00efff37009e4078008ccf500011
:10f9b00008003200b0cdb30080cf50000300320009
:10f9c00081f67c008904e800ddff37002800200074
:10f9d000dbff3700e18f5400d9ff36008cf67c0046
:10f9e0008904e8000040eb00104798008a8f54001b
:10f9f000d3ff39008a1f7800c0e02c00801f7800f8
:10fa000060062000e1ff3700801f780050e42c00e2
:10fa1000801f780050062000dcff37008a1f780026
:10fa2000c0e02c00801f780040062000d7ff370080
:10fa3000801feb0080e72c00801f7800300620003c
:10fa4000faf407000003eb006505200034062000ef
:10fa500043052000c2e92c001159200030b22c00cf
:10fa6000bff40700e48757009aff370060ea2c00d4
:10fa7000801f780020062000ecf407000003eb0054
:10fa8000e50420002406200043052000c2e92c00e4
:10fa9000d158200030b22c00b1f407008f87e90064
:10faa0008aff37008b1f780020002000801f78001d
:10fab000c0ec2c00801f780010062000dbf407004b
:10fac0000003eb002505200014062000430520005c
:10fad000c2e92c009158200030b22c00a0f407009d
:10fae000e687570077ff37000200fa00889fbe00c4
:10faf0008a9fbe0080047800010578000204780027
:10fb0000e17c21009140780070c4b30080cf5000a8
:10fb10003c003200e17c21009140780063405000bd
:10fb200080cf50003700320001022000100020007a
:10fb300060e407000000e000320032000900e0004d
:10fb4000630032000a00e00052003200a0c0b3009f
:10fb5000004f7800120020008e007800020078002c
:10fb600069e007000800e000020032001804e0002d
:10fb700041003a000004eb000a00e0001b003200e4
:10fb8000bb0d200069417c008280fb008b8f500000
:10fb90003600320029003c00000c2000808f50000d
:10fba000230032000204e0001a0035000280fb004e
:10fbb0000000d00021302d006080780057c307007e
:10fbc0000001780069407c000080fb000000d0004c
:10fbd00021302d00e0807800100020004ae007006e
:10fbe0000804e8008a0f5400e6ff39008e00780010
:10fbf000a0c0b300806878001200200002007800e6
:10fc000041e007004f05be004f04be000080fa002f
:10fc1000000006000280fb00801f7800c0ef2c006f
:10fc2000801f7800d8f40700e4875700ecff370006
:10fc30004200200031f02c00e7ff3700c00d20000b
:10fc4000808f5000060032000000e800808f5000d6
:10fc5000d4ff3a004200200081f02c00deff370084
:10fc600042002000d1f02c00dbff370042002000d2
:10fc700021f12c00d8ff37000800780027c30700c7
:10fc80000001780088007800100020001ee00700c6
:10fc9000b8ff3700801feb0071f12c00811f780046
:10fca0009006200061f407000003eb0065052000ca
:10fcb000940620004305200082f32c00816120007f
:10fcc00030b22c0026f40700e48757009fff37006e
:10fcd00030f42c00801f78008006200053f40700c9
:10fce0000003eb00e504200084062000430520000b
:10fcf00082f32c004161200030b22c0018f4070080
:10fd00008f87e9008fff37000800fa00889fbe0048
:10fd10008a9fbe008c1f780080047800010578005f
:10fd20000000e0007c003200595090000080fb0091
:10fd30000000d1000080fb00010020006f00600087
:10fd40008000eb000e02780013002000e2ff2f007d
:10fd5000deda070064044700594890000080fb0089
:10fd60000000d1000080fb00010020006f00600057
:10fd70008000eb000802780013002000e2ff2f0053
:10fd8000d2da0700d95090000100d1006f00600066
:10fd90000e01780001003a00b2842c00821f780026
:10fda0000100d1006f00600031f62c0001003a0024
:10fdb000b1842c00811f7800ee9f4400d948900048
:10fdc0000100d1006f0060000801780001003a00d6
:10fdd000b2842c00821f78000100d1006f00600007
:10fde00031f62c0001003a00b1842c00811f78000c
:10fdf000e69f44008a0078000a00e00044003200d8
:10fe0000811f780051f62c00811f78005ef40700f6
:10fe10000006eb00f087570029d892000004e000ac
:10fe20002f0032006865b8000a8444001860920010
:10fe30000080fb000000d1000080fb0001002000da
:10fe40006f0060008000eb000e02780013002000bd
:10fe5000e2ff2f009dda07001860920051f72c0096
:10fe60000078a30001003a00b1842c00811f7800c3
:10fe70000a804400106092000000d1006f00600012
:10fe80008e00780001003a00b1842c00811f7800b8
:10fe90000a804400106092000000d1006f006000f2
:10fea00031f62c0001003a00b1842c00811f78004b
:10feb0000a804400a1112000811f400070f72c002f
:10fec000801f780030f40700ea8757000c06e8002e
:10fed00029d892000080fb00800f5600d1ff35002a
:10fee000f89f4400b90c9000891f780011f82c008d
:10fef000811f780024f40700e68757004f0678003a
:10ff00004f05be004f04be000080fa00000006004e
:10ff1000b1842c00baff370030f92c00801f780024
:10ff2000a0062000c1f307000003eb00e504200059
:10ff3000a406200043052000a2fb2c00d164200071
:10ff400030b22c0086f307008f87e90076ff370078
:10ff50000000fa00889fbe000004be000000e00020
:10ff60000b0032000800be0017000700b80990001f
:10ff700078014400a4002000c1fc2c0010002000e7
:10ff800005d907004f04be000080fa0000000600fb
:10ff900010fd2c00801f7800a0062000a3f30700ae
:10ffa0000003eb00e5042000a40620004305200028
:10ffb00012ff2c002168200030b22c0068f30700eb
:10ffc0008f87e900e7ff37000800fa00889fbe002e
:10ffd0008a9fbe008c1f780080047800010578009d
:10ffe0000000e000da003200595090000080fb0071
:10fff0000000d1000080fb00010020006f006000c5
:020000040001f9
:100000008000eb000e02780013002000e2ff2f00ba
:100010002eda070064044700594890000080fb0076
:100020000000d1000080fb00010020006f00600094
:100030008000eb000802780013002000e2ff2f0090
:1000400022da0700594990000280fb00c500de005b
:10005000e39f6000c700de00811f7800801f7800ea
:100060000000d1006f0060008800780001003a00b5
:10007000c1ff2c00811f78000200d1006f006000da
:1000800031f62c0001003a00f1ff2c00811f7800ae
:10009000e69f440061002000811f780059519000c4
:1000a0000280fb00c500de00e39f6000c700de00a9
:1000b000811f7800801f78000000d1006f00600071
:1000c0008e00780001003a00c1ff2c00811f7800eb
:1000d0000200d1006f00600031f62c0001003a00f0
:1000e000f1ff2c00811f7800ee9f4400600020008b
:1000f000801f78008a0078000a00e0009200320039
:10010000811f780011002d00811f78009ef30700e9
:100110000006eb000f02b10029d892000004e000b5
:10012000350032006865b8000a8444001860920007
:100130000080fb000000d1000080fb0001002000d7
:100140006f0060008000eb000e02780013002000ba
:10015000e2ff2f00ddd90700186092004500de00a5
:10016000e31f6000186092004700de00e11f60009e
:10017000186092000080fb00801f780018609200d9
:100180000000d1006f0060008e00780001003a008e
:10019000c1ff2c00811f78000a804400106092008b
:1001a0000000d1006f00600031f62c0001003a0021
:1001b000f1ff2c00811f78000a804400a11120006b
:1001c000811f400060002000801f78000c04e800c0
:1001d000881f780001062d00811f78006af3070050
:1001e000f28757000806780029d892000080fb00ab
:1001f000800f5400cbff3500595090000080fb0069
:100200004701de00594890000080fb004700de00f7
:10021000d1082d00804f51000400320091092d00bb
:100220000204e00001003a00910a2d00811f7800cd
:1002300039f892000080fb00801f780029f89200b6
:100240000080fb00801f7800a00b2d00801f78002d
:100250004df3070059f892000084fb00e88757002f
:100260000818a3003300320069309100f930910082
:1002700003cf0700809fbe00829fbe0049309100df
:10028000d9309100fece0700809fbe00829fbe0045
:1002900029309100b9309100f9ce0700809fbe004f
:1002a000829fbe0069f092000080fb00801f7800f2
:1002b00059f092000080fb00801f780049f0920006
:1002c0000080fb00801f780039f092000080fb0066
:1002d000801f780029f092000080fb00801f7800ca
:1002e00089389100811f7800093091009930910080
:1002f000e3ce0700809fbe00829fbe006928910068
:10030000f9289100dece0700809fbe00829fbe00cc
:10031000400e2d000828a30001003a00b0842c00f4
:10032000801f7800c00e2d00801f780016f3070094
:100330008f03b1004f0678004f05be004f04be008a
:100340000080fa0000000600b1842c006cff37002a
:10035000f0152d00801f7800a0062000b3f20700e2
:100360000003eb00e5042000a40620004305200064
:1003700032182d007169200030b22c0078f207008d
:100380008f87e90018ff37000000fa0000027800ac
:100390008003eb00e00f110010003d00e1c17b0085
:1003a0008002eb008640280004c069000402d100ee
:1003b0000008a3000100320006026a000380fb006f
:1003c0008001d1008502e800e78f5200f6ff34007b
:1003d0008703e800828f5300f0ff35000482ea00b3
:1003e000040078000080fa00000006000000fa0017
:1003f000800178000001eb006410b800246c2c0030
:10040000840040001100fb00808f51000600320084
:100410000201e800e70f5100f7ff36000000eb0093
:100420000080fa000000060011009000fcff370079
:100430000200fa00a1022000810f500007003200e4
:1004400060412d00801f7800600b200077f20700cc
:100450008f87e9000080fa0000000600d0422d00de
:10046000801f7800c8f207008f87e9008001eb0049
:10047000120020008e007800020078005cdd07008a
:10048000e10f50000b003a00000178008e00780068
:100490001dde0700e10f500004003a0030c0b30039
:1004a0009e4f1000f1ff3a00eaff370030452d0063
:1004b000e4ff370000462d00e2ff37009602fa0005
:1004c000889fbe008a9fbe008c9fbe00800578007a
:1004d0000e007800be0009000018eb000e00780046
:1004e000ee0007000000e000e6003a001b04be003a
:1004f0000800be0028d107000006be0000057800f5
:10050000cf80de007dce07000001be000800be00e7
:10051000fdcd070002002800b35b2400c6cd070014
:100520001dd107000001be00410620000200780036
:100530000dc207000004be002b009000bb0090001d
:10054000108f9a00218f9a0013d1070000027800c3
:10055000800178000000e000c8003500a200200003
:10056000110009000205d8000045b000604f980056
:100570000143b000714f9800110009000204d80037
:10058000000178000245b0000257980002c3b30092
:1005900002c040000c00e0000200350002c5b300bc
:1005a00002c040001057980030062000808f510094
:1005b000ac003c00a2002000110009008204d80019
:1005c0000001780001c3b3000140410020579800aa
:1005d0000400e0009d003500a20020001100090089
:1005e0008204d800010078000043b0003057980022
:1005f00000c6b300005f980030062000808f5100d5
:1006000088003c007c854100e98f510004003c00db
:100610000300e0007f0035006a0720000305450065
:100620001a5f98006120b90034ce07000001be00b7
:100630001e889200ae889200b3cd07000200280009
:10064000b35b24007ccd0700d3d007000001be00bf
:100650004106200002007800c3c107000004be006c
:10066000000578000000e000680035000a00e000a6
:1006700061003500e90f550062003400b00320002e
:10068000800f55005c003c007c0545002a5f980007
:10069000090078000900e000550035007c4040006a
:1006a000305f98006b009000fb009000020020007b
:1006b0000312240076d0070002002000031e24004d
:1006c00092cd0700d5d00700405f98000b0890003e
:1006d0009b089000b0d0070042062000811f7800e0
:1006e000110009000200d80001017800cf00780055
:1006f0000042b000505f98007c414100625f98006a
:10070000b8d4bf00705f9800b9d4bf0000679800ec
:10071000c050210081c00700000578000000e00003
:100720000b00340000c2b300106798000a01780083
:10073000600f2000800f5500010034000001780098
:10074000c1502100200220000e004000b8c0070068
:100750007800470071c00700300f9800e9172000ab
:100760008e84440042112000890078000e00780039
:100770003efa0700000478000000e0001700350092
:10078000000178008900780020002000fffb0700ae
:10079000880f50000c003200801f7800c2462d00e8
:1007a000821f780000072000a0f107001000200041
:1007b000e48757004f06be004f05be004f04be0041
:1007c0000080fa0000000600b1482d000e007800fd
:1007d0004dfd07000000eb00f6ff3700801f78009a
:1007e00051492d00811f7800f0062000eeff3700f0
:1007f0000900ea00a9ff37008a1f7800b14c2d00dc
:10080000f8ff37008a05b000a0ff37000005ea00b6
:1008100096ff3700831f780050502d00801f78000e
:10082000f1ff3700d006200068854100808f51001d
:100830007bff3400300b2000808f5100f5ff3c001f
:1008400082fb2f000285410075ff3700a2002000c7
:10085000110009008204d800010078000045b000b2
:1008600062ff3700a2002000110009008204d800b6
:100870000001780001c5b30053ff37008001ea0092
:1008800036ff3700f202200001542d001000200036
:100890001ddd07000080eb00c6ff37000000fa00f6
:1008a000889fbe008a9fbe008c9fbe008006780095
:1008b0000000e00060003200ae55e2000f003200a0
:1008c00066804600415b210007000900315878002e
:1008d000a01120000d004000c15b21004000090074
:1008e000315878000000eb004f06be004f05be00f7
:1008f0004f04be000080fa000000060001572d00e2
:10090000e049210045d907000000e0004600320020
:1009100082532100124178000204e0003b003200c3
:100920000006eb00210032006865b800c34c2100ce
:10093000030445008084eb008000eb00d2c2b300ca
:1009400068c07800824f50002e0032008100e8001d
:10095000e68f5000faff3400e18f4400230032009c
:10096000c15b210001004500090178008800780082
:100970002fc0070009004400104090000080fb00d9
:1009800002fd2f0082004000335c2100030045007f
:100990000148d0000c06e800825321001241780083
:1009a0000280fb00800f5600dfff35000280fb0055
:1009b0006800b800b35b2100030040001004a000f1
:1009c00002007800fcf5b70082002000e149210018
:1009d000405b2100acbf0700a654d400bbf5b700b4
:1009e00010c0b300aef5b700b5ff3700c05b210003
:1009f000800045000800780005000900b058780024
:100a0000e4ff370081047800d3ff370072572d00d0
:100a1000821f7800a006200004f107000080eb0090
:100a20008f87e900b0ff3700d1592d00811f780072
:100a3000d0062000f8ff3700905c2d00801f780062
:100a4000a0062000f9f007000003eb00e5042000f9
:100a5000a406200043052000f25e2d0001132000b3
:100a600000602d00bef007008f87e90092ff37007d
:100a70000800fa00008fbe006000b8002007980050
:100a80003107980030be80001e02b80031be8000e1
:100a90001e0090000088b9000501780000014100a7
:100aa0009e00780040be80000088b900000141002f
:100ab000820278002e009000be009000840f50004b
:100ac000858f5800070031002e009000be00900076
:100ad00061004000e080480020079800310798003e
:100ae000e8ff37000080fa00000006000000fa006e
:100af000889fbe008a9fbe008c9fbe000004be007f
:100b00008205780003057800040678000000e00004
:100b10007b0032000900e0006b0032000b08a300ec
:100b20005a003a000c00780032e0b7004d03200074
:100b30009d4678000a00780034e0b7000005eb001d
:100b40008b05d100e08f150049003100183b88006b
:100b50000c00780064e7b70040042400003b8800e4
:100b600021042000914078008180fb00c508de0050
:100b700001007800d4f7b70000ceb3004260b700a0
:100b800050c5b30066e7b700a0cab30066e7b70078
:100b900061e7a800c508dd0042c0bf007f406000db
:100ba0000140700042e0b7006007e200feff350040
:100bb00019017800020cbb0040002400003b8800b3
:100bc00021042000914078008180fb00c508de00f0
:100bd00001007800d4f7b70000ceb3004260b70040
:100be00050c5b30066e7b700a0cab30066e7b70018
:100bf00061e7a800c508dd0042c0bf007f4060007b
:100c00000140700042e0b7006007e200feff3500df
:100c100018007800820f500010003200821f780008
:100c2000801f7800881f7800a0602d00801f78004a
:100c3000501720007df0070018037800650520009c
:100c4000541720006304200022662d007108200044
:100c500010672d0042f00700e88757000884e8007d
:100c60008984e8000a05e8008b0f5500b7ff3900ba
:100c70000d00780034e0b7004f06be004f05be00ff
:100c80004f04be000080fa00000006008b1f7800b1
:100c9000a0672d00801f78008005200063f007000a
:100ca0000b03780065052000840520006304200004
:100cb00022662d00b103200010672d0028f00700e8
:100cc000e487570097ff3700d06a2d00801f780017
:100cd0008005200055f007000003eb00e50420002c
:100ce000840520006304200022662d00710320008b
:100cf00010672d001af007008f87e90087ff370083
:100d0000006d2d00801f78008005200047f007004f
:100d10000003eb00e50420008405200063042000ac
:100d200022662d003103200010672d000cf0070013
:100d30008f87e90077ff37000000fa00881f7800ee
:100d400048032000184478008001fd0034e0b7001b
:100d50008001fd0036bf07000800780034e0b700ce
:0c0d60004f0478000080fa00000006003c
:020000040000fa
:020000040001f9
:100d6c00646d0000637400006f6400006567000030
:100d7c003a20000045720000726f0000723a0000c9
:100d8c002061000072670000207000007472000087
:100d9c00206900006e7000002069000073200000c4
:100dac006e7500006c6c0000206f0000722000005b
:100dbc00656d000070740000793a00002025000079
:100dcc00700a0000006400006d630000746f000086
:100ddc00646500006700000075740000696c000019
:100dec00732e000063000000646d0000637400004b
:100dfc006f640000656700003a2000006465000025
:100e0c0067200000256600002069000073200000a8
:100e1c006f750000742000006f66000020720000e7
:100e2c00616e000067650000205b00002d33000040
:100e3c00363000002e2e000033360000305d0000ee
:100e4c000a000000646d0000637400006f64000011
:100e5c00656700003a200000496e000074650000d0
:100e6c00726e0000616c0000204500007272000080
:100e7c006f7200003a2000006d6900006e200000c7
:100e8c002566000020690000732000006f750000cb
:100e9c00742000006f66000020720000616e00007c
:100eac0067650000205b00002d350000392e000026
:100ebc00393900002e2e0000353900002e39000083
:100ecc00395d00000a000000646d000063740000ce
:100edc006f640000656700003a200000496e000056
:100eec0074650000726e0000616c0000204500000b
:100efc00727200006f7200003a20000073650000ef
:100f0c0063200000256600002069000073200000ab
:100f1c006f750000742000006f66000020720000e6
:100f2c00616e000067650000205b00002d3500003d
:100f3c00392e0000393900002e2e00003539000002
:100f4c002e390000395d00000a000000646d0000bd
:100f5c00637400006f640000656700003a200000b5
:100f6c00496e000074650000726e0000616c000038
:100f7c0020450000727200006f7200003a200000e1
:100f8c00706f0000696e0000746500007220000034
:100f9c006d690000736d00006174000063680000ef
:100fac002c200000737400007020000025700000dd
:100fbc00202100003d200000702000002570000062
:100fcc000a000000646d0000637400006f64000090
:100fdc00656700003a200000496e0000746500004f
:100fec00726e0000616c00002045000072720000ff
:100ffc006f7200003a200000436f00006c6f00001d
:10100c006e200000666f0000726d000061740000bd
:10101c000a000000646d0000637400006f6400003f
:10102c00656700003a20000045720000726f0000f6
:10103c00723a0000204400004d430000206600007e
:10104c006f7200006d610000743a000020610000b6
:10105c006c7200006561000064790000206800007b
:10106c00617600006520000073650000636f00006e
:10107c006e64000073200000282500006629000023
:10108c000a000000646d0000637400006f640000cf
:10109c00656700003a20000045720000726f000086
:1010ac00723a0000204400004d430000206600000e
:1010bc006f7200006d610000743a00002061000046
:1010cc006c7200006561000064790000206800000b
:1010dc006176000065200000646500006772000006
:1010ec0065650000732000002825000066290000bb
:1010fc000a000000646d0000637400006f6400005f
:10110c00656700003a20000045720000726f000015
:10111c00723a0000204400004d430000206600009d
:10112c006f7200006d610000743a000020610000d5
:10113c006c7200006561000064790000206800009a
:10114c0061760000652000006d6900006e7500007e
:10115c00746500007320000028250000662900003b
:10116c000a000000646d0000637400006f640000ee
:10117c00656700003a20000045720000726f0000a5
:10118c00723a0000204400004d430000206600002d
:10119c006f7200006d610000743a0000206900005d
:1011ac006e760000616c0000696400002063000032
:1011bc0068610000723a00002025000063200000e6
:1011cc00283000007825000030320000782900001b
:1011dc000a000000646d0000637400006f6400007e
:1011ec00656700003a200000496e0000746500003d
:1011fc00726e0000616c00002045000072720000ed
:10120c006f7200003a200000446f000074740000fc
:10121c0065640000206600006f7200006d610000c4
:10122c00740a0000006400006d630000746f00001d
:10123c0064650000673a0000204900006e740000ed
:10124c00657200006e6100006c20000045720000a9
:10125c00726f0000723a0000206300006f7500008e
:10126c006c640000206e00006f74000020640000ad
:10127c0065740000657200006d6900006e65000009
:10128c00206600006f7200006d610000740a00009f
:10129c00006400006d630000746f00006465000062
:1012ac00673a000020450000727200006f72000067
:1012bc003a200000436f00006c6f00006e200000ad
:1012cc00666f0000726d0000617400003a2000002f
:1012dc006861000073200000616c00007068000001
:1012ec00612000006368000061720000616300000f
:1012fc0074650000727300003a2000005b730000fc
:10130c005d5b0000445d0000444400003a4d000069
:10131c004d3a0000535300005b2e0000462a00009b
:10132c005d0a0000006400006d630000746f000033
:10133c0064650000673a00002045000072720000ee
:10134c006f7200003a200000436f00006c6f0000c9
:10135c006e200000666f0000726d0000617400006a
:10136c003a200000746f00006f2000006d610000d7
:10137c006e7900002070000065720000696f00003b
:10138c00647300003a2000005b7300005d5b00009a
:10139c00445d0000444400003a4d00004d3a00000a
:1013ac00535300005b2e0000462a00005d0a00002b
:1013bc00006400006d630000746f00006465000041
:1013cc00673a000020450000727200006f72000046
:1013dc003a200000436f00006c6f00006e2000008c
:1013ec00666f0000726d0000617400003a2000000e
:1013fc006d750000737400002068000061760000b9
:10140c006520000032200000636f00006c6f00004c
:10141c006e7300003a2000005b7300005d5b0000ff
:10142c00445d0000444400003a4d00004d3a000079
:10143c00535300005b2e0000462a00005d0a00009a
:10144c00006400006d630000746f000064650000b0
:10145c00673a000020450000727200006f720000b5
:10146c003a200000446f00007474000065640000b2
:10147c00206600006f7200006d610000743a00007d
:10148c00206d00007573000074200000686100007e
:10149c0076650000203200002070000065720000ac
:1014ac00696f0000647300003a2000005b73000059
:1014bc005d5b0000445d0000444400002e4d0000c4
:1014cc004d2e00005b4600002a5d00000a0900005a
:1014dc006f720000204400004d43000020660000a5
:1014ec006f7200006d610000742000006d750000cb
:1014fc007374000020680000617600006520000015
:10150c0061740000206c00006561000073740000c1
:10151c00206f00006e650000206f00006620000048
:10152c005b440000644d00006d430000635d0000ef
:10153c0020690000646500006e740000696600009c
:10154c0069650000727300000a000000646d000001
:10155c00637400006f640000656700003a200000af
:10156c0045720000726f0000723a000020550000b6
:10157c006e720000656300006f6700006e6900000a
:10158c007a65000064200000666f0000726d000038
:10159c00617400003a2000006d7500007374000047
:1015ac0020620000652000006f6e000065200000c6
:1015bc006f660000204400006f740000746500002a
:1015cc00642c0000204300006f6c00006f6e000064
:1015dc00206f000072200000444d0000430a000000
:1015ec0000440000644d00006d43000063000000e7
:1015fc004e6e00004565000000530000735700005c
:10160c0077000000646d0000637400006f640000dc
:10161c00656700003a20000045720000726f000000
:10162c00723a0000204400004d4300002066000088
:10163c006f7200006d610000743a000020620000bf
:10164c006f740000682000006d6900006e7500006a
:10165c0073200000282d000029200000616e00007e
:10166c00642000006469000072650000637400006f
:10167c00696f00006e20000063680000617200005a
:10168c002025000063200000636100006e6e0000e6
:10169c006f74000020620000652000007370000071
:1016ac00656300006966000069650000640a00005b
:1016bc00006400006d630000746f0000646500003e
:1016cc00673a000020450000727200006f72000043
:1016dc003a200000444d000043200000666f0000db
:1016ec00726d0000617400003a200000626f00000f
:1016fc0074680000206400006972000065630000db
:10170c00746900006f6e00002063000068610000c7
:10171c00727300002025000063200000616e000041
:10172c00642000002563000020630000616e00004f
:10173c006e6f0000742000006265000020730000d2
:10174c007065000063690000666900006564000054
:10175c000a000000646d0000637400006f640000f8
:10176c00656700003a20000045720000726f0000af
:10177c00723a0000204400004d4300002066000037
:10178c006f7200006d610000742000006d75000028
:10179c007374000020680000617600006520000072
:1017ac0061740000206c000065610000737400001f
:1017bc00206f00006e650000206f000066200000a6
:1017cc005b440000644d00006d430000635d00004d
:1017dc0020690000646500006e74000069660000fa
:1017ec0069650000727300000a0900006f72000046
:1017fc00204400006f740000746500006420000039
:10180c00666f0000726d0000617400003a200000e9
:10181c00666f0000756e000064200000696c0000ab
:10182c006c650000676100006c20000063680000bc
:10183c00617200006163000074650000723a000080
:10184c00205b0000735d00005b4400005d44000001
:10185c00442e00004d4d00002e5b0000462a000077
:10186c005d0a0000006400006d630000746f0000ee
:10187c0064650000673a00002045000072720000a9
:10188c006f7200003a200000746f00006f2000009f
:10189c006d6100006e790000206d0000696e000023
:1018ac007573000020730000696700006e73000000
:1018bc003a200000256400003a2000006f6e000002
:1018cc006c790000206f00006e650000206900003c
:1018dc0073200000616c00006c6f000077650000e5
:1018ec00640a0000000a0000446500006320000048
:1018fc002048000065780000207c000020200000bb
:10190c003020000020310000202000003220000098
:10191c00203300002020000034200000203500007f
:10192c00202000003620000020370000202000007e
:10193c00202000003820000020390000202000006a
:10194c0061200000206200002020000063200000c5
:10195c0020640000202000006520000020660000ac
:10196c00207c0000203000003132000033340000b5
:10197c003536000037380000396100006263000022
:10198c0064650000660a000000300000313200007f
:10199c003334000035360000373800003961000060
:1019ac00626300006465000066000000686500006a
:1019bc0078640000756d0000703a0000202500006e
:1019cc0073250000736200007566000066650000f8
:1019dc00722000006164000064720000203000007e
:1019ec0078250000702c0000206c0000656e000053
:1019fc0067740000682000002564000020280000a7
:101a0c003078000025780000293a00000a00000018
:101a1c0025340000642000002530000034780000dc
:101a2c007c200000003a00002000000068650000e7
:101a3c0078640000756d0000703a000020620000b0
:101a4c00756600006665000072200000616400008d
:101a5c00647200002030000078250000702c00001b
:101a6c00206c0000656e00006774000068200000a8
:101a7c002564000020280000307800002578000044
:101a8c00293a00000a0000002573000025730000ad
:101a9c006c6500006e670000746800002025000073
:101aac006420000028300000782500007829000010
:101abc003a0a0000006800006578000064750000b8
:101acc006d7000003a2000006c6500006e6700002d
:101adc0074680000202500006420000028300000fd
:101aec0078250000782900003a0a0000006c0000fc
:101afc00656e00006774000068200000256400001b
:101b0c00202800003078000025780000293a0000d9
:101b1c000a0000006865000078640000756d000024
:101b2c00703a000020610000726700002070000015
:101b3c0074720000206200007020000069730000c5
:101b4c00206e0000756c00006c0a0000006800003c
:101b5c0065780000647500006d700000006800007e
:101b6c0065780000647500006d7000003a2000007c
:101b7c00656d000070740000792000006275000033
:101b8c0066660000657200000a00000061740000c7
:101b9c006f6c00006e3a000020450000727200006d
:101bac006f7200003a200000617200006720000094
:101bbc006d610000782000003c200000313a0000ec
:101bcc0020250000640a000000610000746f000012
:101bdc006c6e000000610000746f00006c6e000001
:101bec003a20000045720000726f0000723a00004b
:101bfc002061000072670000207000007472000009
:101c0c00206900006e20000069730000206e000047
:101c1c00756c00006c0a0000006c0000746f000012
:101c2c00616e00003a200000617200006720000025
:101c3c006e20000069730000206900006e760000c1
:101c4c00616c0000696400003a200000256400000b
:101c5c000a0000006c7400006f6100006e00000050
:101c6c006c7400006f6100006e3a0000206300008d
:101c7c006f6e00007665000072730000696f0000e3
:101c8c006e2000006e6f000074200000636f000077
:101c9c006d7000006c650000746500003a20000057
:101cac00696e00007075000074200000256c000047
:101cbc00642c000020770000696400007468000048
:101ccc0020250000640a0000006c0000746f000006
:101cdc00616e00003a200000617200006720000075
:101cec0070740000722000006275000066700000c5
:101cfc0020690000732000006e7500006c6c000001
:101d0c000a000000726100006e670000655f000051
:101d1c00617a0000696d000075740000683a00007b
:101d2c0020450000727200006f7200003a20000023
:101d3c0061720000672000007074000072200000c7
:101d4c00617a00007020000069730000206e0000b2
:101d5c00756c00006c0a000000720000616e0000df
:101d6c00676500005f6100007a6900006d75000016
:101d7c007468000000720000616e0000676500006e
:101d8c005f6100007a6900006d75000074680000e6
:101d9c003a20000045720000726f0000723a000099
:101dac002061000072670000207000007472000057
:101dbc0020720000616e000067650000702000005a
:101dcc0069730000206e0000756c00006c0a000046
:101ddc000000000000000000211000004220000064
